:100000000C94180D0C94F0150C9421160C945216A7
:100010000C9483160C94B4160C94E5160C941617D5
:100020000C9447170C94450D0C94450D0C94450DFC
:100030000C94450D0C94450D0C94450D0C94450DF8
:100040000C94450D0C94D4610C94450D0C94450D05
:100050000C94450D0C94450D0C946E6A0C940F1382
:100060000C94450D0C9438380C94450D0C94450DAA
:100070000C94450D0C94450D0C94450D0C94450DB8
:100080000C94450D0C94450D0C94450D0C94450DA8
:100090000C94450D0C94450D0C94450D0C94450D98
:1000A0000C94450D0C94450D0C94450D0C94450D88
:1000B0000C94450D0C94450D0C94450D0C94450D78
:1000C0000C94450D0C94450D0C94450D0C94450D68
:1000D0000C94450D0C94450D0C94450D0C94450D58
:1000E0000C94450D084AD73B3BCE016E84BCBFFD46
:1000F000C12F3D6C74319ABD56833DDA3D00C77FF8
:1001000011BED9E4BB4C3E916BAAAABE0000008090
:100110003F05A84CCDB2D44EB93836A9020C50B91F
:10012000918688083CA6AAAA2ABE000000803F004B
:10013000002100240027002A002D00300033000198
:10014000010000040107010A010000220025002827
:10015000002B002E003100340002010000050108D0
:10016000010B01000020002300260029002C002F95
:100170000032000001000003010601090105050528
:1001800005070508080808020202020A0A0808040E
:10019000040404010101010101010103030303033C
:1001A000030303040707070C0C0C0C0C0C0C0C02CB
:1001B00002020206060606060606060B0B0B0B0BD2
:1001C0000B0B0B01021020200808102040102040CB
:1001D000800201020108040201010204081020400B
:1001E0008080402010080402018004020180402029
:1001F0001008040201080402010102040810204052
:100200008001020408102040800000090A02080B47
:100210000C0D0706030401000000000000000000B0
:1002200000000000000000000000000000000000CE
:10023000000000000011100F00000000000000008E
:100240000000000000000000000000000000006549
:1002500063686F3A004572726F723A0053544F50A0
:100260005045442E20005072696E7465722073747C
:100270006F707065642064756520746F206572729C
:100280006F72732E204669782074686520657272DB
:100290006F7220616E6420757365204D3939392085
:1002A000746F20726573746172742E202854656DAA
:1002B000706572617475726520697320726573650B
:1002C000742E2053657420697420616674657220F1
:1002D00072657374617274696E6729004B494C4C86
:1002E00045442E20005072696E7465722068616CFE
:1002F0007465642E206B696C6C28292063616C6CBA
:10030000656421006F6B00526573656E643A20006E
:100310002200556E6B6E6F776E20636F6D6D616E30
:10032000643A202200486F74656E64206F666673BD
:100330006574733A007A5F6D61783A20007A5F6D78
:10034000696E3A2000795F6D61783A2000795F6DBF
:10035000696E3A2000785F6D61783A2000785F6DB1
:10036000696E3A20005A3A00593A0020436F756E80
:100370007420583A2000453A005A3A00593A005839
:100380003A004649524D574152455F4E414D453A1C
:100390004D61726C696E2056313B20537072696EEC
:1003A0007465722F6772626C206D6173687570205E
:1003B000666F722067656E36204649524D5741522E
:1003C000455F55524C3A687474703A2F2F666972C3
:1003D0006D776172652E756C74696D616B65722ED7
:1003E000636F6D2050524F544F434F4C5F564552F0
:1003F00053494F4E3A312E30204D414348494E45E6
:100400005F545950453A556C74696D616B65722043
:1004100045585452554445525F434F554E543A3215
:100420000A0042656420646F6E652E0020423A0027
:1004300020453A00543A0042656420486561746979
:100440006E672E0048656174696E6720646F6E6523
:100450002E0020573A0020453A00543A0048656182
:1004600074696E672E2E2E002042403A0020403ADA
:1004700000202F0020423A00202F006F6B20543ABA
:10048000002569206D696E2C202569207365630045
:10049000456E642066696C65206C69737400426502
:1004A00067696E2066696C65206C697374004E6FB5
:1004B000206D6F76652E00526573756D696E6720CD
:1004C0007072696E74005761697420666F7220756E
:1004D0007365722E2E2E00536C6565702E2E2E00C5
:1004E000000000000000000000000000000000000C
:1004F000000000000000000000004D4300004D43DC
:100500000000484300004D4300004D4300004843B5
:100510000000A0400000A0400000803FFFFFFF253A
:100520006920686F757273202569206D696E757416
:10053000657300446F6E65207072696E74696E67D2
:100540002066696C650053544F505045442E20007E
:100550005072696E7465722073746F707065642078
:1005600064756520746F206572726F72732E2046F9
:10057000697820746865206572726F7220616E649C
:1005800020757365204D39393920746F2072657379
:10059000746172742E202854656D70657261747573
:1005A00072652069732072657365742E20536574BB
:1005B000206974206166746572207265737461725B
:1005C00074696E6729006F6B004E6F204C696E6511
:1005D000204E756D62657220776974682063686566
:1005E000636B73756D2C204C617374204C696E6560
:1005F0003A20004E6F20436865636B73756D2077FA
:10060000697468206C696E65206E756D6265722C08
:10061000204C617374204C696E653A2000636865F4
:10062000636B73756D206D69736D617463682C20E5
:100630004C617374204C696E653A20004C696E659C
:10064000204E756D626572206973206E6F74204C48
:10065000617374204C696E65204E756D6265722BF6
:10066000312C204C617374204C696E653A20004D2A
:1006700031313000446F6E6520736176696E67209A
:1006800066696C652E006F6B004D3239002020507A
:100690006C616E6E657242756666657242797465EC
:1006A000733A20002046726565204D656D6F727942
:1006B0003A20004D61722020312032303133004326
:1006C0006F6D70696C65643A2000284461766964D6
:1006D00020427261616D2900207C20417574686F31
:1006E000723A20004D6172202031203230313320A7
:1006F00031323A33343A343800204C617374205527
:100700007064617465643A2000556C74696D616B46
:1007100065723A2031332E30332028323530303074
:10072000305F6475616C29004D61726C696E2000E8
:1007300020536F667477617265205265736574002B
:10074000205761746368646F672052657365740035
:100750002042726F776E206F7574205265736574D6
:10076000002045787465726E616C20526573657403
:1007700000506F7765725570007374617274002257
:1007800000656E717565696E672022002200656ED6
:10079000717565696E672022007C3C3E5E2B3D3F93
:1007A0002F5B5D3B2C2A225C006563686F3A00205A
:1007B000746F6F206C6F6E672065787472757369E3
:1007C0006F6E2070726576656E7465640020636F6D
:1007D0006C6420657874727573696F6E20707265D1
:1007E00076656E7465640045313A200045303A20E4
:1007F000005A3A2000593A2000583A20004D53310F
:100800002C4D53322050696E730A0024F404D92011
:100810001BC40C5C0E9804C4095F0265077101F4E7
:1008200005F900FB04B30048048700C103690058C0
:1008300003550003034500BE023A00840231005311
:10084000022A002902250004022000E4011C00C83D
:10085000011900AF01170098011400840113007101
:100860000110006101100051010E0043010D00361E
:10087000010B002B010B0020010B00150109000CDE
:1008800001090003010800FB000800F3000800EB69
:10089000000700E4000600DE000600D8000600D2D3
:1008A000000600CC000500C7000500C2000500BD21
:1008B000000400B9000400B5000400B1000400AD5C
:1008C000000400A9000400A5000300A20003009F8B
:1008D0000004009B000300980003009500020093B1
:1008E000000300900003008D0002008B00030088CD
:1008F0000002008600020084000300810002007FE5
:100900000002007D0002007B0002007900020077F7
:100910000001007600020074000200720001007104
:100920000002006F0002006D0001006C0002006A0E
:100930000001006900020067000100660001006517
:10094000000100640002006200010061000100601B
:100950000001005F0002005D0001005C0001005B1F
:100960000001005A00010059000100580001005721
:100970000001005600010055000100540001005321
:10098000000000530001005200010051000100501E
:100990000001004F0001004E0000004E0001004D1C
:1009A0000001004C0001004B0000004B0001004A18
:1009B0000001004900010048000000480001004714
:1009C000000100460000004600010045000000450F
:1009D0000001004400010043000000430001004208
:1009E0000000004200010041000000410001004001
:1009F0000001003F0000003F0001003E0000003EFB
:100A00000001003D0000003D0001003C0000003CF2
:100A10000000003C0001003B0000003B0001003AE8
:100A20000000003A000100390000003900010038E0
:100A300000000038000000380001003700000037D7
:100A400000010036000000360000003600010035CD
:100A500000000035000000350001003400000034C3
:100A600000000034000100330000003300000033B8
:100A700000010032000000320000003200010031AD
:100A800000000031000000310001003000000030A3
:100A9000000000300001002F0000002F0000002F98
:100AA0000000002F0001002E0000002E0000002E8C
:100AB0000001002D0000002D0000002D0000002D81
:100AC0000001002C0000002C0000002C0000002C75
:100AD0000001002B0000002B0000002B0000002B69
:100AE0000001002A0000002A0000002A0000002A5D
:100AF0000001002900000029000000290000002951
:100B00000000002900010028000000280000002843
:100B10000000002800000028000100270000002736
:100B20000000002700000027000000270001002629
:100B3000000000260000002600000026000000261D
:100B40000001002500000025000000250000002510
:100B50000000002500000025000100240000002402
:100B600000000024000000240000002400010023F5
:100B700000000023000000230000002300000023E9
:100B800000000023000000230001002200000022DA
:100B900000000022000000220000002200000022CD
:100BA00000010021000000210000002100000021C0
:100BB00000000021000000210000002100010020B1
:100BC00000000020000000200000002000000020A5
:100BD0000000002000000020000000200001001F95
:100BE0000000001F0000001F0000001F0000001F89
:100BF0000000001F0000001F0001001E0000001E7A
:100C00000000001E0000001E00000024F4D430503C
:100C1000C38E20C2A24017828B7011127A910D816F
:100C20006CD90AA861E108C7586607615143061EDE
:100C30004B5D05C145A7041A411104093D98037194
:100C40003931034036DB0265339102D430540280DF
:100C50002E1D02632CEE01752AC501B028A00110DB
:100C60002781018F2564012B244B01E0223401AC44
:100C7000211F018D200D01801FFC00841EED0097B7
:100C80001DDF00B81CD200E61BC600201BBC0064A0
:100C90001AB200B219A8000A19A0006A189900D166
:100CA00017910040178B00B516840031167E00B3F3
:100CB0001579003A157300C7146F0058146A00EED6
:100CC0001366008813630025135E00C7125B006C77
:100CD00012570015125400C111510070114F00211C
:100CE000114B00D61049008D1047004610440002F9
:100CF000104200C00F4000800F3E00420F3C000633
:100D00000F3B00CB0E3800930E37005C0E350027EA
:100D10000E3400F30D3200C10D3100900D30006033
:100D20000D2E00320D2D00050D2C00D90C2B00AE20
:100D30000C2900850C29005C0C2700350C27000EBF
:100D40000C2600E80B2400C40B2400A00B23007D1C
:100D50000B23005A0B2100390B2100180B2000F83F
:100D60000A1F00D90A1E00BB0A1E009D0A1D008032
:100D70000A1D00630A1C00470A1B002C0A1B0011F5
:100D80000A1A00F7091A00DD091900C4091900AB95
:100D9000091900920917007B091800630917004C14
:100DA00009160036091600200916000A091500F573
:100DB000081500E0081400CC081400B8081400A4BA
:100DC000081400900813007D0812006B08130058E7
:100DD00008120046081200340811002308110012FE
:100DE00008110001081100F0071000E0071000D002
:100DF000071000C0071000B0070F00A107100091F6
:100E0000070E0083070F0074070F0065070E0057D9
:100E1000070E0049070E003B070D002E070E0020AD
:100E2000070D0013070D0006070D00F9060C00ED75
:100E3000060D00E0060C00D4060C00C8060C00BC31
:100E4000060C00B0060C00A4060B0099060C008DE1
:100E5000060B0082060B0077060B006C060B006188
:100E6000060A0057060B004C060A0042060A003824
:100E7000060A002E060A0024060A001A060A0010B6
:100E800006090007060A00FD050900F4050900EB44
:100E9000050900E2050900D9050900D0050900C7C8
:100EA000050900BE050900B5050800AD050800A547
:100EB0000509009C050800940508008C05080084BD
:100EC0000508007C050800740508006C050700652E
:100ED0000508005D050700560508004E0507004798
:100EE0000507004005080038050700310507002AFE
:100EF000050700230507001C050600160507000F5F
:100F00000507000805060002050700FB040600F5BA
:100F1000040700EE040600E8040600E2040700DB14
:100F2000040600D5040600CF040600C9040600C369
:100F3000040600BD040600B7040600B1040500ACB9
:100F4000040600A6040600A00405009B0406009504
:100F5000040500900406008A04050085040500804D
:100F60000406007A04050075040500700405006B92
:100F700004050066040500610405005C04050057D3
:100F8000040500520405004D040500480405004313
:100F90000405003E0404003A040500350405003051
:100FA0000404002C04050027040400230405001E8B
:100FB0000404001A04040016040500110404000DC2
:100FC000040400090405000404040000040400FCF7
:100FD000030400F8030400F4030400F0030400EC2D
:100FE000030400E8030400E4030400E0030400DC5D
:100FF000030400D8030400D4030400D0030400CC8D
:10100000030400C8030300C50303006563686F3A67
:1010100000656E6473746F7073206869743A205A47
:1010200000205A3A00656E6473746F7073206869AB
:10103000743A20590020593A00656E6473746F70D9
:1010400073206869743A20580020583A00656E642D
:1010500073746F7073206869743A20004572726F00
:10106000723A004572723A204D415854454D502015
:101070004245440054656D706572617475726520F7
:101080006865617465642062656420737769746360
:10109000686564206F66662E204D415854454D505A
:1010A000207472696767657265642021210045724A
:1010B000723A204D494E54454D50003A20457874BF
:1010C0007275646572207377697463686564206FF4
:1010D00066662E204D494E54454D50207472696706
:1010E00067657265642021004572723A204D41584F
:1010F00054454D50003A20457874727564657220ED
:101100007377697463686564206F66662E204D414D
:101110005854454D50207472696767657265642044
:101120002100202D20496E76616C696420657874F9
:101130007275646572206E756D626572202100653E
:1011400063686F3A0048656174696E67206661691B
:101150006C656400504944204175746F74756E6508
:101160002066696E6973686564202120506C616334
:101170006520746865204B702C204B6920616E647B
:10118000204B6420636F6E7374616E747320696E9C
:101190002074686520636F6E666967757261746933
:1011A0006F6E2E6800504944204175746F74756EDF
:1011B00065206661696C6564212074696D656F7571
:1011C000740020403A006F6B20543A006F6B20424D
:1011D0003A00504944204175746F74756E652066FD
:1011E00061696C6564212054656D70657261747508
:1011F000726520746F206869676800204B643A202C
:1012000000204B693A2000204B703A200020436CAC
:10121000617369632050494420002054753A2000CE
:10122000204B753A2000206D61783A2000206D69CE
:101230006E3A200020643A200020626961733A20EF
:10124000004D383420582059205A204500656368E5
:101250006F3A0043616E6E6F7420656E7465722024
:101260007375626469723A20004D3234004D323336
:10127000202573006175746F25692E6700457272B1
:101280006F723A006572726F722077726974696E5C
:101290006720746F2066696C65004E6F742053443C
:1012A000207072696E74696E67002F00534420705D
:1012B00072696E74696E67206279746520002E0011
:1012C00044656C6574696F6E206661696C65642C39
:1012D0002046696C653A200046696C652064656C3F
:1012E000657465643A002E006F70656E20666169F2
:1012F0006C65642C2046696C653A200057726974ED
:10130000696E6720746F2066696C653A20002E0054
:101310006F70656E206661696C65642C2046696C2F
:10132000653A20002E006F70656E206661696C65FD
:10133000642C2046696C653A200046696C65207310
:10134000656C6563746564002053697A653A2000B2
:1013500046696C65206F70656E65643A20002E00EA
:101360006F70656E206661696C65642C2046696CDF
:10137000653A200053442063617264206F6B006FF4
:1013800070656E526F6F74206661696C656400767B
:101390006F6C756D652E696E6974206661696C6528
:1013A0006400534420696E6974206661696C00654D
:1013B00063686F3A0053746F726564207365747468
:1013C000696E6773207265747265697665643A0048
:1013D0002044002049002020204D3330312050008F
:1013E0005049442073657474696E67733A00205ADB
:1013F0000020590020204D323036205800486F6DB3
:1014000065206F666673657420286D6D293A00202B
:101410004500205A0020580020420020540020207F
:101420004D323035205300416476616E636564202F
:101430007661726961626C65733A20533D4D696EE5
:1014400020666565647261746520286D6D2F73294F
:101450002C20543D4D696E2074726176656C206657
:101460006565647261746520286D6D2F73292C2069
:10147000423D6D696E696D756D207365676D656E52
:10148000742074696D6520286D73292C20583D6D7A
:101490006178696D756D207859206A65726B2028B6
:1014A0006D6D2F73292C20205A3D6D6178696D7503
:1014B0006D205A206A65726B20286D6D2F7329008C
:1014C00020540020204D32303420530041636365A6
:1014D0006C65726174696F6E3A20533D6163636538
:1014E0006C65726174696F6E2C20543D7265747204
:1014F00061637420616363656C65726174696F6EAA
:1015000000204500205A0020590020204D32303163
:101510002058004D6178696D756D20416363656C7D
:1015200065726174696F6E20286D6D2F7332293A70
:1015300000204500205A0020590020204D32303331
:101540002058004D6178696D756D2066656564721F
:101550006174657320286D6D2F73293A0020450052
:10156000205A0020590020204D3932205800537451
:101570006570732070657220756E69743A005365EA
:101580007474696E67732053746F726564002D2DD7
:101590003A2D2D002D2D2D005344002059000120FF
:1015A000000120004E6F2043617264004361726449
:1015B000204D656E750053746F70205072696E74A3
:1015C00000526573756D65205072696E74005061CC
:1015D000757365205072696E7400436F6E74726F1C
:1015E0006C00507265706172650054756E650057CD
:1015F0006174636800052E2E004D61696E004D32E6
:1016000034004D3233202573004D38342058205992
:10161000205A2045004669726D77617265207665B3
:101620007273696F6E00526573746F7265204661E4
:10163000696C73616665004C6F6164206D656D6FE8
:1016400072790053746F7265206D656D6F727900E9
:101650004D6F74696F6E0054656D7065726174755D
:101660007265004D61696E004D617220203120323B
:101670003031332031323A33343A35330032353079
:101680003030305F6475616C00556C74696D616BEE
:1016900065723A2031332E3033004669726D7761BE
:1016A00072652076657273696F6E0045737465703C
:1016B000732F6D6D004573746570732F6D6D005AD7
:1016C00073746570732F6D6D005A73746570732F2A
:1016D0006D6D005973746570732F6D6D005973745F
:1016E0006570732F6D6D005873746570732F6D6D19
:1016F000005873746570732F6D6D00412D726574A1
:101700007261637400412D7265747261637400418B
:101710006D6178206500416D6178206500416D61E3
:1017200078207A00416D6178207A00416D617820DF
:101730007900416D6178207900416D6178207800F1
:10174000416D61782078005654726176206D696E23
:10175000005654726176206D696E00566D696E0098
:10176000566D696E00566D6178206500566D617822
:10177000206500566D6178207A00566D6178207A78
:1017800000566D6178207900566D61782079005699
:101790006D6178207800566D6178207800567879F0
:1017A0002D6A65726B005678792D6A65726B0041FF
:1017B0006363656C00416363656C00436F6E7472B4
:1017C0006F6C00507265686561742041425320431C
:1017D0006F6E66005072656865617420504C4120E0
:1017E000436F6E66005049442D43005049442D43D9
:1017F000005049442D44005049442D440050494470
:101800002D49005049442D49005049442D50005065
:1018100049442D500046616E207370656564004632
:10182000616E207370656564004E6F7A7A6C653204
:10183000004E6F7A7A6C6532004E6F7A7A6C650072
:101840004E6F7A7A6C6500436F6E74726F6C0053E2
:10185000746F7265206D656D6F7279004E6F7A7A64
:101860006C65004E6F7A7A6C650046616E2073700D
:101870006565640046616E2073706565640054653B
:101880006D70657261747572650053746F72652056
:101890006D656D6F7279004E6F7A7A6C65004E6F70
:1018A0007A7A6C650046616E2073706565640046E7
:1018B000616E2073706565640054656D706572615A
:1018C00074757265004D6F76652041786973004DBF
:1018D0003130342053300A4D3134302053300043FE
:1018E0006F6F6C646F776E0050726568656174200D
:1018F000414253005072656865617420504C41004C
:10190000473238004175746F20486F6D65004D385F
:10191000340044697361626C65205374657070654E
:101920007273004D61696E004D6F766520302E3107
:101930006D6D004D6F766520316D6D004D6F766574
:101940002031306D6D0050726570617265004578B0
:10195000747275646572004D6F7665205A004D6F24
:1019600076652059004D6F76652058004D6F76657D
:101970002041786973004578747275646572005A05
:101980000059005800466C6F7700466C6F77004630
:10199000616E2073706565640046616E20737065CA
:1019A0006564004E6F7A7A6C6532004E6F7A7A6C9D
:1019B0006532004E6F7A7A6C65004E6F7A7A6C658C
:1019C000005370656564005370656564004D61691E
:1019D0006E00436172642072656D6F7665640043CA
:1019E00061726420696E73657274656400494E4665
:1019F000494E4954594E414ECDCCCC3D0AD7233C9B
:101A000017B7D13877CC2B329595E6241FB14F0A02
:101A1000000020410000C84200401C4620BCBE4CD3
:101A2000CA1B0E5AAEC59D746E18CC3856BC6718CA
:101A300011241FBECFEFD1E2DEBFCDBF00E00CBF4F
:101A400014E0A0E0B2E0E2EEFCE801E00BBF02C06F
:101A500007900D92AE38B107D9F71BBE10E1AEE882
:101A6000B4E001C01D92A23DB107E1F71AE1CEE258
:101A7000DAE104C02297FE010E9416C6C832D107DF
:101A8000C9F70E94F6C00C9464C60C940000A0E054
:101A9000B0E0EDE4FDE00C9433C6EC015B016115B0
:101AA000710519F0FB0191838083F9908F2D90E0EF
:101AB0000E941AC6892BC9F7FDE2FF1621F4F9909E
:101AC000EE24E39405C02BE2F21609F4F990EE241B
:101AD0008E0101501040C8016DEE79E143E050E005
:101AE0000E94DD0F892B01F58E010E5F1F4FC8018B
:101AF00060EF79E145E050E00E94DD0F892B19F499
:101B00008E01095F1F4FA114B10419F0F501118373
:101B10000083E0FC04C070E090E080E814C070E056
:101B200090E080E86FEF08C1C80165EF79E143E01C
:101B300050E00E94DD0F892B69F4A114B10429F44F
:101B400070E090E080EC6FE7F7C02296F501D1835A
:101B5000C083F6CF8824992440E050E060E070E034
:101B6000EF2DE053EA30A0F5F2E0EF2A8E2D90E061
:101B70009C0128703070E2FE06C0232B79F5089492
:101B8000811C911C2BC0232B19F00894810891080B
:101B9000DB01CA0112E0880F991FAA1FBB1F1A950B
:101BA000D1F7480F591F6A1F7B1F440F551F661F2F
:101BB000771F4E0F511D611D711D483929E95207CC
:101BC00029E9620729E1720748F084E0E82A06C0A3
:101BD000EE3F31F4E3FC39C098E0E92AF990C0CF38
:101BE000E53311F0E53189F529912D3219F4E0E161
:101BF000EE2A05C02B3219F081E090E003C0299154
:101C000082E090E0E22FE053EA3018F0C81BD90BD5
:101C10001CC020E030E0FCE020383F075CF4C90144
:101C2000880F991F880F991F280F391F220F331F04
:101C30002E0F311DE991E053EA3068F3E4FE03C052
:101C4000309521953F4F820E931ECE2CDD24E1FE70
:101C500007C0A114B10421F02197F501D183C083FD
:101C6000CB01BA010E947FC27B018C01F3E0CF223D
:101C7000DD2423E0C216D10421F417FB109517F9D7
:101C8000109557016801C801B70120E030E040E03D
:101C900050E00E94DFC1882309F44AC097FE0DC0BE
:101CA0002CE0E22E2AE1F22E9094819491089394F4
:101CB000C0E2D0E000E010E012C094E2E92E9AE128
:101CC000F92EF6CFF7012591359145915491C60132
:101CD000B5010E94BFC45B016C018C1A9D0A8C1671
:101CE0009D0684F7D595C7950F5F1F4F06301105E8
:101CF00029F08CEF9FEFE80EF91EF1CFC501D60158
:101D00007C018D018C2D880F8D2D881F8F3F51F008
:101D1000C601B50120E030E040E050E00E94DFC1A4
:101D2000882331F482E290E09093D1108093D01018
:101D30007E2D9F2D802F612F272F392F482F562F33
:101D4000B901CA01CDB7DEB7ECE00C944FC62F92B3
:101D50003F925F926F927F928F929F92AF92BF92CB
:101D6000CF92DF92EF92FF920F931F93CF93DF9367
:101D70008C011B01EA016115710519F0FB019183CA
:101D80008083209749F0CE010297839728F020E0C6
:101D900030E040E050E0F6C0F801A1908F018A2DBC
:101DA00090E00E941AC6892BB9F7FDE2AF1631F414
:101DB000F801A1908F015524539407C0FBE2AF16A0
:101DC00019F4F801A1908F015524209719F0C03122
:101DD000D105C1F4F0E3AF1679F4F80180818837BA
:101DE00011F0883549F4F801A1800E5F1F4FF2E031
:101DF0005F2AC0E1D0E006C0209721F480E3A81656
:101E0000E9F427C0C830D10531F1C930D10524F437
:101E1000C230D10531F50CC0CA30D10589F0C031CE
:101E2000D105F9F4C12CD12CE12CB8E0FB2E28C04F
:101E3000C12CD12CE12CA0E4FA2E22C0CAE0D0E0C3
:101E4000FCECCF2EFCECDF2EFCECEF2EFCE0FF2EAA
:101E500017C0C8E0D0E0C12CD12CE12CE0E1FE2E6F
:101E60000FC09E01442737FD4095542F60E070E07D
:101E700080E090E80E94D7C5C901DA016C017D01BC
:101E800020E030E040E050E060E03E01882477FC54
:101E90008094982C70EDB72EBA0CE9E0EB1570F435
:101EA0008A2D81548A3118F499ECB92E06C08A2DF6
:101EB00081568A3150F589EAB82EBA0C8B2D90E004
:101EC0008C179D0714F56F3FE1F0C216D306E406A8
:101ED000F506B0F0CA01B901A40193010E9491C5B1
:101EE0009B01AC012B0D311D411D511D2130F0E036
:101EF0003F07F0E04F07F0E85F0710F461E001C032
:101F00006FEFF801A1908F01C5CF2114310481F04A
:101F1000662331F001501040F1011183008308C0A5
:101F200051FE1AC002501040F1011183008314C009
:101F300067FF12C050FC05C02FEF3FEF4FEF5FE788
:101F400004C020E030E040E050E882E290E090936E
:101F5000D1108093D01016C050FE08C05095409507
:101F6000309521953F4F4F4F5F4F0CC057FF0AC030
:101F700082E290E09093D1108093D0102FEF3FEF4A
:101F80004FEF5FE7B901CA01DF91CF911F910F9128
:101F9000FF90EF90DF90CF90BF90AF909F908F9089
:101FA0007F906F905F903F902F900895FB01DC0130
:101FB00005900D920020E1F70895FB01DC014150EE
:101FC000504088F08D9181341CF08B350CF4805E8C
:101FD000659161341CF06B350CF4605E861B6111F9
:101FE00071F3990B0895881BFCCFFB01DC01415074
:101FF000504048F005900D920020C9F701C01D9295
:1020000041505040E0F70895FB0155915523A9F048
:10201000BF01DC014D9145174111E1F759F4CD01A4
:102020000590002049F04D9140154111C9F3FB0185
:102030004111EFCF81E090E001970895FB01DC01B1
:1020400004C08D910190801921F441505040C8F78F
:10205000881B990B0895FB01DC0102C001900D92D1
:1020600041505040D8F70895FB01DC010D9000204D
:10207000E9F7119701900D920020E1F70895FC0116
:102080008191861721F08823D9F7992708953197F0
:10209000CF010895FB01DC0101900D920020E1F7D2
:1020A0000895FB01DC014150504030F08D910190CA
:1020B000801919F40020B9F7881B990B0895FB01CA
:1020C000DC014150504048F001900D920020C9F7CA
:1020D00001C01D9241505040E0F70895AEE0B0E0DD
:1020E000E4E7F0E10C943BC60E891F898EE08C83F7
:1020F0001A8309838FEF9FE79E838D839E01265E5F
:102100003F4FCE010196688D798DA9010E949210F2
:102110002F813885020F131FF80110822E96E4E0FC
:102120000C9457C6ABE0B0E0E8E9F0E10C942DC6A2
:102130003C012B015A01FC0117821682838181FD2B
:1021400003C06FEF7FEFC6C19AE0892E1E0108948D
:10215000211C311CF3012381F20123FD859123FF12
:1021600081912F01882309F4B2C1853239F423FD0E
:10217000859123FF81912F01853229F490E0B301ED
:102180000E948512E7CF982FFF24EE249924FFE1C7
:10219000FF15D0F09B3269F09C3228F4903259F050
:1021A000933291F40EC09D3249F0903369F441E0CE
:1021B00024C052E0F52A84E0F82A28C098E0F92AE1
:1021C00025C0E0E1FE2A22C0F7FC29C0892F8053F8
:1021D0008A3070F4F6FE05C0989C902C1124980E5D
:1021E00015C0E89CE02C1124E80EF0E2FF2A0EC096
:1021F0009E3229F4F6FC6BC140E4F42A07C09C36F9
:1022000019F450E8F52A02C0983649F4F20123FD8A
:10221000959123FF91912F01992309F0B8CF892F30
:102220008554833018F08052833038F444E050E015
:10223000A40EB51E5FE359830FC0933631F0933778
:1022400079F0933509F056C020C0F501808189836B
:1022500042E050E0A40EB51E610101E010E012C0A2
:10226000F501C080D180F6FC03C06FEF7FEF02C0A4
:10227000692D70E042E050E0A40EB51EC6010E9438
:102280007A128C015FE7F52214C0F501C080D1807D
:10229000F6FC03C06FEF7FEF02C0692D70E042E0F3
:1022A00050E0A40EB51EC6010E946F128C0150E8CA
:1022B000F52AF3FE07C01AC080E290E0B3010E9445
:1022C0008512EA948E2D90E008171907A8F30EC026
:1022D000F601F7FC8591F7FE81916F0190E0B30163
:1022E0000E948512E110EA94015010400115110579
:1022F00079F7EAC0943611F0993669F5F7FE08C00F
:10230000F501208131814281538184E090E00AC04F
:10231000F501808191819C01442737FD4095542F20
:1023200082E090E0A80EB91E9FE6F92257FF09C08F
:1023300050954095309521953F4F4F4F5F4FE0E8C6
:10234000FE2ACA01B901A1012AE030E00E94B112BF
:10235000D82ED21840C0953729F41F2D1F7E2AE0B1
:1023600030E01DC01F2D197F9F3661F0903720F49B
:10237000983509F0ACC00FC0903739F0983709F0A4
:10238000A6C004C028E030E00AC0106114FD14604B
:1023900020E130E004C014FD166020E132E017FFB8
:1023A00008C0F501608171818281938144E050E031
:1023B00008C0F50180819181BC0180E090E042E09D
:1023C00050E0A40EB51EA1010E94B112D82ED21861
:1023D0008FE7F82EF122F6FE0BC05EEFF522D9143E
:1023E00038F4F4FE07C0F2FC05C08FEEF82202C0FC
:1023F0001D2D01C0192DF4FE0DC0FE01ED0DF11DC6
:102400008081803319F499EEF92208C01F5FF2FE33
:1024100005C003C08F2D867809F01F5F0F2DF3FCD8
:1024200014C0F0FE0FC01E1510F09D2C0BC09D2C8B
:102430009E0C911A1E2D06C080E290E0B3010E940E
:1024400085121F5F1E15C0F304C01E1510F4E11A9B
:1024500001C0EE2404FF0FC080E390E0B3010E94AE
:10246000851202FF1DC001FD03C088E790E00EC089
:1024700088E590E00BC0802F867891F001FF02C0C4
:102480008BE201C080E2F7FC8DE290E0B3010E9494
:10249000851206C080E390E0B3010E9485129A94F1
:1024A000D914C0F3DA94F101ED0DF11D808190E0B3
:1024B000B3010E948512DD20A9F706C080E290E0FA
:1024C000B3010E948512EA94EE20C1F743CEF301D6
:1024D00066817781CB012B96E2E10C9449C6FC0121
:1024E0000590615070400110D8F7809590958E0F3F
:1024F0009F1F0895FC016150704001900110D8F7B2
:10250000809590958E0F9F1F08950F931F93CF93E3
:10251000DF938C01EB018B8181FF1BC082FF0DC01B
:102520002E813F818C819D812817390764F4E881D1
:10253000F9810193F983E88306C0E885F985802F46
:102540001995892B31F48E819F8101969F838E830B
:1025500002C00FEF1FEFC801DF91CF911F910F91C4
:102560000895FA01AA27283051F1203181F1E89429
:102570006F936E7F6E5F7F4F8F4F9F4FAF4FB1E076
:102580003ED0B4E03CD0670F781F891F9A1FA11D71
:10259000680F791F8A1F911DA11D6A0F711D811D72
:1025A000911DA11D20D009F468943F912AE0269F37
:1025B00011243019305D3193DEF6CF010895462F96
:1025C0004770405D4193B3E00FD0C9F7F6CF462F77
:1025D0004F70405D4A3318F0495D31FD40524193E0
:1025E00002D0A9F7EACFB4E0A6959795879577959D
:1025F0006795BA95C9F700976105710508959B0124
:10260000AC010A2E06945795479537952795BA95AC
:10261000C9F7620F731F841F951FA01D08951F9295
:102620000F920FB60F9211242F933F938F939F9386
:10263000AF93BF938091920490919304A0919404DE
:10264000B0919504309196040196A11DB11D232FE0
:102650002D5F2D3720F02D570196A11DB11D209320
:1026600096048093920490939304A0939404B0935F
:10267000950480918E0490918F04A0919004B09164
:1026800091040196A11DB11D80938E0490938F0437
:10269000A0939004B0939104BF91AF919F918F91BB
:1026A0003F912F910F900FBE0F901F9018958FB7ED
:1026B000F8942091920430919304409194045091A5
:1026C00095048FBFB901CA0108959B01AC017FB782
:1026D000F89480918E0490918F04A0919004B09111
:1026E000910466B5A89B05C06F3F19F00196A11D26
:1026F000B11D7FBFBA2FA92F982F8827860F911D54
:10270000A11DB11D62E0880F991FAA1FBB1F6A950A
:10271000D1F7BC012DC0FFB7F89480918E04909141
:102720008F04A0919004B0919104E6B5A89B05C0D8
:10273000EF3F19F00196A11DB11DFFBFBA2FA92FC0
:10274000982F88278E0F911DA11DB11DE2E0880FE3
:10275000991FAA1FBB1FEA95D1F7861B970B885EAE
:102760009340C8F2215030404040504068517C4F67
:10277000211531054105510571F60895019739F08C
:10278000880F991F880F991F02970197F1F70895F5
:10279000789484B5826084BD84B5816084BD85B53C
:1027A000826085BD85B5816085BDEEE6F0E0808103
:1027B00081608083E1E8F0E0108280818260808324
:1027C000808181608083E0E8F0E0808181608083A7
:1027D000E1EBF0E0808184608083E0EBF0E08081D9
:1027E00081608083E1E9F0E0808182608083808184
:1027F00081608083E0E9F0E0808181608083E1EAAC
:10280000F0E0808182608083808181608083E0EA63
:10281000F0E0808181608083E1E2F1E0808182608C
:102820008083808181608083E0E2F1E0808181604B
:102830008083EAE7F0E08081846080838081826029
:102840008083808181608083808180688083109212
:10285000C10008951F93CF93DF93182FEB0161E020
:102860000E940A15209709F4CAC0CF3FD10509F488
:10287000C9C0E12FF0E0E75FFD4F8491893009F492
:1028800066C08A30B0F48430F1F1853040F4823093
:1028900059F1833070F5813009F0AEC020C0873027
:1028A00009F443C0883008F048C0863009F0A4C05D
:1028B00034C08D3009F478C08E3038F48B3009F490
:1028C0005AC08C3008F066C04CC0803109F480C01A
:1028D000813109F487C08F3009F08EC06FC084B594
:1028E000806884BDC7BD92C084B5806284BDC8BD08
:1028F0008DC080918000806880938000D093890093
:10290000C093880083C080918000806280938000A3
:10291000D0938B00C0938A0079C08091B00080680A
:102920008093B000C093B30071C08091B00080620A
:102930008093B000C093B40069C08091900080681B
:1029400080939000D0939900C09398005FC08091CD
:102950009000806280939000D0939B00C0939A0077
:1029600055C080919000886080939000D0939D0026
:10297000C0939C004BC08091A00080688093A00011
:102980008091A0008F7B8093A000D093A900C0937A
:10299000A8003CC08091A00080628093A000D093EA
:1029A000AB00C093AA0032C08091A00088608093E1
:1029B000A000D093AD00C093AC0028C0809120014E
:1029C000806880932001D0932901C09328011EC004
:1029D00080912001806280932001D0932B01C093CD
:1029E0002A0114C080912001886080932001D09337
:1029F0002D01C0932C010AC0C038D1051CF4812FD1
:102A000060E002C0812F61E00E94BD15DF91CF918F
:102A10001F910895CF93DF93482F50E0CA018D5343
:102A20009E4FFC01349143585E4FFA0184918823F4
:102A300069F190E0880F991FFC01E15DFE4FA591BF
:102A4000B491FC01E75BFE4FC591D491662351F42C
:102A50002FB7F8948C91932F909589238C9388812C
:102A600089230BC0623061F42FB7F8948C91932FB7
:102A7000909589238C938881832B88832FBF06C0F0
:102A80009FB7F8948C91832B8C939FBFDF91CF914C
:102A90000895893009F449C08A30A0F4843051F196
:102AA000853040F4823079F1833000F5813009F0CF
:102AB00063C026C0873079F1883098F5863009F0F8
:102AC0005BC025C08D3009F442C08E3028F48B30B5
:102AD000B1F18C30C0F52DC0803109F442C0813194
:102AE00009F445C08F3009F047C037C0809180009D
:102AF0008F7703C0809180008F7D80938000089540
:102B000084B58F7702C084B58F7D84BD0895809190
:102B1000B0008F7703C08091B0008F7D8093B000AC
:102B20000895809190008F7707C0809190008F7DED
:102B300003C080919000877F8093900008958091DA
:102B4000A0008F7707C08091A0008F7D03C0809187
:102B5000A000877F8093A0000895809120018F7747
:102B600003C0809120018F7D809320010895809182
:102B70002001877F809320010895FF920F931F9378
:102B8000F62E482F50E0CA01875F9D4FFC0124912B
:102B9000CA018D539E4FFC01149143585E4FFA01B8
:102BA00004910023C9F0222319F0822F0E944915B5
:102BB000E02FF0E0EE0FFF1FE75BFE4FA591B49111
:102BC0009FB7F894FF2021F48C911095812302C0C7
:102BD0008C91812B8C939FBF1F910F91FF90089533
:102BE0001F920F920FB60F920BB60F9211242F93D4
:102BF0003F934F935F936F937F938F939F93AF9385
:102C0000BF93EF93FF9380919B0490919C04892B39
:102C100029F0E0919B04F0919C041995FF91EF91AC
:102C2000BF91AF919F918F917F916F915F914F91E4
:102C30003F912F910F900BBE0F900FBE0F901F90E2
:102C400018951F920F920FB60F920BB60F92112488
:102C50002F933F934F935F936F937F938F939F93A4
:102C6000AF93BF93EF93FF9380919D0490919E0447
:102C7000892B29F0E0919D04F0919E041995FF9114
:102C8000EF91BF91AF919F918F917F916F915F91E4
:102C90004F913F912F910F900BBE0F900FBE0F9051
:102CA0001F9018951F920F920FB60F920BB60F92AE
:102CB00011242F933F934F935F936F937F938F9341
:102CC0009F93AF93BF93EF93FF9380919F04909155
:102CD000A004892B29F0E0919F04F091A00419959C
:102CE000FF91EF91BF91AF919F918F917F916F91E4
:102CF0005F914F913F912F910F900BBE0F900FBEA0
:102D00000F901F9018951F920F920FB60F920BB64F
:102D10000F9211242F933F934F935F936F937F9361
:102D20008F939F93AF93BF93EF93FF938091A104F1
:102D30009091A204892B29F0E091A104F091A204C2
:102D40001995FF91EF91BF91AF919F918F917F91D5
:102D50006F915F914F913F912F910F900BBE0F900C
:102D60000FBE0F901F9018951F920F920FB60F92E3
:102D70000BB60F9211242F933F934F935F936F9352
:102D80007F938F939F93AF93BF93EF93FF93809124
:102D9000970490919804892B29F0E0919704F09181
:102DA00098041995FF91EF91BF91AF919F918F91E9
:102DB0007F916F915F914F913F912F910F900BBE3B
:102DC0000F900FBE0F901F9018951F920F920FB685
:102DD0000F920BB60F9211242F933F934F935F9353
:102DE0006F937F938F939F93AF93BF93EF93FF93D3
:102DF0008091990490919A04892B29F0E09199048B
:102E0000F0919A041995FF91EF91BF91AF919F9125
:102E10008F917F916F915F914F913F912F910F9083
:102E20000BBE0F900FBE0F901F9018951F920F9220
:102E30000FB60F920BB60F9211242F933F934F931F
:102E40005F936F937F938F939F93AF93BF93EF9312
:102E5000FF938091A3049091A404892B29F0E09121
:102E6000A304F091A4041995FF91EF91BF91AF9144
:102E70009F918F917F916F915F914F913F912F9192
:102E80000F900BBE0F900FBE0F901F9018951F92C2
:102E90000F920FB60F920BB60F9211242F933F9300
:102EA0004F935F936F937F938F939F93AF93BF9352
:102EB000EF93FF938091A5049091A604892B29F0AC
:102EC000E091A504F091A6041995FF91EF91BF91AF
:102ED000AF919F918F917F916F915F914F913F91B2
:102EE0002F910F900BBE0F900FBE0F901F90189553
:102EF000CF92DF92EF92FF920F931F93CF93DF93C6
:102F00007C016B018A01C0E0D0E00FC0D6016D9159
:102F10006D01D701ED91FC910190F081E02DC70189
:102F20001995C80FD91F015010400115110571F7EF
:102F3000CE01DF91CF911F910F91FF90EF90DF9025
:102F4000CF900895DC01ED91FC910190F081E02D8E
:102F500019950895CF93DF93EC016115710519F46C
:102F600020E030E00FC0DB010D900020E9F7119761
:102F7000A61BB70BE881F9810280F381E02DAD013A
:102F800019959C01C901DF91CF9108950E94AA175C
:102F9000089508958091F005089567707070E82F86
:102FA000F0E0E75FFD4F84918B3028F48830A0F487
:102FB000863090F106C08E30D0F08F50833060F5AF
:102FC00021C08091B100887F8093B1008091B100D1
:102FD000862B8093B100089580919100887F809323
:102FE000910080919100862B8093910008958091AB
:102FF000A100887F8093A1008091A100862B8093FF
:10300000A100089580912101887F80932101809102
:103010002101862B8093210108958130910549F487
:103020006F5F7F4F09F052C087EA94E00E94C57637
:103030000895892B09F04AC06F5F7F4F09F046C0A1
:1030400083E094E0909377058093760580917D05E9
:10305000882321F08AE795E00E94B13E83E094E066
:10306000909335058093340580913B05882321F0AA
:1030700088E395E00E94B13E83E094E090931605CA
:103080008093150580911C05882321F089E195E046
:103090000E94B13E83E094E09093F7048093F6049D
:1030A0008091FD04882321F08AEF94E00E94B13ED4
:1030B00083E094E09093D6048093D5048091DC045F
:1030C000882321F089ED94E00E94B13E089580E0CC
:1030D00090E06FEF7FEF0E940D18089581E090E07F
:1030E0006FEF7FEF0E940D1808950E94D2698091C2
:1030F000F005882309F03AC081E08093F0058091C3
:10310000F2059091F305A091F405B091F505809337
:10311000F6059093F705A093F805B093F905E5E55A
:10312000F2E0949108C08091C00085FFFCCF90939D
:10313000C600319694919923B1F7E6E6F2E09491B6
:1031400008C08091C00085FFFCCF9093C6003196E7
:1031500094919923B1F78091C00085FFFCCF8AE05C
:103160008093C6008CE592E00E9469BC0895F894B3
:103170000E94D269159A179A429AA09A8FB7F8942A
:1031800090910B01926090930B018FBF8CE060E0F7
:103190000E940A15E5E5F2E0949108C08091C00014
:1031A00085FFFCCF9093C600319694919923B1F797
:1031B000E5EEF2E0949108C08091C00085FFFCCF5D
:1031C0009093C600319694919923B1F78091C000F5
:1031D00085FFFCCF8AE08093C6008CED92E00E94D0
:1031E00078BC809A8898FFCF0E9457136093FA05A5
:1031F0007093FB058093FC059093FD05E0912306F9
:10320000F0912406EB5DF94F80818823A9F4E4E076
:10321000F3E0949108C08091C00085FFFCCF9093AB
:10322000C600319694919923B1F78091C00085FF33
:10323000FCCF8AE08093C6000895EF92FF920F932F
:103240001F930E945713E090FE05F090FF05009138
:103250000006109101062091FA053091FB0540917E
:10326000FC055091FD05621B730B840B950BE61654
:10327000F7060807190738F4E114F10401051105F0
:1032800011F00E94B71880917C0390917D03A0916A
:103290007E03B0917F030097A105B10569F10E94FB
:1032A00057132091FA053091FB054091FC05509190
:1032B000FD05621B730B840B950B20917C033091F1
:1032C0007D0340917E0350917F03261737074807FF
:1032D000590790F490918D0F80918E0F981761F49B
:1032E000159A179A429AA09A9FB7F89480910B0169
:1032F000826080930B019FBF0E9461511F910F91CB
:10330000FF90EF9008956F927F928F929F92AF926D
:10331000BF92CF92DF92EF92FF920F931F93F82EFE
:103320006091020670910306809104069091050653
:103330002091060630910706409108065091090633
:103340000E94FAC33B014C0100D000D00DB71EB75C
:103350000F5F1F4F60916C0370916D03882777FD9D
:103360008095982F0E9481C2209180033091810323
:1033700040918203509183030E94BFC420E030E05B
:1033800040E752E40E94E6C120E030E048EC52E41D
:103390000E94E6C15B016C01F80160827182828249
:1033A0009382F4828091E50585838DEA95E06EE055
:1033B00076E042E056E020E001E032E0E32E0E94B9
:1033C000924B80910E0690910F06A0911006B0913D
:1033D00011068093AD059093AE05A093AF05B09311
:1033E000B0058091120690911306A0911406B09139
:1033F00015068093B1059093B205A093B305B093E1
:10340000B4058091160690911706A0911806B09108
:1034100019068093B5059093B605A093B705B093B0
:10342000B80580911A0690911B06A0911C06B091D8
:103430001D068093B9059093BA05A093BB05B09380
:10344000BC058DB79EB706960FB6F8949EBF0FBE0B
:103450008DBF0E9457136093FA057093FB0580930C
:10346000FC059093FD051F910F91FF90EF90DF9069
:10347000CF90BF90AF909F908F907F906F90089566
:10348000CF92DF92EF92FF920F931F930E945713F8
:103490006093FA057093FB058093FC059093FD05FE
:1034A0006091AD057091AE058091AF059091B0052A
:1034B00020910E0630910F06409110065091110692
:1034C0000E94DFC1882309F07AC06091B105709134
:1034D000B2058091B3059091B40520911206309108
:1034E000130640911406509115060E94DFC18823EF
:1034F00009F065C06091800370918103809182031F
:103500009091830320E030E040E752E40E94E6C15E
:103510007B018C018EE096E062E176E046E156E0C8
:103520002AE136E0E5EECE2EE5E0DE2E0E944E5496
:1035300080910E0690910F06A0911006B091110691
:103540008093AD059093AE05A093AF05B093B00501
:103550008091120690911306A0911406B091150661
:103560008093B1059093B205A093B305B093B405D1
:103570008091160690911706A0911806B091190631
:103580008093B5059093B605A093B705B093B805A1
:1035900080911A0690911B06A0911C06B0911D0601
:1035A0008093B9059093BA05A093BB05B093BC0571
:1035B0001F910F91FF90EF90DF90CF900895609151
:1035C0006C0370916D03882777FD8095982F0E947A
:1035D00081C22091800330918103409182035091F8
:1035E00083030E94BFC420E030E040E752E40E9421
:1035F000E6C120E030E048EC52E488CF8FE398E069
:103600000E94C338E7E0F3E0949108C08091C000C5
:1036100085FFFCCF9093C600319694919923B1F722
:103620004091F2055091F3056091F4057091F50514
:103630004F5F5F4F6F4F7F4F8FE398E02AE030E09E
:103640000E9484398091C00085FFFCCF8AE080937E
:10365000C6000E94F41808952F923F924F925F92F5
:103660006F927F928F929F92AF92BF92CF92DF9292
:10367000EF92FF920F931F93DF93CF9300D000D070
:10368000CDB7DEB78C018330910508F051C13C0104
:10369000660C771C660C771C930123553A4F3A83CE
:1036A000298380E090E0A0E0B0E0F901808391837D
:1036B000A283B3838DEA95E061EB75E045EB55E0BD
:1036C00029EB35E00E94394FF301EC5FFA4F659129
:1036D000759185919491045E1A4FF801E4909301DD
:1036E000225F394F3E832D8320E030E040EC5FE3E2
:1036F0000E94BFC45B016C01FF24E7FCF0940F2D16
:103700001F2DC801B7010E9481C21B012C01C601F7
:10371000B501A20191010E94BFC4AD81BE816D932C
:103720007D938D939C931397F301E45AFC4FFC8394
:10373000EB836081718182819381609380037093B8
:103740008103809382039093830320E030E040E77D
:1037500052E40E94E6C17B018C018EE096E062E1BA
:1037600076E046E156E02AE136E0A5EECA2EA5E075
:10377000DA2E0E944E540E94B76180E090E0A0E0F3
:10378000B0E0E981FA8180839183A283B3838DEADB
:1037900095E061EB75E045EB55E029EB35E00E94E3
:1037A000394FF301E05FFA4F85909590A590B49062
:1037B000C501B4019058A20191010E94BFC4AD811E
:1037C000BE816D937D938D939C931397609180033D
:1037D00070918103809182039091830320E030E017
:1037E00040E752E40E94E6C17B018C018EE096E046
:1037F00062E176E046E156E02AE136E00E944E546E
:103800000E94B761C501B401A50194010E9406C1DF
:10381000A20191010E94BFC4ED81FE81608371838A
:1038200082839383AB81BC816D917D918D919C91BD
:1038300020E030E040E05FE30E94BFC4609380037B
:1038400070938103809382039093830320E030E0A0
:1038500040E752E40E94E6C17B018C018EE096E0D5
:1038600062E176E046E156E02AE136E00E944E54FD
:103870000E94B761F301E052FB4F6591759185910C
:103880009491F301E354FA4FA080B180C280D380B9
:10389000A60195010E9406C17B018C01CB01D801D4
:1038A000E981FA8180839183A283B383F301E45198
:1038B000FB4F6591759185919491F9EC8F2EF5E010
:1038C0009F2E860C971CA60195010E9406C1D4016B
:1038D0006D937D938D939C931397F301E850FB4F69
:1038E0006591759185919491E0E7F3E06E0E7F1EEE
:1038F000A60195010E9406C1D3016D937D938D931E
:103900009C931397C701D801ED81FE818083918339
:10391000A283B38380E090E0A0E0B0E080938003D6
:1039200090938103A0938203B09383030E94A360CA
:1039300026960FB6F894DEBF0FBECDBFCF91DF91B4
:103940001F910F91FF90EF90DF90CF90BF90AF90BD
:103950009F908F907F906F905F904F903F902F90AF
:103960000895682F209123063091240680E690E088
:10397000AC01249FC001259F900D349F900D112410
:10398000815D994F70E00E943F109C0190932E063C
:1039900080932D0680E0232B09F081E00895FC013F
:1039A000949108C08091C00085FFFCCF9093C60021
:1039B000319694919923B1F78FE398E022E030E0BB
:1039C0000E94943A0895FC01949108C08091C0002F
:1039D00085FFFCCF9093C600319694919923B1F75F
:1039E0008FE398E022E030E00E94943A0895FC01D1
:1039F000949108C08091C00085FFFCCF9093C600D1
:103A0000319694919923B1F78FE398E02AE030E062
:103A10000E946539089580912D0690912E06019699
:103A200060E070E04AE050E00E94A70E08958091A7
:103A30002D0690912E06019660E070E00E94470DE1
:103A40000895CF93DF93EC018091E5058093F10514
:103A500084E50E94B11C882309F46FC00E94171DE1
:103A60000E9453C2262F6093F105623008F465C0AE
:103A7000EFE4F2E0949108C08091C00085FFFCCF94
:103A80009093C600319694919923B1F7C936D10528
:103A900099F0CA36D10524F4C836D105F1F50FC026
:103AA000CD36D10531F0CA3DD105B9F5E0E0F2E0FF
:103AB00031C0E7E1F2E023C0EEE2F2E015C0E5E458
:103AC000F2E007C08091C00085FFFCCF3196909353
:103AD000C60090819923B1F720C08091C00085FF76
:103AE000FCCF31969093C60090819923B1F715C011
:103AF0008091C00085FFFCCF31969093C6009081E5
:103B00009923B1F70AC08091C00085FFFCCF3196A0
:103B10009093C60090819923B1F78FE398E0622FCC
:103B200040E050E00E9472398091C00085FFFCCFD8
:103B30008AE08093C60081E001C080E0DF91CF91F0
:103B40000895AF92BF92CF92DF92EF92FF920F93C0
:103B50001F93CF93DF931DEAE12E15E0F12ECEE007
:103B6000D6E000E010E0F801E554FC4F80810E94AF
:103B7000B11C882339F10E94171D5B016C01F8010B
:103B8000E955FA4F8081882311F061E002C060910D
:103B90001E0670E0882777FD8095982F0E9481C2CD
:103BA000F70120813181428153810E94BFC49B0172
:103BB000AC01C601B5010E9406C1688379838A837E
:103BC0009B8309C0F70180819181A281B3818883A1
:103BD0009983AA83BB830F5F1F4F84E090E0E80EB8
:103BE000F91E24960430110509F0BDCF86E40E9429
:103BF000B11C8823E1F00E94171D7B018C016093AA
:103C00001F0670932006809321069093220620E0E1
:103C100030E040E050E00E94EDC3181644F4E0921A
:103C20008003F09281030093820310938303DF915A
:103C3000CF911F910F91FF90EF90DF90CF90BF90A9
:103C4000AF9008950E94A11D89E40E94B11C8823B1
:103C500059F00E94171D609302067093030680932B
:103C60000406909305060CC080E090E0A0E0B0E070
:103C70008093020690930306A0930406B093050672
:103C80008AE40E94B11C882359F00E94171D60939A
:103C90000606709307068093080690930906089518
:103CA00080E090E0A0E0B0E08093060690930706E5
:103CB000A0930806B093090608952F923F924F9261
:103CC0005F926F927F928F929F92AF92BF92CF92AC
:103CD000DF92EF92FF920F931F93DF93CF93CDB7B5
:103CE000DEB76E970FB6F894DEBF0FBECDBF87E488
:103CF0000E94B11C882309F492C30E94171D0E94E0
:103D00004EC26430710509F441C06530710554F448
:103D10006230710541F1633071056CF57723CCF4A5
:103D20000C949C306A35710509F424C36B35710518
:103D300034F46C31710511F00C949C306FC06B350C
:103D4000710509F41BC36C35710511F00C949C309E
:103D50001AC38091F005882331F40E94A11D0E94AE
:103D6000401A0C94C1308091F005882321F40E9400
:103D7000221E81E007C08091F005882339F40E945B
:103D8000221E80E00E9483190C94C13087ED94E0DC
:103D90000E9469BC80E50E94B11C882321F4EE24B6
:103DA000FF24870106C00E94171D0E9453C27B0199
:103DB0008C0183E50E94B11C882361F00E94171DCD
:103DC00020E030E04AE754E40E94BFC40E9453C29E
:103DD0007B018C010E94B7610E9457135B016C014B
:103DE000AE0CBF1CC01ED11E0E9457136093FA0573
:103DF0007093FB058093FC059093FD0506C00E941F
:103E0000AC6E0E941D190E9443BD0E9457136A1593
:103E10007B058C059D0598F30C949C308091800364
:103E200090918103A0918203B0918303809329062E
:103E300090932A06A0932B06B0932C0680916C03D6
:103E400090916D039093AC058093AB0584E690E070
:103E500090936D0380936C030E9457136093FA054F
:103E60007093FB058093FC059093FD0581E00E9413
:103E7000AA608091AD059091AE05A091AF05B0917B
:103E8000B00580930E0690930F06A0931006B09392
:103E900011068091B1059091B205A091B305B09142
:103EA000B4058093120690931306A0931406B09362
:103EB00015068091B5059091B605A091B705B09112
:103EC000B8058093160690931706A0931806B09332
:103ED00019068091B9059091BA05A091BB05B091E2
:103EE000BC0580931A0690931B06A0931C06B09302
:103EF0001D0680E090E0A0E0B0E080938003909306
:103F00008103A0938203B093830388E50E94B11CD0
:103F1000882361F489E50E94B11C882339F48AE57D
:103F20000E94B11C882311F481E001C080E08093DD
:103F30008403882361F488E50E94B11C882309F476
:103F400062C189E50E94B11C882309F45CC180E04C
:103F500090E0A0E0B0E08093AD059093AE05A09313
:103F6000AF05B093B0058093B1059093B205A093CF
:103F7000B305B093B4058DEA95E061EB75E045EBD0
:103F800055E029EB35E00E94394F80E090ECA9E93B
:103F9000B3EC80930E0690930F06A0931006B09397
:103FA00011068093120690931306A0931406B09303
:103FB000150620915C0330915D0340915E035091A2
:103FC0005F032093800330938103409382035093D7
:103FD0008303E0906003F09061030091620310910D
:103FE0006303C801B7010E94DFC1882344F4E09253
:103FF0008003F09281030093820310938303609106
:10400000800370918103809182039091830320E06B
:1040100030E040E752E40E94E6C17B018C018EE073
:1040200096E062E176E046E156E02AE136E0B5EE60
:10403000CB2EB5E0DB2E0E944E540E94B761E0EE1D
:10404000F4E065917591859194912091BD05309131
:10405000BE054091BF055091C0050E9406C1609306
:10406000AD057093AE058093AF059093B005ECEE6F
:10407000F4E065917591859194912091BD05309101
:10408000BE054091BF055091C0050E9406C16093D6
:10409000C9057093CA058093CB059093CC05E8EFD2
:1040A000F4E065917591859194912091BD053091D1
:1040B000BE054091BF055091C0050E9406C16093A6
:1040C0007003709371038093720390937303E4EE13
:1040D000F4E065917591859194912091C10530919D
:1040E000C2054091C3055091C4050E9406C160936A
:1040F000B1057093B2058093B3059093B405E0EFDA
:10410000F4E065917591859194912091C10530916C
:10411000C2054091C3055091C4050E9406C1609339
:10412000CD057093CE058093CF059093D005ECEF2D
:10413000F4E065917591859194912091C10530913C
:10414000C2054091C3055091C4050E9406C1609309
:1041500074037093750380937603909377038DEACD
:1041600095E061EB75E045EB55E029EB35E00E9409
:10417000394F8091AD059091AE05A091AF05B091FA
:10418000B00580930E0690930F06A0931006B0938F
:1041900011068091B1059091B205A091B305B0913F
:1041A000B4058093120690931306A0931406B0935F
:1041B0001506609180037091810380918203909134
:1041C000830320E030E040E752E40E94E6C17B0137
:1041D0008C018EE096E062E176E046E156E02AE16D
:1041E00036E00E944E5480E090E0A0E0B0E0809382
:1041F000800390938103A0938203B09383030E9472
:10420000B7610E94A36080918403882329F488E524
:104210000E94B11C882321F080E090E00E942C1BBA
:1042200080918403882329F489E50E94B11C8823A6
:1042300021F081E090E00E942C1B80918403882370
:1042400029F48AE50E94B11C882321F082E090E0E5
:104250000E942C1B88E50E94B11C8823D9F00E9483
:104260000B1D6115710581059105A1F00E94171DB7
:104270002091BD053091BE054091BF055091C0050C
:104280000E9406C16093AD057093AE058093AF05A3
:104290009093B00589E50E94B11C8823D9F00E9453
:1042A0000B1D6115710581059105A1F00E94171D77
:1042B0002091C1053091C2054091C3055091C405BC
:1042C0000E9406C16093B1057093B2058093B30557
:1042D0009093B4058AE50E94B11C8823D9F00E940E
:1042E0000B1D6115710581059105A1F00E94171D37
:1042F0002091C5053091C6054091C7055091C8056C
:104300000E9406C16093B5057093B6058093B7050A
:104310009093B8058DEA95E061EB75E045EB55E0CB
:1043200029EB35E00E94394F8091290690912A06A9
:10433000A0912B06B0912C0680938003909381036B
:10434000A0938203B09383038091AB059091AC0559
:1043500090936D0380936C030E9457136093FA054A
:104360007093FB058093FC059093FD050E94A3606C
:104370000C949C3010921E060C949C3081E080932B
:104380001E060C949C3085E40E94B11C882311F415
:104390000E94B761ADEAEA2EA5E0FA2EFDEBCF2E22
:1043A000F5E0DF2E00E010E0F801E554FC4F8081DD
:1043B0000E94B11C882331F1033061F40E94171D63
:1043C000F701608371838283938389EB95E00E9478
:1043D0001B4F18C00E94171DF601208131814281B8
:1043E00053810E9406C1F7016083718382839383A6
:1043F0008DEA95E061EB75E045EB55E029EB35E0A2
:104400000E94394F0F5F1F4F24E030E0E20EF31E91
:10441000C20ED31E0430110539F60C949C308DE485
:104420000E94B11C882311F40C94462F0E94171D82
:104430000E944EC26B36710509F4F5C66C367105E3
:104440000CF084C06C31710509F427C26D3171051F
:10445000C4F56531710509F4C1C166317105BCF45B
:104460006131710509F47FC16231710534F4623044
:10447000710510F00C949C3017C16231710509F47C
:10448000E8C66431710511F00C949C307AC1683132
:10449000710509F4C7C16931710554F466317105BC
:1044A00009F4A2C16731710511F00C949C30A2C1CE
:1044B0006A31710509F4CCC16B3171050CF0E7C1AB
:1044C000C1C16335710509F4C0C664357105FCF4DA
:1044D0006A32710509F4E4C26B32710554F46E312D
:1044E000710509F416C26F31710511F00C949C30FE
:1044F00055C26135710509F4A0C6623571050CF02D
:10450000A1C66035710511F00C949C3092C66C35D3
:10451000710509F40DC76D35710554F464357105E5
:1045200009F497C66535710511F00C949C30EAC604
:104530006936710509F427C36A3671050CF042C665
:104540006836710511F00C949C30ECC26D3C71051D
:1045500011F40C94AA2C6E3C71050CF046C068371F
:10456000710511F40C94332B69377105DCF4633752
:10457000710509F462C76437710554F46D3671052D
:1045800009F4D3C36237710511F00C949C307AC7DB
:104590006537710509F460C76737710511F00C9430
:1045A0009C307EC06E3B710509F451C56F3B7105AF
:1045B0005CF46937710511F40C94352B6C38710576
:1045C00011F00C949C30CEC26B3C710511F40C942C
:1045D0006C2C6C3C710514F00C948A2C693C7105B0
:1045E00011F00C949C300C94322C31E06F32730734
:1045F00011F40C94E02E41E0603374073CF56C3DFF
:10460000710511F40C94D12D6D3D710564F46E3C6F
:10461000710511F40C94082D6A3D710511F00C948C
:104620009C300C94262D51E06D32750711F40C94DA
:10463000EF2D81E06E32780714F00C94DC2E6D3D86
:10464000710511F00C949C300C94E02D91E0653FC5
:10465000790711F40C94262FE1E0663F7E076CF495
:10466000F1E060397F0711F40C94202F645F7140F2
:1046700011F00C949C300C94232F31E0673F7307AA
:1046800011F40C942C2F41E0673F740714F40C9440
:10469000292F675E734011F00C949C300C942F2FDF
:1046A000ECE5F2E00C94402B86EC94E00E9469BCAF
:1046B00080E50E94B11C882321F4AA24BB24650153
:1046C00006C00E94171D0E9453C25B016C0183E566
:1046D0000E94B11C882361F00E94171D20E030E089
:1046E0004AE754E40E94BFC40E9453C25B016C01BC
:1046F0000E94B7610E9457136093FA057093FB05FF
:104700008093FC059093FD05A114B104C104D1046C
:1047100001F10E9457137B018C01EA0CFB1C0C1D5C
:104720001D1D0E9457136E157F0580079107A8F481
:1047300080919A1082FD11C00E94AC6E0E941D19DA
:104740000E9443BDEECF0E94AC6E0E941D190E94D4
:1047500043BD80919A1082FFF6CF87EB94E00E94D0
:1047600069BC0C949C308EEA94E00E9469BC159858
:1047700017984298A0989FB7F89480910B018D7F6D
:10478000BDC5EEE9F4E0949108C08091C00085FFBA
:10479000FCCF9093C600319694919923B1F7809104
:1047A000C00085FFFCCF8AE08093C60087EA94E0D2
:1047B0000E942F80E0E9F4E0949108C08091C0004D
:1047C00085FFFCCF9093C600319694919923B1F761
:1047D0008091C00085FFFCCF0C94993087EA94E06B
:1047E0000E94917B0C949C3087EA94E00E948F7524
:1047F0000C949C3080912D0690912E0604966AE2CE
:1048000070E00E943F10FC01009711F03197108278
:1048100060912D0670912E066C5F7F4F87EA94E0C1
:1048200041E073C087EA94E00E9493750E94571399
:104830006093E8057093E9058093EA059093EB0592
:104840000C949C3087EA94E00E949A750C949C30FA
:104850008091A904882311F40C949C3083E50E9474
:10486000B11C882311F40C949C300E940B1DAB01E9
:10487000BC0140939D0550939E0580939F057093C6
:10488000A0058AE795E00E94973D0C949C3087EA4A
:1048900094E00E94A2770C949C3080912D06909118
:1048A0002E0604966AE270E00E943F108C01009789
:1048B00019F1209123063091240680E690E0FC0156
:1048C0002E9FC0012F9F900D3E9F900D1124815D62
:1048D000994F6EE470E00E943F1060E270E00E9429
:1048E0003F109C012F5F3F4F30932E0620932D06E3
:1048F00001501040F801108260912D0670912E0633
:104900006C5F7F4F87EA94E040E00E946E790C94E0
:104910009C308091A904882311F40C949C3087EA80
:1049200094E00E94B07680912D0690912E06049618
:104930006AE270E00E943F108C01009719F120910B
:1049400023063091240680E690E0AC01249FC0014C
:10495000259F900D349F900D1124815D994F6EE439
:1049600070E00E943F1060E270E00E943F109C01E6
:104970002F5F3F4F30932E0620932D06015010409D
:10498000F801108260912D0670912E066C5F7F4FAA
:1049900087EA94E00E94FC770C949C300E945713A5
:1049A0006093EC057093ED058093EE059093EF0511
:1049B0002091E8053091E9054091EA055091EB0519
:1049C000621B730B840B950B28EE33E040E050E044
:1049D0000E94D7C5F22EE32ED42EC52E2DB73EB79A
:1049E000285030400FB6F8943EBF0FBE2DBF0DB714
:1049F0001EB70F5F1F4FCE010196EDB7FEB7928332
:104A0000818381E894E0F801938382836F2D7E2D6A
:104A1000842F952F2CE330E040E050E00E94D7C572
:104A2000F801358324836F2D7E2D8D2D9C2D2CE355
:104A300030E040E050E00E94D7C5F80177836683FC
:104A40000E946E10EFE4F2E094912DB73EB7285F1C
:104A50003F4F0FB6F8943EBF0FBE2DBF08C08091E8
:104A6000C00085FFFCCF9093C600319694919923A6
:104A7000B1F7FE01319607C08091C00085FFFCCFE1
:104A800031969093C60090819923B1F78091C00030
:104A900085FFFCCF8AE08093C600CE010196EFC46B
:104AA00083E50E94B11C882311F40C949C300E9471
:104AB000171D0E944EC27B018C016B0180E50E9494
:104AC000B11C882369F0F7FC0BC03FEFE316F1043B
:104AD00009F034F40E94171D0E944EC28B0102C0DF
:104AE0000DE010E0EFEBF3E08081918180179107FA
:104AF00011F40C949C30329644E0EF33F407A1F7A4
:104B000017FF02C00C949C30802F61E00E940A15B0
:104B1000802F6C2D0E94BD15802FB6010E942A1493
:104B20000C949C3088E690E00E94211D882311F0AF
:104B30000C949C3083E50E94B11C882379F00E947C
:104B4000171D2091F105022F10E0000F111F0351D6
:104B5000104F0E944EC2F801718360830E94E26B85
:104B60000C949C3083E50E94B11C882311F40C94B2
:104B70009C300E94171D0E944EC27093F20F6093EA
:104B8000F10F0C949C3089E690E00E94211D88234F
:104B900011F00C949C30EBE7F4E0949108C0809104
:104BA000C00085FFFCCF9093C60031969491992365
:104BB000B1F7E091F105F0E0EE0FFF1FEE0FFF1FE0
:104BC000E950F04F40815181628173818FE398E019
:104BD00021E030E00E94943AE8E7F4E0949108C0C4
:104BE0008091C00085FFFCCF9093C60031969491D0
:104BF0009923B1F7E091F105F0E0EE0FFF1FE351CB
:104C0000F04F60817181882777FD8095982F0E94F1
:104C100081C2AB01BC018FE398E021E030E00E944B
:104C2000943AE4E7F4E0949108C08091C00085FFD5
:104C3000FCCF9093C600319694919923B1F740919F
:104C400001105091021060910310709104108FE3D5
:104C500098E021E030E00E94943AE1E7F4E094919A
:104C600008C08091C00085FFFCCF9093C6003196AC
:104C700094919923B1F76091F10F7091F20F882709
:104C800077FD8095982F0E9481C2AB01BC018FE314
:104C900098E021E030E00E94943AEDE6F4E094914F
:104CA00008C08091C00085FFFCCF9093C60031966C
:104CB00094919923B1F78091F1050E94C769BC01D5
:104CC0008FE398E04AE050E00E94B939E8E6F4E06A
:104CD000949108C08091C00085FFFCCF9093C600DE
:104CE000319694919923B1F78FEF9FEF0E94C76996
:104CF000BC018FE398E04AE050E00E94B939E5E753
:104D0000F2E007C08091C00085FFFCCF3196909300
:104D1000C60090819923B1F78091C00085FFFCCF38
:104D20008AE08093C6000C94C1308DE690E00E942A
:104D3000211D882311F00C949C308DE594E00E9495
:104D400069BC83E50E94B11C882379F00E94171D7D
:104D50002091F105022F10E0000F111F0351104F99
:104D60000E944EC2F801718360830E94E26B0E9430
:104D700057134B015C012091F105022F10E07724BD
:104D8000000F111FF801E351F04F608171818827F6
:104D900077FD8095982F0E9481C2000F111F095046
:104DA000104FF80120813181428153810E94EDC36F
:104DB000181614F477247394CC24CA94DC2C76014E
:104DC000EAE5F4E04490E6E5F4E05490E2E5F4E04E
:104DD00064900AE0302E2EC1942DEAE5F4E008C07C
:104DE0008091C00085FFFCCF9093C60031969491CE
:104DF0009923B1F7E091F105F0E0EE0FFF1FEE0F00
:104E0000FF1FE950F04F40815181628173818FE330
:104E100098E021E030E00E94943A952DE6E5F4E038
:104E200008C08091C00085FFFCCF9093C6003196EA
:104E300094919923B1F76091F1058FE398E070E0C8
:104E40004AE050E00E94B939962DE2E5F4E008C04E
:104E50008091C00085FFFCCF9093C600319694915D
:104E60009923B1F7F7FE03C0E6E7F2E028C00E94FD
:104E70005713A70196012854344F4F4F5F4F261BFD
:104E8000370B480B590BCA01B90128EE33E040E05B
:104E900050E00E94D7C58FE398E0BA01A9012AE04B
:104EA00030E00E9465398091C00085FFFCCF0EC0C4
:104EB0008091C00085FFFCCF31969093C600908111
:104EC0009923B1F78091C00085FFFCCF3092C600D6
:104ED0000E9457134B015C010E94AC6E0E941D1989
:104EE0000E9443BDFFEFCF16FFEFDF06FFEFEF0697
:104EF000FFEFFF0609F050C0E091F105772031F196
:104F0000F0E08F01000F111F000F111F0950104F0B
:104F1000EE0FFF1FE351F04F60817181882777FD0D
:104F20008095982F0E9481C220E030E040E85FE346
:104F30000E9405C19B01AC01F801608171818281F1
:104F400093810E94EDC387FF58C05EC0F0E08F01DF
:104F5000000F111F000F111F0950104FEE0FFF1F00
:104F6000E351F04F60817181882777FD8095982FFC
:104F70000E9481C220E030E040E85FE30E9406C169
:104F80009B01AC01F80160817181828193810E9453
:104F9000DFC1181694F538C0F7FC36C0E091F10572
:104FA000F0E08F01000F111F000F111F0950104F6B
:104FB000EE0FFF1FE351F04F60817181882777FD6D
:104FC0008095982F0E9481C29B01AC01F8016081FD
:104FD0007181828193810E9405C10E944EC297FF18
:104FE00007C090958095709561957F4F8F4F9F4F2B
:104FF00064307105810591053CF00E945713AC01A6
:10500000CB01DA016C017D01FFEFCF16FFEFDF0668
:10501000FFEFEF06FFEFFF0669F0F7FE02C00C940A
:105020009F300E9457136C197D09685B7B4010F01C
:105030000C949F300E945713681979098A099B09BB
:10504000695E73408040904008F0C6CE45CF87E34C
:1050500094E00E9469BC83E50E94B11C882341F062
:105060000E94171D0E944EC27093F20F6093F10FC1
:105070000E9457137B018C01E4E3F4E0B490E0E379
:10508000F4E0C490ECE2F4E0D4903AE0A32E7DC0CA
:105090000E9457136E197F09800B910B695E734054
:1050A0008040904008F46BC0E091E505F0E0EE0F21
:1050B000FF1FEE0FFF1FE950F04F408151816281C9
:1050C00073819B2DE4E3F4E008C08091C00085FF6C
:1050D000FCCF9093C600319694919923B1F78FE35A
:1050E00098E022E030E00E94943A9C2DE0E3F4E066
:1050F00008C08091C00085FFFCCF9093C600319618
:1051000094919923B1F76091E5058FE398E070E001
:105110004AE050E00E94B9399D2DECE2F4E008C06D
:105120008091C00085FFFCCF9093C600319694918A
:105130009923B1F740910110509102106091031032
:10514000709104108FE398E021E030E00E94943ADF
:10515000E5E7F2E007C08091C00085FFFCCF319603
:105160009093C60090819923B1F78091C00085FF8C
:10517000FCCFA092C6000E9457137B018C010E94B5
:10518000AC6E0E941D190E9443BD6091F10F709199
:10519000F20F882777FD8095982F0E9481C2209179
:1051A00001103091021040910310509104100E94A0
:1051B000EDC318160CF46CCF82E294E00E9469BC37
:1051C0000C94AD3083E50E94B11C882321F10E942C
:1051D000171D20E030E040E050E00E94DFC188234E
:1051E0001CF460E070E011C00E94171D20E030E068
:1051F0004FE753E40E94EDC318161CF46FEF70E004
:1052000004C00E94171D0E944EC27093E705609370
:10521000E6050C949C308FEF90E09093E705809327
:10522000E6050C949C301092E7051092E6050C946C
:105230009C30269A2E980C949C300E94B761809ADC
:1052400088987AC71092AA0577C781E08093AA054B
:1052500073C783E50E94B11C882399F00E94171D33
:1052600020E030E04AE754E40E94BFC40E9453C2E9
:1052700060937C0370937D0380937E0390937F0300
:105280005BC788E50E94B11C882309F071C789E5D6
:105290000E94B11C882309F06BC78AE50E94B11CEB
:1052A000882309F065C785E40E94B11C882309F0B2
:1052B0005FC70E94B761A09A9FB7F89480910B01D5
:1052C000826080930B019FBF0E94C56135C7159A0C
:1052D00089E50E94B11C8111179A8AE50E94B11CD0
:1052E0008111429A85E40E94B11C882309F424C7E5
:1052F000A09A9FB7F89480910B01826080930B0174
:105300009FBF1AC783E50E94B11C0E94171D20E0B1
:1053100030E04AE754E40E94BFC40E9453C2609345
:10532000FE057093FF05809300069093010604C765
:1053300091E6692E9AE0792E81E5282E8AE0382EB2
:105340000DE9402E0AE0502E88249924F401E554FA
:10535000FC4F80810E94B11C882309F45DC053E09A
:10536000851609F052C00E94171D5B016C0120E0F8
:1053700030E040EA51E40E94DFC188230CF03FC0D6
:10538000F3016081718182819381A60195010E9460
:10539000E6C17B018C016091950A7091960A80911B
:1053A000970A9091980AA80197010E94BFC4609340
:1053B000950A7093960A8093970A9093980AF10140
:1053C0006081718182819381A80197010E94BFC48D
:1053D000F1016083718382839383F2016081718123
:1053E000828193810E947FC2A80197010E94BFC45D
:1053F0000E9453C2F2016083718382839383F3011D
:10540000A082B182C282D38207C00E94171DF3011D
:1054100060837183828393830894811C911C24E0B0
:1054200030E0620E731E220E331E420E531E34E015
:105430008316910409F08ACF7FC6E2E8F3E09491E5
:1054400008C08091C00085FFFCCF9093C6003196C4
:1054500094919923B1F770C680912D0690912E06F4
:1054600005966AE270E00E943F10FC01009711F07F
:105470003197108280912D0690912E0605960E94FC
:105480008CBC5AC6EFE7F3E0949108C08091C0004D
:1054900085FFFCCF9093C600319694919923B1F784
:1054A0004091AD055091AE056091AF057091B0058A
:1054B0008FE398E022E030E00E94943AECE7F3E0DA
:1054C000949108C08091C00085FFFCCF9093C600E6
:1054D000319694919923B1F74091B1055091B2055D
:1054E0006091B3057091B4058FE398E022E030E05D
:1054F0000E94943AE9E7F3E0949108C08091C000DB
:1055000085FFFCCF9093C600319694919923B1F713
:105510004091B5055091B6056091B7057091B805F9
:105520008FE398E022E030E00E94943AE6E7F3E06F
:10553000949108C08091C00085FFFCCF9093C60075
:10554000319694919923B1F74091B9055091BA05DC
:105550006091BB057091BC058FE398E022E030E0DC
:105560000E94943AEBE6F3E0949108C08091C00069
:1055700085FFFCCF9093C600319694919923B1F7A3
:1055800080E00E9482610E9481C22091610A309174
:10559000620A4091630A5091640A0E94E6C1AB011D
:1055A000BC018FE398E022E030E00E94943AE8E604
:1055B000F3E0949108C08091C00085FFFCCF9093E8
:1055C000C600319694919923B1F781E00E948261DF
:1055D0000E9481C22091650A3091660A4091670A53
:1055E0005091680A0E94E6C1AB01BC018FE398E0CC
:1055F00022E030E00E94943AE5E6F3E0949108C09E
:105600008091C00085FFFCCF9093C60031969491A5
:105610009923B1F782E00E9482610E9481C22091A9
:10562000690A30916A0A40916B0A50916C0A0E9493
:10563000E6C1AB01BC018FE398E022E030E00E94BC
:10564000943AE5E7F2E007C08091C00085FFFCCF07
:1056500031969093C60090819923B1F78091C00054
:1056600085FFFCCF66C580E001C081E00E94AA6092
:1056700063C58091C00085FFFCCF31969093C60032
:1056800090819923B1F78091C00085FFFCCF8AE01B
:105690008093C600EDE5F3E0949108C08091C000CE
:1056A00085FFFCCF9093C600319694919923B1F772
:1056B000009B03C0E8E7F2E00AC0EDE7F2E007C0B4
:1056C0008091C00085FFFCCF31969093C6009081F9
:1056D0009923B1F78091C00085FFFCCF8AE08093C9
:1056E000C600E5E5F3E0949108C08091C00085FF15
:1056F000FCCF9093C600319694919923B1F7029B09
:1057000003C0E8E7F2E00AC0EDE7F2E007C08091ED
:10571000C00085FFFCCF31969093C60090819923FD
:10572000B1F78091C00085FFFCCF8AE08093C6006E
:10573000EDE4F3E0949108C08091C00085FFFCCFB8
:105740009093C600319694919923B1F7049B03C0BE
:10575000E8E7F2E00AC0EDE7F2E007C08091C000A0
:1057600085FFFCCF31969093C60090819923B1F7C5
:105770008091C00085FFFCCF8AE08093C600E5E4FD
:10578000F3E0949108C08091C00085FFFCCF909316
:10579000C600319694919923B1F7069B03C0E8E7C0
:1057A000F2E00AC0EDE7F2E007C08091C00085FF9B
:1057B000FCCF31969093C60090819923B1F78091E8
:1057C000C00085FFFCCF8AE08093C600EDE3F3E0E4
:1057D000949108C08091C00085FFFCCF9093C600D3
:1057E000319694919923B1F7379B03C0E8E7F2E033
:1057F0000AC0EDE7F2E007C08091C00085FFFCCF52
:1058000031969093C60090819923B1F78091C000A2
:1058100085FFFCCF8AE08093C600E5E3F3E0949136
:1058200008C08091C00085FFFCCF9093C6003196E0
:1058300094919923B1F7359B03C0E8E7F2E00AC0E1
:10584000EDE7F2E007C08091C00085FFFCCF319604
:105850009093C60090819923B1F78091C00085FF95
:10586000FCCF67C41BEBC12E13E0D12EEE24FF2426
:10587000F60180810E94B11C882309F10E94171D46
:1058800087010F58154F0E9453C2F801608371833E
:10589000828393830E94171D87010356154FF701DA
:1058A000EF59F54F20813181428153810E94BFC45D
:1058B0000E9453C2F80160837183828393830894AA
:1058C000C11CD11C24E030E0E20EF31E3FEBC316F6
:1058D00033E0D30669F630C40BEB13E0B1E5EB2EF1
:1058E000BAE0FB2EF80180810E94B11C882339F0B8
:1058F0000E94171DF70160837183828393830F5F7A
:105900001F4F24E030E0E20EF31E33E00F3B13079D
:1059100049F712C483E50E94B11C882351F00E940C
:10592000171D6093850A7093860A8093870A909367
:10593000880A84E50E94B11C882309F4FDC30E94F3
:10594000171D6093890A70938A0A80938B0A90933B
:105950008C0AF2C383E50E94B11C882351F00E9497
:10596000171D6093810A7093820A8093830A909333
:10597000840A84E50E94B11C882351F00E94171DFF
:105980006093990A70939A0A80939B0A90939C0A59
:1059900082E40E94B11C882361F00E94171D0E94BE
:1059A00053C260934D0A70934E0A80934F0A9093AE
:1059B000500A88E50E94B11C882351F00E94171DEF
:1059C00060938D0A70938E0A80938F0A9093900A49
:1059D0008AE50E94B11C882351F00E94171D609334
:1059E000910A7093920A8093930A9093940A85E4A3
:1059F0000E94B11C882309F49FC30E94171D609365
:105A0000950A7093960A8093970A9093980A94C384
:105A10000BEB13E0ADEBEA2EA5E0FA2EF801808146
:105A20000E94B11C882339F00E94171DF701608382
:105A30007183828393830F5F1F4F24E030E0E20E77
:105A4000F31E33E00E3B130749F776C38AED90E06F
:105A50000E94211D882309F06FC388E50E94B11CB4
:105A6000882389F08091F105082F10E00E94171D0E
:105A7000000F111F000F111F0B521A4FF801608306
:105A800071838283938389E50E94B11C882389F006
:105A90008091F105082F10E00E94171D000F111FC3
:105AA000000F111F03521A4FF80160837183828324
:105AB0009383EFE4F2E0949108C08091C00085FFE9
:105AC000FCCF9093C600319694919923B1F7E5E20B
:105AD000F3E0949108C08091C00085FFFCCF9093C3
:105AE000C600319694919923B1F71092F10540C008
:105AF0008091C00085FFFCCF11969093C6009C91C9
:105B00009923B1F7F0E0EE0FFF1FEE0FFF1FEB52EE
:105B1000FA4F40815181628173818FE398E022E0E6
:105B200030E00E94943AE7E8F2E007C08091C000BC
:105B300085FFFCCF31969093C60090819923B1F7F1
:105B4000E091F105F0E0EE0FFF1FEE0FFF1FE352B3
:105B5000FA4F40815181628173818FE398E022E0A6
:105B600030E00E94943A8091F1058F5F8093F105B7
:105B7000E091F105E23018F0E5E7F2E00AC0A9E8AB
:105B8000B2E0BDCF8091C00085FFFCCF31969093ED
:105B9000C60090819923B1F78091C00085FFFCCFAA
:105BA000C8C283E50E94B11C882309F4C5C20E94C3
:105BB000171D0E944EC270936D0360936C03BCC2AC
:105BC00083E50E94B11C882309F4B6C20E94171D08
:105BD0000E944EC270936F0360936E03ADC280E566
:105BE0000E94B11C882351F00E94171D60938A0304
:105BF00070938B0380938C0390938D0389E40E94B0
:105C0000B11C882381F00E94171D2DEB37E346E07D
:105C10005EE30E94BFC460938E0370938F038093F2
:105C200090039093910384E40E94B11C882381F037
:105C30000E94171D2DEB37E346E05EE30E94E6C1AC
:105C400060939203709393038093940390939503CE
:105C500083E40E94B11C882351F00E94171D6093B9
:105C600096037093970380939803909399030E94EF
:105C7000A469EBE8F2E007C08091C00085FFFCCF8B
:105C800031969093C60090819923B1F7EEE8F2E047
:105C900007C08091C00085FFFCCF31969093C6006D
:105CA00090819923B1F740918A0350918B036091C1
:105CB0008C0370918D038FE398E022E030E00E9426
:105CC000943AE2E9F2E007C08091C00085FFFCCF82
:105CD00031969093C60090819923B1F760918E031D
:105CE00070918F0380919003909191032DEB37E396
:105CF00046E05EE30E94E6C1AB01BC018FE398E0A1
:105D000022E030E00E94943AE6E9F2E007C0809198
:105D1000C00085FFFCCF31969093C60090819923F7
:105D2000B1F76091920370919303809194039091E5
:105D300095032DEB37E346E05EE30E94BFC4AB0161
:105D4000BC018FE398E022E030E00E94943AEAE957
:105D5000F2E007C08091C00085FFFCCF31969093A0
:105D6000C60090819923B1F76091960370919703D3
:105D700080919803909199032DEB37E346E05EE321
:105D80000E94BFC4AB01BC018FE398E022E030E089
:105D90000E94943AE5E7F2E007C08091C00085FFD9
:105DA000FCCF31969093C60090819923B1F78091F2
:105DB000C00085FFFCCFBDC181E00E94184FBCC16F
:105DC00085E40E94B11C882319F4CC24DD2412C080
:105DD0000E94171D0E944EC26B0177FF0BC00F2E51
:105DE000F0E0EF2EF0E0FF2EFCE80F2FF2E41F2F83
:105DF000F02D0AC00F2EF0E0EF2EF0E0FF2EF6E1BE
:105E00000F2FF3E41F2FF02D83E50E94B11C882390
:105E100021F00E94171D7B018C0183E40E94B11CBC
:105E2000882319F425E030E005C00E94171D0E9468
:105E30004EC29B01C801B701A6010E941A717CC124
:105E40000E94B76179C10E947C8076C10E945A8706
:105E500073C10E949A8270C10E941C846DC110920D
:105E6000F0050E94588B8091F6059091F705A0915E
:105E7000F805B091F9058093F2059093F305A0938E
:105E8000F405B093F5050E94FE1A56C184E50E9400
:105E9000B11C882309F405C10E94171D0E9453C23A
:105EA000262F6093F1056230A0F1EFE4F2E09491C7
:105EB00008C08091C00085FFFCCF9093C60031964A
:105EC00094919923B1F7EEE9F2E007C08091C00008
:105ED00085FFFCCF31969093C60090819923B1F74E
:105EE0008FE398E0622F40E050E00E947239E0EAD0
:105EF000F2E007C08091C00085FFFCCF31969093FF
:105F0000C60090819923B1F78091C00085FFFCCF36
:105F100010C186E40E94B11C882311F4EE241EC037
:105F20000E94171D7B018C0160931F067093200651
:105F3000809321069093220620E030E040E050E07C
:105F40000E94EDC3181644F4E0928003F09281039E
:105F50000093820310938303EE24E3949091F10560
:105F60008091E505981709F473C0AEE0B6E0EDEA5C
:105F7000F5E080E101900D928150E1F72091E50577
:105F8000C22EDD24CC0CDD1CCC0CDD1CF601EB524A
:105F9000FA4F6091AD057091AE058091AF0590917B
:105FA000B00520813181428153810E9405C1F0906A
:105FB000F1050F2D10E0000F111F000F111FF80148
:105FC000EB52FA4F20813181428153810E9406C1F8
:105FD0006093AD057093AE058093AF059093B005C7
:105FE0002DED35E0C20ED31E6091B1057091B20562
:105FF0008091B3059091B405F601208131814281F1
:1060000053810E9405C103521A4FF801208131814A
:10601000428153810E9406C16093B1057093B2051D
:106020008093B3059093B405F092E5058DEA95E071
:1060300061EB75E045EB55E029EB35E00E94394F07
:10604000EE2031F08091F005882311F40E94401A6F
:10605000EFE4F2E0949108C08091C00085FFFCCF8E
:106060009093C600319694919923B1F7E1EBF2E059
:1060700007C08091C00085FFFCCF31969093C60089
:1060800090819923B1F76091E5058FE398E070E086
:106090004AE050E00E94B9398091C00085FFFCCFF2
:1060A00048C0EFE4F2E0949108C08091C00085FF01
:1060B000FCCF9093C600319694919923B1F7E2E119
:1060C000F3E0949108C08091C00085FFFCCF9093CD
:1060D000C600319694919923B1F72091230630910F
:1060E000240680E690E0289FF001299FF00D389F5C
:1060F000F00D1124E15DF94F07C08091C00085FFCC
:10610000FCCF31969093C60090819923B1F7E0E1DE
:10611000F3E0949108C08091C00085FFFCCF90937C
:10612000C600319694919923B1F78091C00085FF04
:10613000FCCF8AE08093C6000E94F41822C084E459
:1061400094E00E9469BC0E9457136093E805709325
:10615000E9058093EA059093EB050E94571360933D
:10616000FA057093FB058093FC059093FD05E4CF41
:106170000E94B76188E50E94B11C882309F0A7C876
:10618000A7C86E960FB6F894DEBF0FBECDBFCF91F5
:10619000DF911F910F91FF90EF90DF90CF90BF9014
:1061A000AF909F908F907F906F905F904F903F90B7
:1061B0002F9008952F923F924F925F926F927F920D
:1061C0008F929F92AF92BF92CF92DF92EF92FF9207
:1061D0000F931F93DF93CF93CDB7DEB76E970FB6B4
:1061E000F894DEBF0FBECDBF20E6A22EB12CE0E5B5
:1061F000F5E084909AE0792EE6ECF5E09490662440
:10620000639413C22D3071F02A3321F48091B007CA
:10621000882341F08091B1079091B2078F359105A5
:106220000CF4DFC1E091B107F091B207309709F4A7
:10623000F3C2A091B307B091B407AA9D7001AB9DC2
:10624000F00CBA9DF00C1124EE0DFF1DE15DF94F2D
:1062500010828091B007882309F0BEC11092B00768
:10626000AB5DB94F1C928701015D194FC8016EE407
:1062700070E00E943F109C01009709F4F7C09093D2
:106280002E0680932D062F5F3F4F201B310B2E0DC6
:106290003F1DC901815D994F60E070E04AE050E028
:1062A0000E94A70E6093B5077093B6078093B70757
:1062B0009093B807C090F205D090F305E090F405F4
:1062C000F090F505A70196012F5F3F4F4F4F5F4FAD
:1062D000621773078407950709F441C38091B307D8
:1062E0009091B4079C012A9DC0012B9D900D3A9D71
:1062F000900D1124815D994F6FE676E00E940410A5
:10630000892B09F02CC3E5E5F2E0949108C0809157
:10631000C00085FFFCCF9093C600319694919923DD
:10632000B1F7ECE3F6E0949108C08091C00085FFDE
:10633000FCCF9093C600319694919923B1F78FE3E7
:1063400098E0B701A6012AE030E00E9484398091EC
:10635000C00085FFFCCF73C0FE264F5FFC01E40F39
:10636000F11DE15DF94FE081EA32B1F730932E067D
:1063700020932D06C901019660E070E00E94470D50
:106380000E944EC22F2D30E02617370709F45DC05A
:10639000E5E5F2E0949108C08091C00085FFFCCF54
:1063A0009093C600319694919923B1F7EDE1F6E010
:1063B000949108C08091C00085FFFCCF9093C600E7
:1063C000319694919923B1F74091F2055091F305DC
:1063D0006091F4057091F5058FE398E02AE030E0D4
:1063E0000E9484398091C00085FFFCCF28C0E5E57C
:1063F000F2E0949108C08091C00085FFFCCF90939B
:10640000C600319694919923B1F7E3EFF5E09491AA
:1064100008C08091C00085FFFCCF9093C6003196E4
:1064200094919923B1F78FE398E0B701A6012AE090
:1064300030E00E9484398091C00085FFFCCF8AE063
:106440008093C6000E94FE1A4AC08091B5079091C1
:10645000B607A091B707B091B8078093F205909363
:10646000F305A093F405B093F5053EC0C8016AE2B8
:1064700070E00E943F10009709F436C0E5E5F2E0B5
:10648000949108C08091C00085FFFCCF9093C60016
:10649000319694919923B1F7E9ECF5E0949108C015
:1064A0008091C00085FFFCCF9093C60031969491F7
:1064B0009923B1F74091F2055091F3056091F405ED
:1064C0007091F5058FE398E02AE030E00E9484396E
:1064D0008091C00085FFFCCF8AE08093C6001092B7
:1064E000B2071092B1075AC28091B3079091B407D6
:1064F0008A9D70018B9DF00C9A9DF00C11248701F0
:10650000015D194FC80167E470E00E943F109C01D3
:10651000009709F44BC090932E0680932D062F5FB1
:106520003F4F201B310B2E0D3F1DC901815D994F3F
:1065300060E070E00E94470D0E944EC26430710519
:10654000A8F58091F0058823C9F48091A7048823D9
:1065500069F5992DE6ECF5E008C08091C00085FF53
:10656000FCCF9093C600319694919923B1F7809116
:10657000C00085FFFCCF7092C60018C0982DE0E5E2
:10658000F5E008C08091C00085FFFCCF9093C60065
:10659000319694919923B1F78091C00085FFFCCF8B
:1065A0007092C60086E495E00E9469BC8091B307B2
:1065B0009091B407019664E070E00E94C4C5909386
:1065C000B4078093B3078091B9079091BA070196F9
:1065D0009093BA078093B9071092B2071092B1074F
:1065E00024C02B3311F46092B0078091B007882348
:1065F000E1F42091B1073091B2078091B3079091F7
:10660000B4078A9DF0018B9DF00D9A9DF00D112429
:10661000E20FF31FE15DF94F8091AF0780832F5F99
:106620003F4F3093B2072093B10780913B08909180
:106630003C0820913D0830913E08821B930B8F77D8
:106640009070892B09F4A5C18091B9079091BA0780
:1066500004970CF09EC18FE398E00E94A538282F84
:106660008093AF078A3009F0CDCDDCCD8091B107A2
:106670009091B207892B09F425C190C14D3089F062
:106680004A3321F48091B007882359F08091B107F3
:106690009091B2078F35910524F42F5F3F4F09F099
:1066A000ECC020919D0530919E0540919F05509131
:1066B000A0058091950590919605A0919705B091C0
:1066C0009805281739074A075B0708F49EC0962DDE
:1066D000E3E3F5E008C08091C00085FFFCCF909314
:1066E000C600319694919923B1F78091C00085FF3F
:1066F000FCCF3092C6000E9457136093EC05709354
:10670000ED058093EE059093EF052091E80530911B
:10671000E9054091EA055091EB05621B730B840B70
:10672000950B28EE33E040E050E00E94D7C5F22EF2
:10673000E32ED42EC52EEDB7FEB738970FB6F894DA
:10674000FEBF0FBEEDBF0DB71EB70F5F1F4FB2826A
:10675000A182F80153824282622F732F842F952FDA
:1067600020E13EE040E050E00E94D7C5F8013583CB
:1067700024836F2D7E2D8D2D9C2D2CE330E040E069
:1067800050E00E94D7C5CA01B9012CE330E040E0D7
:1067900050E00E94D7C5F801778366830E946E108F
:1067A000972DEFE4F2E02DB73EB7285F3F4F0FB6CD
:1067B000F8943EBF0FBE2DBF08C08091C00085FF7A
:1067C000FCCF9093C600319694919923B1F7F501CF
:1067D00007C08091C00085FFFCCF31969093C60022
:1067E00090819923B1F78091C00085FFFCCF309252
:1067F000C600C5010E948CBC87EA94E00E94E47543
:1068000087EA94E061E00E94707C2091B1073091AA
:10681000B2072115310519F41092B007BFC080915D
:10682000B3079091B407889DF001899DF00D989D64
:10683000F00D1124E20FF31FE15DF94F1082FC010E
:10684000EB5DF94F20822091B9073091BA072F5F95
:106850003F4F3093BA072093B907019664E070E088
:106860000E94C4C59093B4078093B3071092B007F9
:106870001092B2071092B1073AC04B3311F4209234
:10688000B0078091B007882391F52091B10730912E
:10689000B2078091B3079091B407889DF001899D5C
:1068A000F00D989DF00D1124E20FF31FE15DF94FFB
:1068B0008091AF0780832F5F3F4F3093B2072093C3
:1068C000B10715C080E6882E912C22242394E3E39F
:1068D000F5E064900AE0302E5E010894A11CB11C22
:1068E0001FE1412E15E0512EEFE4F2E0749020916B
:1068F0009D0530919E0540919F055091A005809186
:10690000950590919605A0919705B0919805281747
:1069100039074A075B0708F041C08091B907909199
:10692000BA070497DCF58091820590918305A091C8
:106930008405B091850580939D0590939E05A09355
:106940009F05B093A0058AE795E00E945E419C01F7
:10695000482F8093AF078A3009F090CEA2CE809165
:10696000B3079091B4078A9D80018B9D100D9A9D6D
:10697000100D1124C801815D994F6AE270E00E94F8
:106980003F109C01009709F432CDFF2440E0C8017C
:10699000E5CC8091A804882309F068CE6E960FB6E6
:1069A000F894DEBF0FBECDBFCF91DF911F910F9145
:1069B000FF90EF90DF90CF90BF90AF909F908F901F
:1069C0007F906F905F904F903F902F900895CF935E
:1069D000DF938091B9079091BA07039714F40E944E
:1069E000DA3087EA94E060E00E94707C8091B90719
:1069F0009091BA07892B09F465C08091A704882378
:106A000009F448C0209123063091240680E690E0E6
:106A1000289FE001299FD00D389FD00D1124C15D22
:106A2000D94FCE0169E876E00E940410892BC1F4A9
:106A300087EA94E0BE010E942A77E6E8F6E09491A6
:106A400008C08091C00085FFFCCF9093C6003196AE
:106A500094919923B1F78091C00085FFFCCF16C0B7
:106A600087EA94E00E94B076E4E7F6E0949108C0EB
:106A70008091C00085FFFCCF9093C6003196949121
:106A80009923B1F78091C00085FFFCCF8AE0809305
:106A9000C60002C00E945D1E8091B9079091BA079E
:106AA00001979093BA078093B9078091230690913C
:106AB0002406019664E070E00E94C4C59093240609
:106AC000809323060E94AC6E0E941D190E94FA68F2
:106AD0000E9443BDDF91CF910895EF92FF920F93F3
:106AE0001F93DF93CF930F920F92CDB7DEB7809AAB
:106AF000889A269A2E988FE398E040E950ED63E05B
:106B000070E00E946D38E9E7F7E0949108C0809149
:106B1000C00085FFFCCF9093C600319694919923D5
:106B2000B1F78091C00085FFFCCF8AE08093C6005A
:106B30004FE452E0FA01949108C08091C00085FFB3
:106B4000FCCF9093C600319694919923B1F784B706
:106B5000282F80FF15C0E1E7F7E0949108C08091ED
:106B6000C00085FFFCCF9093C60031969491992385
:106B7000B1F78091C00085FFFCCF8AE08093C6000A
:106B800021FF15C0E1E6F7E0949108C08091C000B4
:106B900085FFFCCF9093C600319694919923B1F76D
:106BA0008091C00085FFFCCF8AE08093C60022FF61
:106BB00015C0E0E5F7E0949108C08091C00085FF22
:106BC000FCCF9093C600319694919923B1F78091B0
:106BD000C00085FFFCCF8AE08093C60023FF15C06C
:106BE000E0E4F7E0949108C08091C00085FFFCCFFD
:106BF0009093C600319694919923B1F78091C0008B
:106C000085FFFCCF8AE08093C60025FF15C0E0E336
:106C1000F7E0949108C08091C00085FFFCCF90936D
:106C2000C600319694919923B1F78091C00085FFF9
:106C3000FCCF8AE08093C60014BEE8E2F7E09491AE
:106C400008C08091C00085FFFCCF9093C6003196AC
:106C500094919923B1F7E9E0F7E0949108C080910D
:106C6000C00085FFFCCF9093C60031969491992384
:106C7000B1F78091C00085FFFCCF8AE08093C60009
:106C8000FA019491EFE4F2E008C08091C00085FF22
:106C9000FCCF9093C600319694919923B1F7E9EF18
:106CA000F6E0949108C08091C00085FFFCCF9093DE
:106CB000C600319694919923B1F7E4EEF6E09491F1
:106CC00008C08091C00085FFFCCF9093C60031962C
:106CD00094919923B1F7E8EDF6E0949108C0809182
:106CE000C00085FFFCCF9093C60031969491992304
:106CF000B1F7EAECF6E0949108C08091C00085FFFE
:106D0000FCCF9093C600319694919923B1F780916E
:106D1000C00085FFFCCF8AE08093C600EFEBF6E071
:106D2000949108C08091C00085FFFCCF9093C6006D
:106D3000319694919923B1F7E3EBF6E0949108C072
:106D40008091C00085FFFCCF9093C600319694914E
:106D50009923B1F78091C00085FFFCCF8AE0809332
:106D6000C600FA019491EFE4F2E008C08091C000FF
:106D700085FFFCCF9093C600319694919923B1F78B
:106D8000E4EAF6E0949108C08091C00085FFFCCF52
:106D90009093C600319694919923B1F72091CC102D
:106DA0003091CD10CE0101962115310519F4825D87
:106DB000904102C0821B930B9A83898369817A81F7
:106DC0008FE398E04AE050E00E94B939EDE8F6E040
:106DD000949108C08091C00085FFFCCF9093C600BD
:106DE000319694919923B1F78FE398E060ED74E0C8
:106DF0004AE050E00E94B9398091C00085FFFCCF85
:106E00008AE08093C6001092250610922606109202
:106E10002706109228060E945A87EE24FF24870135
:106E20000356154FF701EF58F54F6081718182814C
:106E300093810E947FC2F701EF59F54F2081318184
:106E4000428153810E94BFC40E9453C2F8016083F3
:106E500071838283938384E090E0E80EF91E90E1D1
:106E6000E916F104E1F60E947C6D0E9485510E94B2
:106E700032890E94B3600E9419BE0F900F90CF918B
:106E8000DF911F910F91FF90EF900895BC018091C9
:106E9000B9079091BA0704970CF070C02091B3071E
:106EA0003091B40780E690E0AC01249FC001259F9B
:106EB000900D349F900D1124815D994F0E94D60F43
:106EC000EFE4F2E0949108C08091C00085FFFCCF10
:106ED0009093C600319694919923B1F7E1E8F7E0D9
:106EE000949108C08091C00085FFFCCF9093C600AC
:106EF000319694919923B1F72091B3073091B4075B
:106F000080E690E0289FF001299FF00D389FF00D5A
:106F10001124E15DF94F07C08091C00085FFFCCFCF
:106F200031969093C60090819923B1F7EFE7F7E08F
:106F3000949108C08091C00085FFFCCF9093C6005B
:106F4000319694919923B1F78091C00085FFFCCFD1
:106F50008AE08093C600C901019664E070E00E9457
:106F6000C4C59093B4078093B3078091B9079091FB
:106F7000BA0701969093BA078093B9070895BC01A8
:106F80008091B9079091BA0704970CF070C02091D6
:106F9000B3073091B40780E690E0AC01249FC001B4
:106FA000259F900D349F900D1124815D994F0E9473
:106FB0004A10EFE4F2E0949108C08091C00085FF90
:106FC000FCCF9093C600319694919923B1F7EEE8E7
:106FD000F7E0949108C08091C00085FFFCCF9093AA
:106FE000C600319694919923B1F72091B30730915F
:106FF000B40780E690E0289FF001299FF00D389FAC
:10700000F00D1124E15DF94F07C08091C00085FFAC
:10701000FCCF31969093C60090819923B1F7ECE8AC
:10702000F7E0949108C08091C00085FFFCCF909359
:10703000C600319694919923B1F78091C00085FFE5
:10704000FCCF8AE08093C600C901019664E070E03D
:107050000E94C4C59093B4078093B3078091B90789
:107060009091BA0701969093BA078093B907089553
:107070001F920F920FB60F920BB60F9211242F93FF
:107080003F934F938F939F93EF93FF934091C6004D
:10709000E0913B08F0913C0831969F012F773070CA
:1070A000319780913D0890913E082817390739F0B3
:1070B000E554F84F408330933C0820933B08FF9100
:1070C000EF919F918F914F913F912F910F900BBE18
:1070D0000F900FBE0F901F9018959A01AB012030B2
:1070E00081EE380780E0480780E0580749F182E0E8
:1070F0008093C00060E079E08DE390E00E94F9C5E4
:107100002150304040405040CA01B90122E030E0F7
:1071100040E050E00E94F9C53093C5002093C400C0
:107120008091C10080618093C1008091C10088601E
:107130008093C1008091C10080688093C100089550
:107140001092C00020E130E0E7CF20913D0830915F
:107150003E0880913B0890913C088217930719F4F0
:107160002FEF3FEF0EC0F901E554F84F80812F5FFC
:107170003F4F2F77307030933E0820933D08282FE3
:1071800030E0C901089580913D0890913E089093A8
:107190003C0880933B08089508952F923F924F92A8
:1071A0005F926F927F928F929F92AF92BF92CF9297
:1071B000DF92EF92FF920F931F93DF93CF93CDB7A0
:1071C000DEB7A0970FB6F894DEBF0FBECDBF1C018F
:1071D0006A017B01411551056105710549F440E3E0
:1071E00050E060E070E020E030E00E94843954C05C
:1071F000882499245401422E55246624772401E0E2
:1072000010E00C0F1D1F080D191DC701B601A301C9
:1072100092010E94D7C5F80160830894811C911CDB
:10722000A11CB11CC701B601A30192010E94D7C5E0
:10723000C901DA016C017D01C114D104E104F1043A
:10724000F1F681E0E82EF12CEC0EFD1EE80CF91CA5
:107250003E010894611C711CD501C4010197A1096C
:10726000B1096C01C818D90814C0F601EE0DFF1D54
:1072700040814A3010F4405D01C0495C50E060E05C
:1072800070E0C10120E030E00E9484390894E108F8
:10729000F1086E147F0449F7A0960FB6F894DEBF8C
:1072A0000FBECDBFCF91DF911F910F91FF90EF9057
:1072B000DF90CF90BF90AF909F908F907F906F9016
:1072C0005F904F903F902F9008952115310539F42C
:1072D0008091C00085FFFCCF4093C60008950E94B6
:1072E000CD380895EF92FF920F931F939A01E62EE7
:1072F000FF2400E010E0B801A7010E9465391F914A
:107300000F91FF90EF900895EF92FF920F931F93CC
:10731000CF93DF93EC017A018B012115310539F40C
:107320008091C00085FFFCCFE092C6001BC02A30D0
:107330003105B1F477FF10C04DE250E060E070E03D
:1073400020E030E00E94843910950095F094E0949C
:10735000E11CF11C011D111DCE01B801A7012AE09D
:107360000E94CD38DF91CF911F910F91FF90EF9048
:107370000895EF92FF920F931F937B019A010027CC
:10738000F7FC0095102FB801A7010E9484391F91C6
:107390000F91FF90EF9008950F931F938C014DE094
:1073A00050E060E070E020E030E00E948439C801E5
:1073B0004AE050E060E070E020E030E00E94843974
:1073C0001F910F910895CF92DF92EF92FF920F934A
:1073D0001F938C019A016B01EE24FF24B701A601D3
:1073E0000E946539C8010E94CC391F910F91FF900E
:1073F000EF90DF90CF9008959F92AF92BF92CF927F
:10740000DF92EF92FF920F931F93CF93DF93EC01E4
:107410007A018B01922ECB01BA0120E030E040E0EE
:1074200050E00E94DFC188236CF4CE014DE250E0B1
:1074300060E070E020E030E00E94843917FB109596
:1074400017F9109520E030E040E05FE3AA240BC07C
:10745000CA01B90120E030E040E251E40E94E6C1F7
:107460009B01AC01A394A91498F3C801B7010E9431
:1074700006C17B018C010E9453C25B016C010E941A
:107480007FC29B01AC01C801B7010E9405C17B010D
:107490008C01CE01B601A5012AE030E00E946539D9
:1074A0009920A1F1E3ECF2E007C08091C00085FFD4
:1074B000FCCF31969093C60090819923B1F726C0F6
:1074C000C801B70120E030E040E251E40E94BFC4AF
:1074D0007B018C010E944EC25B016C01CC24B7FC85
:1074E000C094DC2CCE01B601A5012AE030E00E9458
:1074F0008439C601B5010E9481C29B01AC01C8015B
:10750000B7010E9405C17B018C019A949920C1F6B4
:10751000DF91CF911F910F91FF90EF90DF90CF906F
:10752000BF90AF909F9008950E94FC390895FF92FC
:107530000F931F93CF93DF938B010E945713EB019F
:10754000FF24FA9409C00E9457136C1B7D0B60172F
:10755000710710F080E008C0FEBC0DB407FEFDCF3F
:107560008EB58F3F81F781E0DF91CF911F910F9111
:10757000FF900895FC014281242F30E0C9019595C8
:10758000879580658CBD40FF02C080E004C080E02C
:10759000463009F081E08DBD808160E00E94BD151C
:1075A0000895DF92EF92FF920F931F93CF93DF9393
:1075B000EC01D62E79018A010E94BA3ACE016CE222
:1075C00071E00E94973A8D2D80648EBD0DB407FE48
:1075D000FDCF28E130E0D801C701022E04C0B695E6
:1075E000A795979587950A94D2F78EBD0DB407FE9F
:1075F000FDCF285030408FEF283F380761F7DD205E
:1076000011F485E906C088E0D81611F487E801C0B6
:107610008FEF8EBD0DB407FEFDCF8CE0D81631F490
:107620008FEF8EBD0DB407FEFDCF8EB59FEF2FEF10
:107630002EBD0DB407FEFDCF8EB587FF04C0992384
:1076400011F09150F5CF8B83DF91CF911F910F9166
:10765000FF90EF90DF900895FC01808161E00E942F
:10766000BD150895DC016EBDFA0120E030E00DB4D7
:1076700007FEFDCF80818EBD0DB407FEFDCF818159
:107680008EBD2E5F3F4F329682E02030380779F76B
:107690000DB407FEFDCF8FEF8EBD0DB407FEFDCFFD
:1076A0008FEF8EBD0DB407FEFDCF8FEF8EBD0DB4F5
:1076B00007FEFDCF8EB513968C9313978F7185308F
:1076C00011F481E0089583E111968C931197CD0117
:1076D0000E942C3B80E00895CF92DF92EF92FF92C0
:1076E0000F931F93CF93DF93EC017A018B01690114
:1076F0008C81833039F059E0EE0CFF1C001F111F04
:107700005A95D1F7CE0168E1A80197010E94D13ABC
:10771000882311F086E023C0CE016EEFA6010E94FF
:10772000323B8823E9F0CE0168E572E00E94973A87
:10773000882311F487E113C0CE016DE020E030E032
:1077400040E050E00E94D13A882341F48FEF8EBD93
:107750000DB407FEFDCF8EB5882379F086E18983CD
:10776000CE010E942C3B80E0DF91CF911F910F91C1
:10777000FF90EF90DF90CF900895CE010E942C3BB8
:1077800081E0F2CFBF92CF92DF92EF92FF920F9300
:107790001F93CF93DF93EC016B017A010E94571383
:1077A0008B01BB24BA9409C00E945713601B710B54
:1077B0006D52714010F081E10BC0BEBC0DB407FEEC
:1077C000FDCF8EB58B838F3F79F38E3F39F08FE0FD
:1077D0008983CE010E942C3B80E02FC0D7011197F6
:1077E000EF28D9F08FEF8EBD20E030E09FEF0BC087
:1077F0000DB407FEFDCF8EB5F601E20FF31F8083B7
:107800009EBD2F5F3F4F2A173B0790F30DB407FE35
:10781000FDCF8EB5AC0DBD1D8C938FEF8EBD0DB41D
:1078200007FEFDCF8EB58FEF8EBD0DB407FEFDCFE9
:107830008EB5CE010E942C3B81E0DF91CF911F914C
:107840000F91FF90EF90DF90CF90BF900895CF926F
:10785000DF92EF92FF920F931F93CF93DF93EC0190
:107860007A018B0169018C81833039F0A9E0EE0C3B
:10787000FF1C001F111FAA95D1F7CE0161E1A801DD
:1078800097010E94D13A882339F084E08983CE01A0
:107890000E942C3B80E006C0CE01B60140E052E0E1
:1078A0000E94C23BDF91CF911F910F91FF90EF900B
:1078B000DF90CF900895BF92CF92DF92EF92FF9228
:1078C0000F931F93CF93DF93EC01B62E1C82198286
:1078D00048830E9457136B01888161E00E940A155A
:1078E000CE010E942C3B82E360E00E940A1583E3F4
:1078F00061E00E940A1584E361E00E940A1585E3B5
:1079000061E00E940A1585E361E00E94BD1585E0F3
:107910008A8382E58CBD1DBC80E09FEF9EBD0DB4C7
:1079200007FEFDCF8F5F8A30C9F709C00E94571349
:107930006C197D09615D774010F081E05EC0CE0179
:1079400060E020E030E040E050E00E94D13A182FA3
:107950008B83813059F7CE0168E02AEA31E040E0BC
:1079600050E00E94D13A82FF02C01C8311C080E027
:107970002FEF2EBD0DB407FEFDCF9EB58F5F843077
:10798000C1F79B839A3A11F082E037C082E08C8382
:107990008C81823021F0EE24FF2487010FC0E12C7E
:1079A000F12C012D00E4102F09C00E9457136C190F
:1079B0007D09615D774010F08AE01FC0CE0167E36A
:1079C00020E030E040E050E00E94D13ACE0169E290
:1079D000A80197010E94D13A8B83882331F78C81CB
:1079E000823029F5CE016AE320E030E040E050E04B
:1079F0000E94D13A882331F088E08983CE010E9429
:107A00002C3B21C08FEF8EBD0DB407FEFDCF8EB590
:107A1000807C803C11F483E08C8380E09FEF9EBDEE
:107A20000DB407FEFDCF2EB58F5F8330C1F7CE01B9
:107A30000E942C3B86E08B1518F488E1898303C0F3
:107A4000BA8281E001C080E0DF91CF911F910F9158
:107A5000FF90EF90DF90CF90BF900895CF93DF938A
:107A6000EB01DC0190E020E03EE28C91803269F095
:107A7000283029F4FE01E90FF11D30839F5FFE01DC
:107A8000E90FF11D8C9180839F5F2F5F11962B3042
:107A900061F7C90FD11D1882DF91CF910895CF935F
:107AA000DF93DC01EB01BA0180E090E020E2FE010F
:107AB000E80FF91F208301968B309105C1F757E03D
:107AC00040E022C02E3219F089E997E007C05A3011
:107AD00049F15AE048E017C0321721F1FC01019644
:107AE00034913323C9F75417E8F02132D8F02F37F7
:107AF000C8F4822F81568A3108F42052FE01E40F27
:107B0000F11D20834F5F11962C91222311F02F320B
:107B1000C9F6FB01B183A08390E08881803219F01F
:107B200091E001C090E0892FDF91CF9108956F928D
:107B30007F928F929F92AF92BF92CF92DF92EF92FD
:107B4000FF920F931F93CF93DF93EC017A018B0188
:107B50002B81222309F480C089899A89AB89BC8949
:107B600084179507A607B70708F476C085C0E11407
:107B7000F1040105110551F41C821D821E821F8231
:107B8000188619861A861B8681E067C02885398584
:107B90004A855B85E98DFA8D858590E009962150AF
:107BA00030404040504039014A01082E04C09694AC
:107BB0008794779467940A94D2F72F5F3F4F4F4F83
:107BC0005F4F0894E108F1080109110957016801A4
:107BD00004C0D694C794B794A7948A95D2F7089412
:107BE000E11CF11C011D111DA614B704C804D90421
:107BF00028F0211531054105510549F48D899E89EB
:107C0000AF89B88D8C839D83AE83BF8316C0A618C1
:107C1000B708C808D90811C04C815D816E817F8189
:107C2000898D9A8D94010E9443490894A108B10856
:107C3000C108D108882331F40FC084E0882E912C2C
:107C40008C0E9D1EA114B104C104D10429F7E8864D
:107C5000F9860A871B8798CF80E0DF91CF911F912B
:107C60000F91FF90EF90DF90CF90BF90AF909F90DB
:107C70008F907F906F900895223009F078CFE7CFF2
:107C8000CF93DF93EC018C859D85AE85BF8540E069
:107C9000611141E0BC01CD010E941947882319F40C
:107CA00020E030E00AC08889282F30E095E0220FDC
:107CB000331F9A95E1F72A5B374FC901DF91CF91C6
:107CC00008950F931F93CF93DF938C01FC01838161
:107CD0008823F1F1818187FF38C0C80161E00E94EB
:107CE000403EEC010097A1F18881853E89F1F801C1
:107CF0008381823040F481899289A389B4898C8FF1
:107D00009D8FAE8FBF8FF801858996899B8F8A8F53
:107D100085899689A789B08DCD01AA27BB279D8B20
:107D20008C8BE0914008F0914108309751F0BE01F2
:107D30006A5E7F4FCE0148961995888D998D9B8BF1
:107D40008A8BF80181818F7781830E94DE4604C08F
:107D500081E0F801808380E0DF91CF911F910F9146
:107D600008950F931F938C010E94613EF8011382C6
:107D70001F910F910895FC018381882319F0CF0191
:107D80000E94B13E0895CF93DF93FC01EB01838104
:107D9000882391F08250823020F48FE28883198208
:107DA00009C0CF0160E00E94403E009729F0BE016B
:107DB0000E942E3D81E001C080E0DF91CF910895C7
:107DC0006F927F928F929F92AF92BF92CF92DF92EB
:107DD000EF92FF920F931F93DF93CF9300D00F92F8
:107DE000CDB7DEB77C015A016B01DC0113968C9193
:107DF0001397813009F091C011968C9181FF8DC04D
:107E0000A0C00097A105B10511F481E087C0F7017A
:107E10006084718482849384C701B601A5010E94A5
:107E2000973D882309F479C0D70159968D919C918B
:107E30005A97A114B104C104D10489F455964D9107
:107E40005D916D917C9158970E94B949882309F4FE
:107E500064C0F701158A168A178A108E44C0D701AC
:107E600014964D915D916D917C9117979E012F5FB6
:107E70003F4F0E944349882309F44FC0D7015996C8
:107E8000ED91FC915A9749815A816B817C81878958
:107E9000803149F4483FBFEF5B07B0E06B07B0E0CB
:107EA0007B0748F020C0483F8FEF58078FEF6807E7
:107EB0008FE07807C0F4CF010E94B949882369F1A7
:107EC000D70114964D915D916D917C9117975996BC
:107ED0008D919C915A970FEF1FEF2FEF3FE00E947B
:107EE000BC488823D1F0F701A18AB28AC38AD48A18
:107EF000818180688183C7010E94613E882369F087
:107F0000B601A5016A147B048C049D0410F4B4012D
:107F1000A301C7010E94973D01C080E00F900F9020
:107F20000F900F90CF91DF911F910F91FF90EF90E5
:107F3000DF90CF90BF90AF909F908F907F906F9089
:107F40000895F70181899289A389B48984179507D7
:107F5000A607B70708F055CFE0CFCF93DF93EC012A
:107F600040E050E060E070E00E94E03E882369F06D
:107F7000CE0161E00E94403EFC01009731F085EEA9
:107F800080831B820E94DE4601C080E0DF91CF919A
:107F900008952F923F924F925F926F927F928F92AD
:107FA0009F92AF92BF92CF92DF92EF92FF920F9388
:107FB0001F93CF93DF93EC012A018B81882309F46F
:107FC000B6C0898180FFB3C0C8C025014E185F08C4
:107FD0003B0174E0272E312C2C0E3D1E4201A1C026
:107FE000288539854A855B856FEFA62E61E0B62E20
:107FF000A222B3228B8179018A0199E01695079517
:10800000F794E7949A95D1F7E98DFA8D823049F487
:10801000428D538D648D758D4E0D5F1D601F711FD8
:108020003FC0D480DA94DE20A114B104D9F4DD205D
:10803000C9F4211531054105510549F48D899E8901
:10804000AF89B88D8C839D83AE83BF830BC04C8179
:108050005D816E817F81CF0191010E944349882318
:1080600009F465C0E98DFA8D4C815D816E817F8157
:108070004250504060407040058404C0440F551F7A
:10808000661F771F0A94D2F786859785A089B189E4
:10809000480F591F6A1F7B1F4D0D511D611D711D1A
:1080A00080E092E08A199B0984018815990508F4FB
:1080B0008C0182E00030180709F067C08091420807
:1080C00090914308A0914408B0914508481759077A
:1080D0006A077B0709F459C08091460A9091470AC4
:1080E00093010E94273C882349F421C095012A5B13
:1080F000374FC301B901A8010E942B10600E711EF9
:10810000980140E050E088859985AA85BB85820F5B
:10811000931FA41FB51F88879987AA87BB87801ADA
:10812000910A8114910409F05BCFA20102C04FEFC4
:108130005FEFCA01DF91CF911F910F91FF90EF90F8
:10814000DF90CF90BF90AF909F908F907F906F9077
:108150005F904F903F902F900895A988BA88CB8860
:10816000DC88E884F9840A851B859A0140E050E0A8
:10817000D601C5018E199F09A00BB10B281739072D
:108180004A075B0708F021CF23CFCB01BA0140E0BB
:108190000E941947882309F0A9CFC9CFCF92DF9257
:1081A000EF92FF920F931F93CF93DF937C01EB012C
:1081B0008A01FC018381823008F46FC0808591853B
:1081C000A285B3858F719070A070B0700097A105E3
:1081D000B10509F062C06DC0F8011082EDE0CE2E4D
:1081E000D12CC701BE0140E250E00E94C93F9C0172
:1081F0008032910521F0009709F04FC050C04881AE
:10820000442309F44CC0453E61F34E3251F38B8553
:108210008F738F30E9F501151105D1F18A8D9B8D92
:10822000892BB1F5842F90E08F719070009781F1C8
:10823000833091056CF58C9D90018D9D300D9C9D3A
:10824000300D11242D503040F801E20FF31F8981C9
:1082500080838B8181838D8182838F8183838985D4
:1082600084838E858583888986838A8987838C89A0
:1082700080878E898187888D82878C8D83878E8D7C
:108280008487888186FF04C0F801E20FF31F1586FA
:108290008B8583FDA6CF822F03C08FEF01C080E0C6
:1082A000DF91CF911F910F91FF90EF90DF90CF90D2
:1082B00008954115510509F08FCF90CFDF93CF93EB
:1082C0000F92CDB7DEB7BE016F5F7F4F41E050E048
:1082D0000E94C93F019719F02FEF3FEF03C089813A
:1082E000282F30E0C9010F90CF91DF910895EF92D0
:1082F000FF920F931F93CF93DF93EC018B8182301A
:1083000038F1E884F9840A851B85CE010E945E411C
:1083100097FD1EC088859985AA85BB854F96A11DAE
:10832000B11D88879987AA87BB87A5E01695079511
:10833000F794E794AA95D1F72E2D30E02F70307086
:10834000F5E0220F331FFA95E1F72A5B374F02C0A1
:1083500020E030E0C901DF91CF911F910F91FF9094
:10836000EF9008950F931F93CF93DF93EC018B0150
:108370008B81882309F040C0FB018789803109F097
:1083800041C082E08B831D8A1E8A1F8A188E808DD1
:10839000918DA0E0B0E045E0880F991FAA1FBB1F98
:1083A0004A95D1F7898B9A8BAB8BBC8B13C083E03A
:1083B0008B83F801428D538D648D758D4D8B5E8B53
:1083C0006F8B788F9E012F5E3F4FC8010E94174A26
:1083D000882391F01A8F098F81E089831C821D8286
:1083E0001E821F82188619861A861B861C861D8689
:1083F0001E861F86188A01C080E0DF91CF911F91F1
:108400000F9108958032C1F7D2CF1F93CF93DF939E
:10841000EC01142F262F30E0F90175E0EE0FFF1F5D
:108420007A95E1F7EA5BF74F8385817121F0842F1C
:10843000827109F069C08091420890914308A0912F
:108440004408B09145088C879D87AE87BF87688BAD
:10845000F90165E0EE0FFF1F6A95E1F7EA5BF74F60
:1084600084899589A0E0B0E0DC01992788278D8B6D
:108470009E8BAF8BB88F228D338DA90160E070E0A9
:10848000482B592B6A2B7B2B4D8B5E8B6F8B788FF8
:10849000838590E088719070009751F4848D958D5C
:1084A000A68DB78D898B9A8BAB8BBC8B81E00CC072
:1084B000409751F59E012F5E3F4F898D9A8D0E9406
:1084C000174A882309F184E08B83812F8F70898379
:1084D0001C821D821E821F82188619861A861B86A0
:1084E00014FF18C0CE0140E050E060E070E00E9450
:1084F000E03E882379F40AC049895A896B897C89CE
:10850000CE010E94973D02C01B8280E0DF91CF9197
:108510001F91089515FDF0CF81E0F8CFCF93DF9341
:10852000EC019C012C5F3F4F898D9A8D41E050E01A
:1085300060E070E00E94834A8823A1F08D899E89C3
:10854000AF89B88D0097A105B10559F48C819D8143
:10855000AE81BF818D8B9E8BAF8BB88F89818068F8
:10856000898381E0DF91CF9108952F923F924F92BE
:108570005F927F928F929F92AF92BF92CF92DF9243
:10858000EF92FF920F931F93DF93CF9300D000D011
:10859000CDB7DEB76C01162F072F5E834D83DC014C
:1085A00013968C911397813009F06FC111968C91BD
:1085B00081FF6BC188C1F601418952896389748941
:1085C00080859185A285B38584179507A607B7078F
:1085D00031F0C6010E94973D882309F456C1812FCE
:1085E000902F9C0119014D805E8013C1D6015996D0
:1085F000ED91FC915A97DA01C90149E0B695A7952A
:10860000979587954A95D1F774807A9478228FEF61
:10861000882E81E0982E82229322772009F053C081
:108620008114910409F04FC0D60114964D915D91CB
:108630006D917C911797411551056105710581F484
:1086400055968D919D910D90BC91A02D0097A105FF
:10865000B10561F1F60184839583A683B78333C0A6
:10866000CF019E012F5F3F4F0E944349882309F4A9
:108670000CC129813A814B815C81D6015996ED91DB
:10868000FC915A978789803149F4283FBFEF3B0717
:10869000B0E04B07B0E05B0778F008C0283FEFEF91
:1086A0003E07EFEF4E07EFE05E0730F0C6010E9495
:1086B0008E42882341F4E9C0D60114962D933D9350
:1086C0004D935C93179780E092E0881999095201C5
:1086D0008415950508F45C01D6015996ED91FC913D
:1086E0005A971496ED90FD900D911C9117978EEF6F
:1086F0009FEFAFEFBFEFE80EF91E0A1F1B1F0584A7
:1087000004C0EE0CFF1C001F111F0A94D2F78685CF
:108710009785A089B189E80EF91E0A1F1B1FE70C77
:10872000F11C011D111D90E0A91692E0B90639F562
:108730008091420890914308A0914408B091450867
:108740008E159F05A007B10771F41092480A8FEFAC
:108750009FEFAFEFBFEF8093420890934308A09341
:108760004408B09345088091460A9091470AB801A1
:10877000A70191010E946C3B8823B9F586C0811442
:10878000910419F5D60118962D913D914D915C916A
:108790001B9751968D919D910D90BC91A02D2817FE
:1087A00039074A075B0788F00E94DE46882309F4F0
:1087B0006CC081E08093480AE0924208F09243083E
:1087C000009344081093450808C0C801B70141E070
:1087D0000E941947882309F458C094012A5B374F37
:1087E000C901B101A5010E942B10950140E050E0A4
:1087F000F60180859185A285B385820F931FA41F02
:10880000B51F80879187A287B3872A0C3B1C4A1823
:108810005B08D60118962D913D914D915C911B9767
:108820004114510409F0E2CE51968D919D910D9025
:10883000BC91A02D82179307A407B50748F4F60151
:10884000218B328B438B548B81818068818311C053
:108850008091400890914108892B59F08D819E812B
:10886000892B39F0D60111968C9111978068119659
:108870008C93F601818183FF05C0C6010E94613E91
:10888000882319F04D815E8105C081E0D6018C936B
:108890004FEF5FEFCA0126960FB6F894DEBF0FBE0A
:1088A000CDBFCF91DF911F910F91FF90EF90DF909F
:1088B000CF90BF90AF909F908F907F905F904F90A0
:1088C0003F902F90089582FD76CE89CEDF92EF9271
:1088D000FF920F931F93CF93DF93EC0189899A89BD
:1088E000AB89BC89805E9F4FAF41B04008F071C03A
:1088F000CE010E948E42882309F46BC00E94DE469E
:10890000882309F466C0E98DFA8DEC80FD800E8124
:108910001F818EEF9FEFAFEFBFEFE80EF91E0A1F2A
:108920001B1F058404C0EE0CFF1C001F111F0A94BE
:10893000D2F786859785A089B189E80EF91E0A1FAE
:108940001B1F81E08093480AE0924208F09243089E
:10895000009344081093450880E092E0E6E4F8E0D4
:10896000DF019C011D9221503040E1F7DD24D394BA
:1089700011C0B801A7014D0D511D611D711D8091E0
:10898000460A9091470A26E438E00E946C3B88230F
:1089900001F1D394E98DFA8D8481D81650F320E04B
:1089A00032E040E050E0058404C0220F331F441F32
:1089B000551F0A94D2F789899A89AB89BC89820F9D
:1089C000931FA41FB51F898B9A8BAB8BBC8B81E047
:1089D00001C080E0DF91CF911F910F91FF90EF9048
:1089E000DF9008958F929F92AF92BF92CF92DF92C5
:1089F000EF92FF920F931F93CF93DF936C01EB01E4
:108A0000942E852EA22E898D9A8DD6015A969C93EE
:108A10008E935997CB0140E050E060E070E00E94F7
:108A2000973DBB2438C0CE010E947741FC010097DE
:108A300009F493C055E016950795F794E7945A9575
:108A4000D1F71E2D1F708081882311F0853EC9F457
:108A5000BB2099F42091420830914308409144088A
:108A600050914508D6011C962D933D934D935C93F0
:108A70001F9750961C93BB24B3948081882359F48C
:108A800018C0892D982DBF014BE050E00E941E10A8
:108A9000009709F470C0E884F9840A851B858989E8
:108AA0009A89AB89BC89E816F9060A071B0708F4FE
:108AB000BACFA6FE52C0A1FE50C0BB2051F0F601B5
:108AC0001089C60161E00E94403EEC01009769F404
:108AD00044C08B81823009F440C0CE010E946644BC
:108AE0008823D9F110E0C6E4D8E080E2DE011D92CF
:108AF0008A95E9F7DE01292D382DC901FC018BE0AB
:108B000001900D928150E1F7E0914008F091410809
:108B1000309739F0BE01625F7F4FCE0140961995C4
:108B200008C081E298E2998B888B80E098E09F876B
:108B30008E87888999899B8B8A8B998F888F8E8560
:108B40009F859F8B8E8B0E94DE46882331F0C60165
:108B5000612F4A2D0E94054201C080E0DF91CF9134
:108B60001F910F91FF90EF90DF90CF90BF90AF904B
:108B70009F908F900895A7FEEACFEFCF2F923F925C
:108B80004F925F926F927F928F929F92AF92BF921D
:108B9000CF92DF92EF92FF920F931F93DF93CF93C9
:108BA000CDB7DEB7C654D0400FB6F894DEBF0FBEC7
:108BB000CDBF3C016B01DE01AE5BBF4F11965C93F4
:108BC0004E9325962FAF25971C861F861FA21AA6A7
:108BD0006115710509F480C0FC018381882309F0C7
:108BE0007BC0FA0180818F32F1F08601ECE0EE2E3D
:108BF000F12CEC0EFD1E72E4A72EB12CAC0EBD1EA6
:108C00004E010894811C911C2796FFAEEEAE27976B
:108C100067E2262E312C2C0E3D1E270124C0119612
:108C2000B183A08301C0FD01A081B1818C918F32FD
:108C3000B1F3D60113968C91139782508230A8F22B
:108C40008E01095D1F4F59966D917C915A97C8010D
:108C50000E94B241882351F63FC0342D252D870153
:108C6000832F922F7C01F50180819181B401A501B0
:108C70000E944F3D882329F42FC03196D501ED93F2
:108C8000FC93D501ED91FC9180818F32B1F3882363
:108C9000C9F0C701B801A40121E00E94F244882371
:108CA000D9F00C151D0519F0C8010E94B13E279698
:108CB000EEADFFAD2797EE16FF0679F6C101322D16
:108CC000292FCDCFC301B801A40125962FAD25973B
:108CD0000E94F244182F01C010E0CE0187960E9436
:108CE000BB3ECE010C960E94BB3E812FCA5BDF4F7C
:108CF0000FB6F894DEBF0FBECDBFCF91DF911F91AD
:108D00000F91FF90EF90DF90CF90BF90AF909F902A
:108D10008F907F906F905F904F903F902F9008952D
:108D20000F931F93DF93CF93CDB7DEB76B970FB63B
:108D3000F894DEBF0FBECDBF9C01AB0119821C822F
:108D40008E010F5F1F4FC801B90122E00E94BE458E
:108D5000882311F410E004C0C8010E94AD3F182F11
:108D6000CE0101960E94BB3E812F6B960FB6F89400
:108D7000DEBF0FBECDBFCF91DF911F910F91089540
:108D8000DB010D900020E9F71197A61BB70B0496A5
:108D9000AD010E94B5420895DF93CF930F92CDB7F6
:108DA000DEB769830496BE016F5F7F4F41E050E0FC
:108DB0000E94B5420F90CF91DF9108958091480AAB
:108DC000882399F1409142085091430860914408EA
:108DD000709145088091460A9091470A26E438E050
:108DE0000E946C3B882319F14091490A50914A0A2C
:108DF00060914B0A70914C0A41155105610571054E
:108E000091F08091460A9091470A26E438E00E944A
:108E10006C3B882361F01092490A10924A0A109222
:108E20004B0A10924C0A1092480A81E0089580E0A3
:108E30000895DF92EF92FF920F931F937B018C01B5
:108E4000D42E8091420890914308A0914408B0919B
:108E500045088E159F05A007B107C1F00E94DE46A8
:108E60008823E1F08091460A9091470AB801A70152
:108E700026E438E00E94273C882381F0E0924208F3
:108E8000F09243080093440810934508DD2011F444
:108E900081E005C081E08093480A01C080E01F9115
:108EA0000F91FF90EF90DF9008958F929F92AF9275
:108EB000BF92CF92DF92EF92FF920F931F93CF93C7
:108EC000DF936C01142F7093470A6093460AFC01EC
:108ED000178A82E090E0A0E0B0E080839183A283D3
:108EE000B3831092480A1092490A10924A0A1092CB
:108EF0004B0A10924C0A8FEF9FEFAFEFBFEF8093BA
:108F0000420890934308A0934408B0934508442333
:108F100021F488249924540140C0453008F01EC132
:108F200060E070E080E090E040E00E941947882314
:108F300009F414C1C12FD0E02197FE0174E0EE0FB7
:108F4000FF1F7A95E1F7EA5BF74FE254FE4F80810D
:108F5000EE5BF14090E08F779070892B09F0FEC0B6
:108F6000E653FE4F80819181A281B38184369105C1
:108F7000A105B10508F4F2C064E0CC0FDD1F6A95CD
:108F8000E1F7C45FD54F88809980AA80BB808114A7
:108F90009104A104B10409F4E1C0C501B40140E0A9
:108FA0000E941947882309F4D9C0809151089091F3
:108FB00052088050924009F0D1C0209156082223D7
:108FC00009F4CCC08091540890915508892B09F47C
:108FD000C5C080915308882309F4C0C0F601228BD4
:108FE000809153088483158661E070E007C04F5F6D
:108FF000F60145874150483008F0B0C0F60145857C
:10900000848190E09B01042E02C0220F331F0A943A
:10901000E2F78217930759F720915C0830915D08B9
:109020002115310519F040E050E008C020916A0890
:1090300030916B0840916C0850916D08F6012583C2
:10904000368347835087E0905408F090550800E03D
:1090500010E0E80CF91C0A1D1B1DE38AF48A058B3D
:10906000168B8091570890915808918F808F60914E
:10907000560870E080E090E00E9491C56E0D7F1D63
:10908000801F911FF601628F738F848F958F2091BF
:1090900057083091580855E0220F331F5A95E1F7D1
:1090A00021503E4F232F3327269540E050E0260FD6
:1090B000371F481F591F26873787408B518B809158
:1090C000590890915A08009719F0A0E0B0E008C044
:1090D0008091660890916708A0916808B09169082E
:1090E00085017401E21AF30A040B150BA80197011C
:1090F000280F391F4A1F5B1FF601058404C05695CF
:109100004795379527950A94D2F721873287438769
:109110005487253FFFE03F07F0E04F07F0E05F078F
:1091200020F48CE0F601878B19C0255F3F4F40404B
:10913000504018F480E1F6010EC0809172089091C1
:109140007308A0917408B0917508F601828F938F0F
:10915000A48FB58F80E2878B81E001C080E0DF9132
:10916000CF911F910F91FF90EF90DF90CF90BF9024
:10917000AF909F908F9008956F927F928F929F9261
:10918000AF92BF92CF92DF92EF92FF920F931F9315
:10919000CF93DF93EC015A016B0138014901423052
:1091A00051056105710508F45EC089859A85AB8516
:1091B000BC850196A11DB11D84179507A607B707A9
:1091C00008F451C08F89803129F4E52EF62E072F3F
:1091D00011270CC0803209F046C07A018B0187E06C
:1091E00016950795F794E7948A95D1F78B899C8912
:1091F000AD89BE89E80EF91E0A1F1B1FC801B70101
:1092000041E00E941947882371F18F89803149F428
:10921000F501F070EE0FFF1FEA5BF74F718260827D
:109220000DC0F501EF77F070EE0FFF1FEE0FFF1F7F
:10923000EA5BF74F60827182828293828A898230F0
:1092400080F08D819E81AF81B885E80EF91E0A1FDE
:109250001B1FE092490AF0924A0A00934B0A1093AE
:109260004C0A81E001C080E0DF91CF911F910F9106
:10927000FF90EF90DF90CF90BF90AF909F908F9036
:109280007F906F900895CF92DF92EF92FF920F93AD
:109290001F93CF93DF93EC017A018B0169018985DC
:1092A0009A85AB85BC850196A11DB11D84179507D4
:1092B000A607B70708F453C08F89803129F45527D2
:1092C000412F302F2F2D0CC0803209F048C09A0159
:1092D000AB0167E056954795379527956A95D1F785
:1092E0008B899C89AD89BE89280F391F4A1F5B1F56
:1092F0008091420890914308A0914408B09145089C
:10930000281739074A075B0739F0CA01B90140E05D
:109310000E941947882319F18F89803159F4F70188
:10932000F070EE0FFF1FEA5BF74F80819181A0E0A4
:10933000B0E00EC0F701EF77F070EE0FFF1FEE0FF9
:10934000FF1FEA5BF74F80819181A281B381BF70DB
:10935000F60180839183A283B38381E001C080E022
:10936000DF91CF911F910F91FF90EF90DF90CF9001
:109370000895AF92BF92CF92DF92EF92FF920F9338
:109380001F93DF93CF9300D00F92CDB7DEB76C0160
:109390007A018B0182E090E0A0E0B0E0F6018083EA
:1093A0009183A283B3835E010894A11CB11CC60102
:1093B000B801A70195010E944349882341F1C601E4
:1093C000B801A70100E010E020E030E00E94BC48B6
:1093D0008823E9F0E980FA800B811C81F6018789F6
:1093E000803151F4F8EFEF16FFEFFF06F0E00F07C2
:1093F000F0E01F07E0F209C088EFE8168FEFF806EB
:109400008FEF08078FE0180790F281E001C080E03D
:109410000F900F900F900F90CF91DF911F910F91B0
:10942000FF90EF90DF90CF90BF90AF9008954F9254
:109430005F926F927F928F929F92AF92BF92CF92E4
:10944000DF92EF92FF920F931F93DF93CF9300D0A1
:109450000F92CDB7DEB76C0149835A836B837C834F
:109460003901EE24FF2487012E010894411C511C70
:10947000812CE2E09E2EA12CB12C49815A816B8176
:109480007C81C60192010E944349882339F1D501AC
:10949000C401F601058404C0880F991FAA1FBB1FD1
:1094A0000A94D2F7E80EF91E0A1F1B1F29813A8180
:1094B0004B815C818789803131F4285F3F4F404088
:1094C0005040D8F205C0285F3F4F4F4F5F40A8F291
:1094D000F301E082F1820283138381E00F900F9009
:1094E0000F900F90CF91DF911F910F91FF90EF9010
:1094F000DF90CF90BF90AF909F908F907F906F90B4
:109500005F904F9008952F923F924F925F926F928B
:109510007F928F929F92AF92BF92CF92DF92EF9203
:10952000FF920F931F93DF93CF93CDB7DEB72F97A3
:109530000FB6F894DEBF0FBECDBF1C014A875B8714
:109540006C877D873F872E87DC0119968D919D91D1
:109550000D90BC91A02D0196A11DB11D8E839F83FE
:10956000A887B987F9010081118122813381011512
:1095700011052105310549F0480159010894811C64
:10958000911CA11CB11C1D8210C0D1018D909D9019
:10959000AD90BC901D828A859B85AC85BD85019769
:1095A000A105B10511F491E09D8375016401442486
:1095B000552432018E010F5F1F4FF1018185928585
:1095C000A385B485481659066A067B0608F090C044
:1095D0008E819F81A885B9858C159D05AE05BF0537
:1095E00050F4A2E08A2E912CA12CB12CF2E0CF2EC7
:1095F000D12CE12CF12CC101B701A60198010E94E8
:109600004349882309F474C089819A81AB81BC8164
:10961000A70196012F5F3F4F4F4F5F4F0097A10566
:10962000B10519F049015A010DC0281939094A0933
:109630005B098A859B85AC85BD85281739074A0754
:109640005B0759F00894411C511C611C711C089463
:10965000C11CD11CE11CF11CB0CFC101A601B70196
:109660000FEF1FEF2FEF3FE00E94BC48882399F4D3
:109670003FC026013701089441085108610871086C
:10968000C101B301A201970186010E94BC48882351
:1096900079F1730162018C149D04AE04BF0448F398
:1096A000AE85BF854D915D916D917C9141155105C0
:1096B0006105710539F0C101950184010E94BC4822
:1096C0008823B1F0EE85FF8580829182A282B382E9
:1096D000FD81FF2359F00894811C911CA11CB11C31
:1096E000D1018D929D92AD92BC92139781E001C001
:1096F00080E02F960FB6F894DEBF0FBECDBFCF919E
:10970000DF911F910F91FF90EF90DF90CF90BF906E
:10971000AF909F908F907F906F905F904F903F9011
:109720002F9008952F923F924F925F926F927F9267
:109730008F929F92AF92BF92CF92DF92EF92FF9261
:109740000F931F93DF93CF93CDB7DEB7CD55D040A6
:109750000FB6F894DEBF0FBECDBF2F969FAF8EAF72
:109760002F9761967FAF6EAF61972A0162962FAFF8
:10977000629763960FAF63976496EFAE64976896AF
:10978000ACAEBDAECEAEDFAE6897E22EFF24EE0CDF
:10979000FF1CEE0CFF1C9A012E0D3F1D2D963FAFB6
:1097A0002EAF2D97D9016D907D908D909C90FC01EE
:1097B000EE0DFF1DC401B30120813181428153812F
:1097C0000E9406C169AF7AAF8BAF9CAF10E0000F6B
:1097D000111F000F111FF201E00FF11F2B96FFAFB9
:1097E000EEAF2B97A080B180C280D3802F96EEADD4
:1097F000FFAD2F97E00FF11FC601B5012081318128
:10980000428153810E9406C16DAB7EAB8FAB98AF96
:1098100064962FAD6497E22FF0E0EE0FFF1FEE0F7E
:10982000FF1F2F96AEADBFAD2F97AE0FBF1F4D914F
:109830005D916D917C9129964CAF5DAF6EAF7FAF1E
:10984000299761966EAD7FAD6197E60FF71F608136
:1098500071818281938129962CAD3DAD4EAD5FAD76
:1098600029970E9405C169AB7AAB8BAB9CAB619623
:10987000AEADBFAD61971C968D919D910D90BC9141
:10988000A02D25968CAF9DAFAEAFBFAF25972F967D
:10989000AEADBFAD2F971C962D913D914D915C9132
:1098A0001F9721962CAF3DAF4EAF5FAF2197A4011C
:1098B000930150582DA73EA74FA758ABB601A5015D
:1098C000705849A75AA76BA77CA761966EAD7FAD6C
:1098D0006197E60EF71ED7016D917D918D919C9158
:1098E00029AD3AAD4BAD5CAD0E9405C13B014C01C9
:1098F0006196EEADFFAD61970E0F1F1FD8016D9100
:109900007D918D919C912DA93EA94FA958AD0E94A2
:1099100005C15B016C016DA57EA58FA598A9A60167
:1099200095010E94BFC47B018C0169A57AA58BA516
:109930009CA5A40193010E94BFC49B01AC01C80176
:10994000B7010E9405C11B012C016DA57EA58FA545
:1099500098A9A40193010E94BFC47B018C0169A551
:109960007AA58BA59CA5A60195010E94BFC49B0169
:10997000AC01C801B7010E9406C19B01AC01C20144
:10998000B1010E9479C15B016C0120E030E040E050
:1099900050E00E94DFC1882354F4C601B5012BEDCD
:1099A0003FE049EC50E40E9406C15B016C01E8967F
:1099B0008FADE897882351F0C601B5012BED3FE04C
:1099C00049EC50E40E9405C15B016C01C601B50180
:1099D000E7962CAD3DAD4EAD5FADE7970E94BFC49D
:1099E00029A93AA94BA95CA95F770E94FAC37B0118
:1099F0008C012FE632E143E85AE30E94DFC187FD84
:109A0000F6C1C801B7010E94BCC20E9453C278A728
:109A10006FA3672B21F4E1E0F0E0F8A7EFA32FA1FB
:109A200038A5B90180E090E00E947FC27B018C01E3
:109A3000C601B501A80197010E94E6C16BA37CA3F2
:109A40008DA39EA369A97AA98BA99CA9A8019701B6
:109A50000E94E6C16F8F78A389A39AA325966CAD67
:109A60007DAD8EAD9FAD259721962CAD3DAD4EAD14
:109A70005FAD21970E9405C1A80197010E94E6C130
:109A80006B8F7C8F8D8F9E8F6BA17CA18DA19EA1F2
:109A900020E030E040E05FEB0E94BFC42BA13CA17E
:109AA0004DA15EA10E94BFC420E030E040E85FE32A
:109AB0000E9406C16F8B788F898F9A8F64963FAD15
:109AC0006497E32FF0E0EE0FFF1FEE0FFF1F9E01E4
:109AD0002F5F3F4FE20FF31F29964CAD5DAD6EAD8A
:109AE0007FAD299740835183628373832F96AEADF8
:109AF000BFAD2F971C964D915D916D917C911F97F5
:109B00004D875E876F87788B41E050E05A8B498B99
:109B1000662462967FAD6297672F70E0660F771FAD
:109B2000660F771FC901860F971F6A969FAF8EAF8A
:109B30006A976396BFAD6397AB2FB0E0AA0FBB1FC8
:109B4000AA0FBB1F21E030E02C0F3D1F2A0F3B1F47
:109B50006C963FAF2EAF6C976E96FFAFEEAF6E97E1
:109B60001AC138E136150CF446C06DA57EA58FA547
:109B700098A92BA13CA14DA15EA10E94BFC47B016D
:109B80008C0169A57AA58BA59CA52F89388D498D57
:109B90005A8D0E94BFC49B01AC01C801B7010E944D
:109BA00006C17B018C016DA57EA58FA598A92F8983
:109BB000388D498D5A8D0E94BFC45B016C0169A527
:109BC0007AA58BA59CA52BA13CA14DA15EA10E94CD
:109BD000BFC49B01AC01C601B5010E9405C16DA7C0
:109BE0007EA78FA798AB6394C701D80189A79AA7CE
:109BF000ABA7BCA765C049895A89BA0180E090E04B
:109C00000E947FC22BA13CA14DA15EA10E94BFC4B6
:109C10007B018C01C8010E94E3C16B8B7C8B8D8B17
:109C20009E8BB701C8010E9422C53B014C012D96B5
:109C3000AEADBFAD2D97ED90FD900D911C9117FB32
:109C4000109517F910952B96EEADFFAD2B97208050
:109C5000318042805380C801B7012B893C894D89EE
:109C60005E890E94BFC45B016C01C201B101A40105
:109C700093010E94BFC49B01AC01C601B5010E94C3
:109C800006C16DA77EA78FA798ABC801B701A40135
:109C900093010E94BFC47B018C01C201B1012B89D9
:109CA0003C894D895E890E94BFC49B01AC01C801FB
:109CB000B7010E9405C169A77AA78BA79CA7662454
:109CC00069AD7AAD8BAD9CAD2DA53EA54FA558A92C
:109CD0000E9406C16A96AEADBFAD6A976D937D9343
:109CE0008D939C9313976DA97EA98FA998AD29A5F3
:109CF0003AA54BA55CA50E9406C16C96EEADFFADE2
:109D00006C9760837183828393836E96AEADBFAD93
:109D10006E976D917D918D919C912F8D38A149A168
:109D20005AA10E9406C16E96EEADFFAD6E9760839C
:109D30007183828393836D857E858F8598892B8D32
:109D40003C8D4D8D5E8D0E9406C16D877E878F870D
:109D5000988BCE0101960E94C917CE010196BE01D3
:109D60006B5F7F4FAE01475F5F4F9E01235F3F4FA9
:109D70006896ECACFDAC0EAD1FAD6897F8E7CF2E42
:109D8000D12CCC0EDD1E0E944E5429893A892F5FBA
:109D90003F4F3A8B298B49895A896FA178A546177D
:109DA000570708F4DECE61964EAD5FAD6197485F10
:109DB0005F4F61962EAD3FAD6197245F3F4F619637
:109DC0008EAD9FAD6197DC0114966196BFAFAEAFCB
:109DD0006197BD016896ECACFDAC0EAD1FAD689708
:109DE000E8E7CE2ED12CCC0EDD1E0E944E54C35A75
:109DF000DF4F0FB6F894DEBF0FBECDBFCF91DF911E
:109E00001F910F91FF90EF90DF90CF90BF90AF9098
:109E10009F908F907F906F905F904F903F902F908A
:109E2000089580918D0F90918E0F891B8F700895EA
:109E300080938F0F0895FC016081718182819381ED
:109E400020916D0A30916E0A40916F0A5091700A0C
:109E50000E94BFC40E948FC46093B90A7093BA0A6B
:109E60008093BB0A9093BC0A89EB9AE00E947161CF
:109E700008958F929F92AF92BF92CF92DF92EF920E
:109E8000FF920F931F93FC018B015A0149016081DE
:109E90007181828193812091610A3091620A40919F
:109EA000630A5091640A0E94BFC40E948FC43DEAB5
:109EB000C32E3AE0D32E6093AD0A7093AE0A80931E
:109EC000AF0A9093B00AF801608171818281938119
:109ED0002091650A3091660A4091670A5091680A9C
:109EE0000E94BFC40E948FC424E0E22EF12CEC0C2F
:109EF000FD1C6093B10AF701718382839383F5019E
:109F000060817181828193812091690A30916A0A0E
:109F100040916B0A50916C0A0E94BFC40E948FC48A
:109F20008601085F1F4F6093B50AF8017183828331
:109F30009383F401608171818281938120916D0A04
:109F400030916E0A40916F0A5091700A0E94BFC40E
:109F50000E948FC4F6013C966093B90A7183828394
:109F60009383C601B701A8019F010E94376180E079
:109F700090E0A0E0B0E08093900F9093910FA093B9
:109F8000920FB093930F8093940F9093950FA0939B
:109F9000960FB093970F8093980F9093990FA0937B
:109FA0009A0FB0939B0F80939C0F90939D0FA0935B
:109FB0009E0FB0939F0F8093A00F9093A10FA0933B
:109FC000A20FB093A30F1F910F91FF90EF90DF901E
:109FD000CF90BF90AF909F908F9008958F929F9257
:109FE000AF92BF92CF92DF92EF92FF920F931F93A7
:109FF000CF93DF93EC016B01009709F45CC08FA94C
:10A00000882309F058C0EEA0FFA008A519A5FB0100
:10A01000B6A0A7A090A481A4C801B7012B2D3A2D0A
:10A02000492D582D0E94DFC188230CF044C0C8017F
:10A03000B701A80197010E94BFC47B018C016AA9E6
:10A040007BA98CA99DA9905820E030E040E050EC1D
:10A050000E94BFC42EA53FA548A959A90E94BFC40C
:10A060009B01AC01C801B7010E9406C10E942CC52A
:10A070007B018C016B2D7A2D892D982D9701A801DC
:10A080000E94DFC1882324F4EB2CFA2C092D182D13
:10A090006B2D7A2D892D982D9701A8010E94DFC183
:10A0A000882349F0C701D801F60186A397A3A0A78A
:10A0B000B1A781E086ABDF91CF911F910F91FF9007
:10A0C000EF90DF90CF90BF90AF909F908F900895CA
:10A0D000EF92FF920F931F93CF93DF93F0908E0F29
:10A0E00000E010E020E030E04DE4E42E12C0FE9CE1
:10A0F000E0011124C354D54FC901B801AE010E943B
:10A10000EE4F8F2D8F5F803109F480E0F82E98019B
:10A110008E0180918D0FF81651F7C901B80140E00A
:10A1200050E00E94EE4FDF91CF911F910F91FF9071
:10A13000EF900895AF92BF92CF92DF92EF92FF928D
:10A140000F931F93CF93DF93EB018A016115710584
:10A1500009F466C04115510509F462C0DAA4CBA424
:10A16000BCA4ADA46EA17FA188A599A52D2D3C2DE1
:10A170004B2D5A2D0E94DFC1882309F451C08FA9AD
:10A18000882309F043C0F801E6A0F7A000A511A5B7
:10A190006D2D7C2D8B2D9A2DA80197010E94EDC36A
:10A1A0001816A4F5C801B701A80197010E94BFC401
:10A1B0007B018C016AA97BA98CA99DA9905820E0FC
:10A1C00030E040E050EC0E94BFC42EA53FA548A956
:10A1D00059A90E94BFC49B01AC01C801B7010E94EC
:10A1E00006C10E942CC57B018C016D2D7C2D8B2D11
:10A1F0009A2D9701A8010E94DFC1882324F4ED2C39
:10A20000FC2C0B2D1A2DC701D80104C08D2D9C2DBF
:10A21000AB2DBA2D8EA39FA3A8A7B9A781E08EABC3
:10A22000DF91CF911F910F91FF90EF90DF90CF9032
:10A23000BF90AF900895CF92DF92EF92FF920F936D
:10A24000DF93CF930F920F92CDB7DEB780918D0F32
:10A250008FB7F894F0908E0F8FBF80918D0F90E0A4
:10A2600040968F1991098F709070049704F10091B6
:10A270008D0F03500F70CC24DD2440E050E06DE4DE
:10A28000E62E13C0802F002309F480E1082F01502F
:10A290000E9DC00111248354954F9A838983B60182
:10A2A0000E949A50A601C980DA800F1559F70F90C5
:10A2B0000F90CF91DF910F91FF90EF90DF90CF90B3
:10A2C00008956091E60590918E0F80918D0F9817FB
:10A2D000B9F040918E0F242F30E08DE490E0289F5C
:10A2E000F001299FF00D389FF00D1124EB5FF44F22
:10A2F000608102C04F5F4F7080918D0F4817D1F77A
:10A3000087E070E00E942A14089510928D0F109239
:10A310008E0F80E1EDEAFAE0DF011D928A95E9F700
:10A3200080E090E0A0E0B0E08093940F9093950FD0
:10A33000A093960FB093970F8093980F9093990FD7
:10A34000A0939A0FB0939B0F80939C0F90939D0FB7
:10A35000A0939E0FB0939F0F8093A00F9093A10F97
:10A36000A093A20FB093A30F8093900F9093910F9F
:10A37000A093920FB093930F08952F923F924F9214
:10A380005F926F927F928F929F92AF92BF92CF9285
:10A39000DF92EF92FF920F931F93DF93CF93CDB78E
:10A3A000DEB766970FB6F894DEBF0FBECDBF9E8BAB
:10A3B0008D8B6A017B0148015901DC01D8966D91B2
:10A3C0007D918D919C91DB970E947FC2698B7A8BE6
:10A3D0008B8B9C8BA70196010E94BFC40E94CCC1AD
:10A3E0000E9453C26D837E838F83988769897A899F
:10A3F0008B899C89A50194010E94BFC40E94CCC195
:10A400000E9453C269837A838B839C832D813E8112
:10A410004F815885283731054105510540F448E7FB
:10A4200050E060E070E04D835E836F8378876981E0
:10A430007A818B819C81683771058105910540F493
:10A4400088E790E0A0E0B0E089839A83AB83BC8387
:10A45000AD89BE89AC5BBF4FAD90BD90CD90DC9017
:10A460001397A454B040BE8BAD8BDC966D917D915B
:10A470008D919C91DF970E947FC26D877E878F8729
:10A48000988BC601B5010E9481C21B012C0120E0FE
:10A4900030E040E050E00E94DFC1882321F4E0E09A
:10A4A00070E060E028C069897A898B899C899B016A
:10A4B000AC010E94BFC47B018C016D857E858F85B8
:10A4C00098899B01AC010E94BFC49B01AC01C801EB
:10A4D000B7010E9405C17B018C01C201B101A2013B
:10A4E00091010E9406C19B01AC01C801B7010E9405
:10A4F000E6C1E62F692F2E2F372F482F562FB9018F
:10A50000CA010E94CCC10E944EC23B014C01ED89A0
:10A51000FE89E05CFF4F60817181828193810E949E
:10A520007FC269877A878B879C8766277727CB01CD
:10A530006A197B098C099D090E9481C25B016C012B
:10A5400020E030E040E050E00E94DFC1882321F4A9
:10A55000E0E070E060E028C069857A858B859C85A5
:10A560009B01AC010E94BFC47B018C0169897A897F
:10A570008B899C899B01AC010E94BFC49B01AC01EB
:10A58000C801B7010E9405C17B018C01C601B5015C
:10A59000A60195010E9406C19B01AC01C801B7014B
:10A5A0000E94E6C1E62F692F2E2F372F482F562FF6
:10A5B000B901CA010E94BCC2ED89FE89A088B18898
:10A5C000C288D38886017501E618F70808091909B9
:10A5D0000E944EC2A8019701261B370B480B590B4E
:10A5E00057FF71C0C201B10120E030E040E050E00F
:10A5F0000E94DFC1882321F4E0E070E060E044C005
:10A60000C201B101A20191010E9406C17B018C012E
:10A61000C601B5010E947FC29B01AC01C801B70110
:10A620000E94BFC47B018C016D857E858F859889D2
:10A630009B01AC010E94BFC49B01AC01C801B701E2
:10A640000E9405C17B018C0169857A858B859C857B
:10A650009B01AC010E94BFC49B01AC01C801B701C2
:10A660000E9406C17B018C01C201B10120E030E0F3
:10A6700040E850E40E94BFC49B01AC01C801B7018F
:10A680000E94E6C1E62F692F2E2F372F482F562F15
:10A69000B901CA010E94CCC10E944EC2AC01CB01DB
:10A6A000DA013C014D0197FE03C066247724430183
:10A6B0006A147B048C049D0410F03501460120E0EF
:10A6C00030E040E050E09FB7F8946D897E89645B8C
:10A6D0007F4FDB018C91AC54B040BE8BAD8B882397
:10A6E00021F5FD01648A758A868A978A260D371DB1
:10A6F000481D591D58962D933D934D935C935B9740
:10A700002D813E814F815885DC962D933D934D934D
:10A710005C93DF97A05CBF4F29813A814B815C81BC
:10A720002D933D934D935C9313979FBF66960FB601
:10A73000F894DEBF0FBECDBFCF91DF911F910F9177
:10A74000FF90EF90DF90CF90BF90AF909F908F9051
:10A750007F906F905F904F903F902F9008954F9211
:10A760005F927F928F929F92AF92BF92CF92DF9231
:10A77000EF92FF920F931F93CF93DF9370908E0F02
:10A78000C0E0D0E07DE4472E512C46C02097B1F1C7
:10A790008EA9882361F4849CF001859CF00D949C23
:10A7A000F00D1124E354F54F86A9882339F1EAA06E
:10A7B000FBA00CA11DA16EA17FA188A599A5A80150
:10A7C00097010E94E6C15B016C01849CF001859CAD
:10A7D000F00D949CF00D1124E354F54F66A177A180
:10A7E00080A591A5A80197010E94E6C18B019C015B
:10A7F000CE01B601A5010E94BD511EAA739480E14D
:10A80000781609F47724849CE001859CD00D949CF3
:10A81000D00D1124C354D54F872C992487FC9094D4
:10A8200080918D0F90E08816990609F0AFCF2097A0
:10A83000F1F0EAA0FBA00CA11DA16EA17FA188A54B
:10A8400099A5A80197010E94E6C15B016C016DEC1E
:10A850007CEC8CE49DE3A80197010E94E6C18B018A
:10A860009C01CE01B601A5010E94BD511EAADF9137
:10A87000CF911F910F91FF90EF90DF90CF90BF90FD
:10A88000AF909F908F907F905F904F9008950E941F
:10A890001B510E9468500E94AF5308952F923F921F
:10A8A0004F925F926F927F928F929F92AF92BF92E0
:10A8B000CF92DF92EF92FF920F931F93DF93CF938C
:10A8C000CDB7DEB7C859D0400FB6F894DEBF0FBE83
:10A8D000CDBF5C014B013A012901CB56DF4FE88225
:10A8E000C559D040CA56DF4FF882C659D040C95624
:10A8F000DF4F0883C759D040C856DF4F1883C85967
:10A90000D040E396DFAECEAEE39780918D0F8F5FA0
:10A91000803109F480E0282F332727FD30953CA7AC
:10A920002BA706C00E94AC6E0E941D190E9443BD59
:10A9300080918E0F90E04BA55CA58417950791F34D
:10A940006091610A7091620A8091630A9091640A31
:10A95000E1966CAF7DAF8EAF9FAFE197D5012D91A2
:10A960003D914D915C910E94BFC40E948FC4C1581B
:10A97000DF4F6883CF57D040C058DF4F7883C0582F
:10A98000D040CF57DF4F8883C158D040CE57DF4FDC
:10A990009883C258D0402091650A3091660A409150
:10A9A000670A5091680AAD962CAF3DAF4EAF5FAFCE
:10A9B000AD97CA01B901D4012D913D914D915C91A2
:10A9C0000E94BFC40E948FC4CD57DF4F6883C35815
:10A9D000D040CC57DF4F7883C458D040CB57DF4F9F
:10A9E0008883C558D040CA57DF4F9883C658D04097
:10A9F0002091690A30916A0A40916B0A50916C0A61
:10AA0000A9962CAF3DAF4EAF5FAFA997CA01B90170
:10AA1000D3012D913D914D915C910E94BFC40E9444
:10AA20008FC4C957DF4F6883C758D040C857DF4F1E
:10AA30007883C858D040C757DF4F8883C958D04063
:10AA4000C657DF4F9883CA58D04020916D0A309185
:10AA50006E0A40916F0A5091700AA5962CAF3DAFD7
:10AA60004EAF5FAFA597CA01B901D2012D913D91BB
:10AA70004D915C910E94BFC40E948FC4C557DF4FA7
:10AA80006883CB58D040C457DF4F7883CC58D04030
:10AA9000C357DF4F8883CD58D040C257DF4F9883CC
:10AAA000CE58D0408091B90A9091BA0AA091BB0AC1
:10AAB000B091BC0AC557DF4F288139814A815B813B
:10AAC000CB58D040281739074A075B0709F4B9C0AB
:10AAD000E091E505F0E0EE0FFF1FEE0FFF1FE950DC
:10AAE000F04F608171818281938120E030E04AE201
:10AAF00053E40E94DFC188230CF038C080918F0F8F
:10AB0000882309F033C0C557DF4F488159816A81D6
:10AB10007B81CB58D0404093B90A5093BA0A6093D6
:10AB2000BB0A7093BC0AE9EAF7E0949108C08091EF
:10AB3000C00085FFFCCF9093C60031969491992375
:10AB4000B1F7EDECF7E0949108C08091C00085FF6B
:10AB5000FCCF9093C600319694919923B1F78091E0
:10AB6000C00085FFFCCF8AE08093C6008091B90ABF
:10AB70009091BA0AA091BB0AB091BC0AC557DF4FA9
:10AB8000288139814A815B81CB58D040281B390B01
:10AB90004A0B5B0BCA01B90157FF07C0909580951E
:10ABA000709561957F4F8F4F9F4F0E9481C27B01AF
:10ABB0008C01A5966CAD7DAD8EAD9FADA59720E0C7
:10ABC00030E04DEC53E40E94BFC49B01AC01C801CE
:10ABD000B7010E94EDC318160CF033C0C557DF4F04
:10ABE000488159816A817B81CB58D0404093B90A12
:10ABF0005093BA0A6093BB0A7093BC0AE9EAF7E083
:10AC0000949108C08091C00085FFFCCF9093C6004E
:10AC1000319694919923B1F7EFEAF7E0949108C047
:10AC20008091C00085FFFCCF9093C600319694912F
:10AC30009923B1F78091C00085FFFCCF8AE0809313
:10AC4000C60080918D0F682F70E0A1967FAF6EAF28
:10AC5000A1978DE490E0689FF001699FF00D789FC7
:10AC6000F00D1124E354F54FE45BFF4F1082EC54D8
:10AC7000F0408091AD0A9091AE0AA091AF0AB091D8
:10AC8000B00A6F968CAF9DAFAEAFBFAF6F97C15894
:10AC9000DF4F288139814A815B81CF57D040281B03
:10ACA000390B4A0B5B0B6B962CAF3DAF4EAF5FAFD2
:10ACB0006B97208331834283538357FF0DC0DA01A2
:10ACC000C901B095A095909581959F4FAF4FBF4F0B
:10ACD00080839183A283B3834091B10A5091B20AD9
:10ACE0006091B30A7091B40A67964CAF5DAF6EAFD6
:10ACF0007FAF6797CD57DF4F88819981AA81BB814C
:10AD0000C358D040841B950BA60BB70B63968CAF32
:10AD10009DAFAEAFBFAF63978DE490E0A196AEADAF
:10AD2000BFADA197A89FF001A99FF00DB89FF00DAE
:10AD30001124E354F54F63962CAD3DAD4EAD5FADA0
:10AD40006397248335834683578357FF0DC0DA0109
:10AD5000C901B095A095909581959F4FAF4FBF4F7A
:10AD600084839583A683B7834091B50A5091B60A30
:10AD70006091B70A7091B80A2F964CAF5DAF6EAF75
:10AD80007FAF2F97C957DF4F88819981AA81BB81F7
:10AD9000C758D040841B950BA60BB70B2B968CAFD6
:10ADA0009DAFAEAFBFAF2B978DE490E0A196AEAD57
:10ADB000BFADA197A89FF001A99FF00DB89FF00D1E
:10ADC0001124E354F54F2B962CAD3DAD4EAD5FAD48
:10ADD0002B97208731874287538757FF0DC0DA01B1
:10ADE000C901B095A095909581959F4FAF4FBF4FEA
:10ADF00080879187A287B3872090B90A3090BA0ADA
:10AE00004090BB0A5090BC0AC557DF4F488159811A
:10AE10006A817B81CB58D040421953096409750976
:10AE20004DA35EA36FA378A760916E0370916F032B
:10AE300027967FAF6EAF27976DA17EA18FA198A5B2
:10AE400097FF07C090958095709561957F4F8F4FC4
:10AE50009F4F2796AEADBFAD27979D01442737FD85
:10AE60004095542F0E9491C524E630E040E050E028
:10AE70000E94F9C58DE490E0A1966EAD7FADA197DB
:10AE8000689FF001699FF00D789FF00D1124E35445
:10AE9000F54FDF011C96248711963C93119712966B
:10AEA0004C93129713965C9360807180828093809C
:10AEB000A480B580C680D780E084F18402851385A4
:10AEC000C901DA018E159F05A007B10714F4D80156
:10AED000C7018A159B05AC05BD0514F4D601C50153
:10AEE0009C01AD0186159705A805B90514F4A401C8
:10AEF00093018DE490E0A196AEADBFADA197A89F60
:10AF0000B001A99F700DB89F700D11246354754F47
:10AF1000FB01208B318B428B538B26303105410551
:10AF2000510510F40C948960E85BFF4F8091E605B1
:10AF30009091E705AA2797FDA095BA2F808391836A
:10AF4000A283B383DB0190961C92C158DF4F288106
:10AF500039814A815B81CF57D0406F968CAD9DADD2
:10AF6000AEADBFAD6F97281739074A075B0724F4CA
:10AF700081E0DB0190968C93CD57DF4F288139819A
:10AF80004A815B81C358D04067966CAD7DAD8EAD74
:10AF90009FAD6797261737074807590794F48DE444
:10AFA00090E0A196AEADBFADA197A89FF001A99F7B
:10AFB000F00DB89FF00D1124E354F54F80A182608D
:10AFC00080A3C957DF4F288139814A815B81C758E7
:10AFD000D0402F966CAD7DAD8EAD9FAD2F972617CF
:10AFE00037074807590794F48DE490E0A196AEAD79
:10AFF000BFADA197A89FF001A99FF00DB89FF00DDC
:10B000001124E354F54F80A1846080A3C557DF4F1E
:10B01000288139814A815B81CB58D0402215330584
:10B020004405550594F48DE490E0A1964EAD5FADD6
:10B03000A197489FF001499FF00D589FF00D1124F2
:10B04000E354F54F80A1886080A38DE490E0A19641
:10B050006EAD7FADA197689FF001699FF00D789F5D
:10B06000F00D1124E354F54FE396AEADBFADE39779
:10B070008C9181A3208131814281538125962CAF0F
:10B080003DAF4EAF5FAF2597211531054105510505
:10B0900009F015988DE490E0A1964EAD5FADA197B3
:10B0A000489FF001499FF00D589FF00D1124E35483
:10B0B000F54F6480758086809780611471048104E7
:10B0C000910409F017988DE490E0A1966EAD7FADE4
:10B0D000A197689FF001699FF00D789FF00D1124F2
:10B0E000E354F54FA084B184C284D384A114B10485
:10B0F000C104D10409F042988DE490E0A196AEAD70
:10B10000BFADA197A89FF001A99FF00DB89FF00DCA
:10B110001124E354F54F84859585A685B78500975E
:10B12000A105B10591F0A0989FB7F89480910B010B
:10B130008D7F80930B019FBF2090810A3090820AFF
:10B140004090830A5090840A08C02090990A309059
:10B150009A0A40909B0A50909C0ACB56DF4F688118
:10B16000C559D040CA56DF4F7881C659D040C9561C
:10B17000DF4F8881C759D040C856DF4F9881C859E2
:10B18000D040A20191010E94DFC187FD16C0CB56BD
:10B19000DF4F8881C559D040CA56DF4F9881C659C4
:10B1A000D040C956DF4FA881C759D040C856DF4F9D
:10B1B000B881C859D0401C012D016B966CAD7DAD96
:10B1C0008EAD9FAD6B970E9481C2E1962CAD3DADD7
:10B1D0004EAD5FADE1970E94E6C1EC966FAFEC9784
:10B1E000ED967FAFED97EE968FAFEE97EF969FAF10
:10B1F000EF97AC01CB01DA0189839A83AB83BC83DF
:10B2000063966CAD7DAD8EAD9FAD63970E9481C29C
:10B21000AD962CAD3DAD4EAD5FADAD970E94E6C194
:10B22000E8966FAFE897E9967FAFE997EA968FAF18
:10B23000EA97EB969FAFEB97AC01CB01DA018D83D8
:10B240009E83AF83B8872B966CAD7DAD8EAD9FADE1
:10B250002B970E9481C2A9962CAD3DAD4EAD5FAD3E
:10B26000A9970E94E6C1E4966FAFE497E5967FAF99
:10B27000E597E6968FAFE697E7969FAFE797AC0125
:10B28000CB01DA0189879A87AB87BC876DA17EA144
:10B290008FA198A50E9481C2A5962CAD3DAD4EAD63
:10B2A0005FADA5970E94E6C17B018C012796EEADAC
:10B2B000FFAD2797BF01882777FD8095982F0E94C3
:10B2C00081C29B01AC01C801B7010E94BFC420E04C
:10B2D00030E048EC52E40E94E6C19B01AC016D876E
:10B2E0007E878F87988B25966CAD7DAD8EAD9FAD9B
:10B2F000259766307105810591051CF576E0671686
:10B30000710481049104ECF486E0A816B104C10430
:10B31000D104BCF48DE490E0A196AEADBFADA19791
:10B32000A89FF001A99FF00DB89FF00D1124E354E0
:10B33000F54FDA01C901BF7786A797A7A0ABB1ABDC
:10B3400055C0EC962FADEC97ED963FADED97EE9690
:10B350004FADEE97EF965FADEF97B901CA010E942E
:10B3600076C53B014C01E8962FADE897E9963FADD5
:10B37000E997EA964FADEA97EB965FADEB97B90187
:10B38000CA010E9476C55B016C01E4962FADE4977B
:10B39000E5963FADE597E6964FADE697E7965FAD4C
:10B3A000E797B901CA010E9476C57B018C01C401EF
:10B3B000B301A60195010E9406C1A80197010E9450
:10B3C00006C10E942CC52DE430E0A1964EAD5FADC4
:10B3D000A197429FF001439FF00D529FF00D112461
:10B3E000E354F54F66A777A780AB91AB8DE490E06F
:10B3F000A1966EAD7FADA197689FF001699FF00D9A
:10B40000789FF00D1124E354F54F86A597A5A0A9C8
:10B41000B1A921968CAF9DAFAEAFBFAF219760E0D1
:10B4200070E080E89FE321962CAD3DAD4EAD5FAD61
:10B4300021970E94E6C19B01AC01C201B1010E94AB
:10B44000BFC42B013C0180918D0F90918E0FA82FCE
:10B45000B0E05096A91BB109AF70B070BAA7A9A708
:10B46000A230B1050CF451C05D01CC24B7FCC094EE
:10B47000DC2CC601B5010E9481C220E030E040E032
:10B4800051E40E94DFC188230CF03FC060E074E209
:10B4900084E799E4A30192010E94E6C10E948FC44F
:10B4A0007B018C0160914D0A70914E0A80914F0A88
:10B4B0009091500AE616F7060807190730F56E193D
:10B4C0007F09800B910B660F771F881F991FA601BC
:10B4D00095010E94D7C5CA01B9010E947FC20E948E
:10B4E0008FC49B01AC012E0D3F1D401F511FCA018F
:10B4F000B9010E947FC29B01AC0160E074E284E765
:10B5000099E40E94E6C12B013C018DE490E0A196F4
:10B51000EEADFFADA197E89F8001E99F100DF89F68
:10B52000100D11240354154F21966CAD7DAD8EADD9
:10B530009FAD2197A30192010E94BFC4D8019296AA
:10B540006D937D938D939C93959750966D917D917E
:10B550008D919C9153970E947FC2A30192010E94FA
:10B56000BFC40E94CCC10E9453C2F80160AF71AF4A
:10B5700082AF93AFC157DF4F1882CF58D040C0572A
:10B58000DF4F1882C059D04020E8222E9FE3392E89
:10B5900088249924E1E0F0E0EC0FFD1FE80DF91D8F
:10B5A000C301B20120813181428153810E94BFC415
:10B5B000E1E1F0E0EC0FFD1FE80DF91D6083718300
:10B5C000828393835B016C01E894D7F8F401EF5A0E
:10B5D000F54FE080F18002811381C601B501A80119
:10B5E00097010E94EDC31816CCF4C801B701A6015B
:10B5F00095010E94E6C16B017C01C157DF4F688154
:10B60000CF58D040C057DF4F7881C059D040C101DA
:10B61000A70196010E94DFC188236CF4C157DF4F58
:10B620008881CF58D040C057DF4F9881C059D04053
:10B63000D1016C017D0124E030E0820E931E30E1E7
:10B640008316910471F0D701C601C157DF4FC8823C
:10B65000CF58D040C057DF4F9883C059D0401D010C
:10B6600099CFC701B60120E030E040E85FE30E94D7
:10B67000DFC188230CF04CC08E010F5E1F4F81E2AA
:10B68000A82EB12CAC0EBD1ED8016D917D918D916F
:10B690009C91A70196010E94BFC4F8016193719328
:10B6A000819391938F01EA15FB0571F78DE490E08A
:10B6B000A1962EAD3FADA197289F8001299F100D27
:10B6C000389F100D11240354154FD80192966D9197
:10B6D0007D918D919C919597A70196010E94BFC481
:10B6E000F80162A373A384A395A360AD71AD82AD8D
:10B6F00093AD0E947FC2A70196010E94BFC40E9421
:10B7000053C2D801D8966D937D938D939C93DB970C
:10B710008DE490E0A196EEADFFADA197E89F80018A
:10B72000E99F100DF89F100D11240354154FD801F7
:10B7300050966D917D918D919C9153970E947FC2FF
:10B74000F80126A537A540A951A90E94E6C11B0111
:10B750002C01F80180819181A281B3810097A1051C
:10B76000B10549F584819581A681B7810097A1052E
:10B77000B10509F580859185A285B3850097A1055E
:10B78000B105C9F4C201B1012091890A30918A0A38
:10B7900040918B0A50918C0A0E94BFC40E94CCC178
:10B7A0000C5B1F4F0E9453C2D8016D937D938D9304
:10B7B0009C93139771C1C201B1012091850A309108
:10B7C000860A4091870A5091880A0E94BFC40E944D
:10B7D000CCC10E9453C22DE430E0A196EEADFFAD86
:10B7E000A197E29F6001E39FD00CF29FD00C11243F
:10B7F0002DEB3AE0C20ED31EB4E46B2E712C6C0C10
:10B800007D1CD3016D937D938D939C9313978090B2
:10B810009D0A90909E0AA0909F0AB090A00A0E9454
:10B820007FC27B018C01F6016081718182819381ED
:10B830000E9481C29B01AC01C801B7010E94BFC434
:10B840007B018C01D60150966D917D918D919C91DB
:10B8500053970E947FC29B01AC01C801B7010E94AF
:10B86000E6C17B018C01C501B4010E947FC29B012E
:10B87000AC01C801B7010E94EDC318162CF4F30106
:10B8800080829182A282B3828090A10A9090A20AC3
:10B89000A090A30AB090A40A8DE490E0A1962EADEA
:10B8A0003FADA197289F6001299FD00C389FD00CF5
:10B8B00011244DEB5AE0C40ED51EA4E46A2E712C5F
:10B8C0006C0C7D1CD3016D917D918D919C910E949A
:10B8D0007FC27B018C01F60164817581868197812D
:10B8E0000E9481C29B01AC01C801B7010E94BFC484
:10B8F0007B018C01D60150966D917D918D919C912B
:10B9000053970E947FC29B01AC01C801B7010E94FE
:10B91000E6C17B018C01C501B4010E947FC29B017D
:10B92000AC01C801B7010E94EDC318162CF4F30155
:10B9300080829182A282B3828090A90A9090AA0A02
:10B94000A090AB0AB090AC0A8DE490E0A1962EAD29
:10B950003FADA197289F6001299FD00C389FD00C44
:10B9600011244DEB5AE0C40ED51EF4E46F2E712C59
:10B970006C0C7D1CD3016D917D918D919C910E94E9
:10B980007FC27B018C01F60164857585868597856C
:10B990000E9481C29B01AC01C801B7010E94BFC4D3
:10B9A0007B018C01D60150966D917D918D919C917A
:10B9B00053970E947FC29B01AC01C801B7010E944E
:10B9C000E6C17B018C01C501B4010E947FC29B01CD
:10B9D000AC01C801B7010E94EDC318162CF4F301A5
:10B9E00080829182A282B3828090A50A9090A60A5A
:10B9F000A090A70AB090A80A8DE490E0A1962EAD81
:10BA00003FADA197289F6001299FD00C389FD00C93
:10BA100011244DEB5AE0C40ED51EE4E46E2E712CB9
:10BA20006C0C7D1CD3016D917D918D919C910E9438
:10BA30007FC27B018C01F6016085718582859385CB
:10BA40000E9481C29B01AC01C801B7010E94BFC422
:10BA50007B018C01D60150966D917D918D919C91C9
:10BA600053970E947FC29B01AC01C801B7010E949D
:10BA7000E6C17B018C01C501B4010E947FC29B011C
:10BA8000AC01C801B7010E94EDC318162CF4F301F4
:10BA900080829182A282B3828DE490E0A1962EAD45
:10BAA0003FADA197289F6001299FD00C389FD00CF3
:10BAB00011244DEB5AE0C40ED51EF601EC5BFF4F8E
:10BAC00060817181828193810E947FC27B018C01A0
:10BAD000A20191010E94E6C1D601D2966D937D9399
:10BAE0008D939C93D597C801B7012DEB37E346E0C2
:10BAF00051E40E94BFC40E944EC2F601648F758F4C
:10BB0000868F978F60908D0A70908E0A80908F0A32
:10BB10009090900AC401B30120E030E040E05FE380
:10BB20000E94BFC45B016C01298D3A8D4B8D5C8DE9
:10BB300029AF3AAF4BAF5CAF4091910A5091920A56
:10BB40006091930A7091940A4DAB5EAB6FAB78AF86
:10BB5000CB01BA0120E030E040E05FE30E94BFC4C7
:10BB60007B018C0169AD7AAD8BAD9CAD9F77A8014F
:10BB700097010E94EDC3181644F4C601B501A8014F
:10BB800097010E94DFC1882314F4860175016D8D31
:10BB90007E8D8F8D98A169AB7AAB8BAB9CAB80917E
:10BBA000950A9091960AA091970AB091980A8DA74C
:10BBB0009EA7AFA7B8ABBC01CD0120E030E040E0CC
:10BBC0005FE30E94BFC41B012C0169A97AA98BA95C
:10BBD0009CA99F77A20191010E94EDC3181644F41D
:10BBE000C801B701A20191010E94DFC1882314F4AA
:10BBF000170128018DE490E0A196AEADBFADA197ED
:10BC0000A89FF001A99FF00DB89FF00D1124E354F7
:10BC1000F54F22A133A144A155A129A33AA34BA3D7
:10BC20005CA3C201B1010E94DFC187FD04C029A04D
:10BC30003AA04BA05CA049A55AA5423051050CF48E
:10BC400005C15091900FCF56DF4F5883C159D04056
:10BC50006091910FCE56DF4F6883C259D0407091EA
:10BC6000920FCD56DF4F7883C359D0408091930F08
:10BC7000CC56DF4F8883C459D040652FCE56DF4F56
:10BC80007881C259D040CD56DF4F8881C359D0400A
:10BC9000CC56DF4F9881C459D04027E137EB41EDB6
:10BCA00058E30E94EDC318160CF0D0C069897A8958
:10BCB0008B899C892091940F3091950F4091960F1C
:10BCC0005091970F0E9405C19B01AC010E94BFC417
:10BCD0007B018C016D897E898F89988D2091980FC9
:10BCE0003091990F40919A0F50919B0F0E9405C17E
:10BCF0009B01AC010E94BFC49B01AC01C801B7010C
:10BD00000E9406C10E942CC57B018C01A4019301F5
:10BD10000E94EDC318165CF00F2EF0E06F2EF0E0DD
:10BD20007F2EF0E88F2EFFE39F2EF02D08C0C40178
:10BD3000B301A80197010E94E6C13B014C0169AD26
:10BD40007AAD8BAD9CAD20919C0F30919D0F4091B1
:10BD50009E0F50919F0F0E9405C17B018C01E894BA
:10BD600017F9C801B7012DA93EA94FA958AD0E94E6
:10BD7000EDC3181694F46DA97EA98FA998ADA801FA
:10BD800097010E94E6C15B016C01C401B301A601E9
:10BD900095010E94DFC1882314F46401530169A94D
:10BDA0007AA98BA99CA92091A00F3091A10F409155
:10BDB000A20F5091A30F0E9405C17B018C01E89452
:10BDC00017F9C801B7012DA53EA54FA558A90E9496
:10BDD000EDC3181694F46DA57EA58FA598A9A801AA
:10BDE00097010E94E6C17B018C01C601B501A80143
:10BDF00097010E94DFC1882314F48601750169A1AF
:10BE00007AA18BA19CA1A80197010E94BFC47B01CC
:10BE10008C01CF56DF4F6881C159D040CE56DF4FDD
:10BE20007881C259D040CD56DF4F8881C359D04068
:10BE3000CC56DF4F9881C459D040A80197010E9489
:10BE4000DFC187FD19C0D801C70102C0D201C101FD
:10BE5000CF56DF4F8883C159D040CE56DF4F9883ED
:10BE6000C259D040CD56DF4FA883C359D040CC56DD
:10BE7000DF4FB883C459D0408DE490E0A196AEADB9
:10BE8000BFADA197A89F8001A99F100DB89F100D6D
:10BE900011240354154FCF56DF4F8881C159D0402C
:10BEA000CE56DF4F9881C259D040CD56DF4FA88182
:10BEB000C359D040CC56DF4FB881C459D040F801A7
:10BEC00082A793A7A4A7B5A762A973A984A995A9D6
:10BED000905820E030E040E050EC0E94BFC4D80110
:10BEE0009E962D913D914D915C91D1970E94BFC43A
:10BEF0002BE037ED43E25BE30E9406C10E942CC5B4
:10BF0000F62EE72ED82EC92ECF56DF4F6881C159A5
:10BF1000D040CE56DF4F7881C259D040CD56DF4F4A
:10BF20008881C359D040CC56DF4F9881C459D04046
:10BF30002F2D3E2D4D2D5C2D0E94DFC187FD14C09D
:10BF4000CF56DF4FF882C159D040CE56DF4FE8823E
:10BF5000C259D040CD56DF4FD882C359D040CC56BD
:10BF6000DF4FC882C459D0408DE490E0A196EEAD79
:10BF7000FFADA197E89F8001E99F100DF89F100D7C
:10BF800011240354154FCF56DF4F8881C159D0403B
:10BF9000CE56DF4F9881C259D040CD56DF4FA88191
:10BFA000C359D040CC56DF4FB881C459D040F801B6
:10BFB00086A397A3A0A7B1A762A173A184A195A10D
:10BFC0002F2D3E2D4D2D5C2D0E94DFC118162CF01B
:10BFD00081E0D801D7968C9302C0F80117AA8DE4AE
:10BFE00090E0A1962EAD3FADA197289FF001299F2B
:10BFF000F00D389FF00D1124E354F54F81E086AB2E
:10C00000A4E9BFE0FE01719680E101900D9281509C
:10C01000E1F78DE490E0A1964EAD5FADA197489F0A
:10C020006001499FD00C589FD00C11246DEB7AE031
:10C03000C60ED71ED6019296ED90FD900D911C91E3
:10C040009597E092900FF092910F0093920F1093BA
:10C05000930F96966D917D918D919C919997A801E2
:10C0600097010E94E6C14B015C01C201B101A80128
:10C0700097010E94E6C18B019C01C601B501A40194
:10C080000E94BD51BBA5B0938D0FC557DF4F2881CE
:10C0900039814A815B81CB58D0402093B90A3093D3
:10C0A000BA0A4093BB0A5093BC0AC957DF4F488174
:10C0B00059816A817B81C758D0404093B50A50931B
:10C0C000B60A6093B70A7093B80ACD57DF4F6881FC
:10C0D00079818A819B81C358D0406093B10A709363
:10C0E000B20A8093B30A9093B40AC158DF4F888193
:10C0F0009981AA81BB81CF57D0408093AD0A90939C
:10C10000AE0AA093AF0AB093B00A0E9447540E94AF
:10C11000AD60C856DF4F0FB6F894DEBF0FBECDBF7F
:10C12000CF91DF911F910F91FF90EF90DF90CF9013
:10C13000BF90AF909F908F907F906F905F904F9047
:10C140003F902F9008951092D80F1092DB0F10920D
:10C15000DE0F0895809389030895EFE6F0E0808173
:10C16000826080830895099A3C9A9A9AEAE0F1E005
:10C170008081806180838081846080830D9A159A9C
:10C180000F9A179A3A9A429A989AA09A8081826056
:10C1900080839FB7F894EBE0F1E080818260808338
:10C1A0009FBF0898109A0C98149A3F98479A0A983B
:10C1B000129A0E98169A3D98459A0B9A1398159ACA
:10C1C0003E9A4698179A389A4098429AEAE0F1E0E7
:10C1D0008081806480839FB7F894EBE0F1E08081F8
:10C1E0008F7B80839FBFA09AEAE0F1E0808181602D
:10C1F00080839FB7F894EBE0F1E080818E7F8083AD
:10C200009FBF9FB7F894EBE0F1E08081826080836C
:10C210009FBFA1E8B0E08C918F7E8C938C91886059
:10C220008C93E0E8F0E080818D7F808380818E7F39
:10C23000808380818F73808380818F7C80838C91C9
:10C24000887F82608C9380E090E490938900809353
:10C2500088001092850010928400EFE6F0E0808163
:10C260008260808381E080938903789408951F938E
:10C27000FC011FB7F89480819181A281B3818093E2
:10C28000B20F9093B30FA093B40FB093B50FFB010F
:10C2900080819181A281B3818093B60F9093B70F73
:10C2A000A093B80FB093B90FFA0180819181A28158
:10C2B000B3818093BA0F9093BB0FA093BC0FB09340
:10C2C000BD0FF90180819181A281B3818093BE0F5E
:10C2D0009093BF0FA093C00FB093C10F1FBF1F91CA
:10C2E0000895FC012FB7F89480819181A281B381D8
:10C2F0008093BE0F9093BF0FA093C00FB093C10F58
:10C300002FBF0895E82F8FB7F894F0E0EE0FFF1FCE
:10C31000EE0FFF1FEE54F04F208131814281538197
:10C320008FBFB901CA01089580916F008D7F8093FE
:10C330006F0006C080918E0F8F5F8F7080938E0F7D
:10C3400090918D0F80918E0F981751F41092A50F38
:10C350001092A40F80916F00826080936F00089507
:10C3600090918D0F80918E0F981751F3E3CF90919C
:10C370008D0F80918E0F981739F00E94AC6E0E943D
:10C380001D190E9443BDF3CF08950E94B761159A0D
:10C39000179A429AA09A9FB7F894EBE0F1E0808157
:10C3A000826080839FBF08951F920F920FB60F92F5
:10C3B0000BB60F921124AF92BF92CF92DF92EF9201
:10C3C000FF920F931F932F933F934F935F936F931E
:10C3D0007F938F939F93AF93BF93CF93DF93EF930D
:10C3E000FF938091A40F9091A50F892B09F08EC126
:10C3F00090918D0F80918E0F981719F4E0E0F0E086
:10C4000014C080918E0F90E02DE430E0829FF00107
:10C41000839FF00D929FF00D1124E354F54FE45BE0
:10C42000FF4F81E08083EC54F040F093A50FE09340
:10C43000A40F309709F464C1E45BFF4F81E080836F
:10C44000EC54F0401092E70F1092E80F1092E90FB1
:10C450001092EA0F60AD71AD2CE96134720718F0EB
:10C4600060E47CE904C03EE46132730730F0769505
:10C4700067957695679584E007C047E26131740758
:10C4800030F07695679582E08093E00F07C0809347
:10C49000E00F6032710510F460E270E060527040AD
:10C4A00058E060307507E8F0472F50E0440F551F03
:10C4B000440F551F455F574F9A012E5F3F4FF901BB
:10C4C000859194919C01AA27639FC001629F810D71
:10C4D0009A1F06948A1F9A1F1124FA0145915491BC
:10C4E0001EC0CB01969587958C7F855F934FFC018D
:10C4F00045915491FC01329625913491862F90E01C
:10C5000087709070FC012E9FC0012F9F900D3E9F61
:10C51000900D1124B3E096958795BA95E1F7481BE5
:10C52000590B44365105A8F4E5ECF2E007C08091C0
:10C53000C00085FFFCCF31969093C600908199236F
:10C54000B1F78FE398E04AE050E00E94E33944E617
:10C5500050E05093EC0F4093EB0FE091A40FF0915B
:10C56000A50F64AD75AD7093E60F6093E50FFCE920
:10C5700061347F0718F060E47CE904C02EE4613286
:10C58000720730F0769567957695679584E007C0D9
:10C5900037E26131730730F07695679582E08093DA
:10C5A000E00F08C081E08093E00F6032710510F465
:10C5B00060E270E06052704048E060307407E8F07C
:10C5C000472F50E0440F551F440F551F455F574FED
:10C5D0009A012E5F3F4FF901859194919C01AA2702
:10C5E000639FC001629F810D9A1F06948A1F9A1F44
:10C5F0001124FA01459154911EC0CB01969587955F
:10C600008C7F855F934FFC0145915491FC013296DC
:10C6100025913491862F90E087709070FC012E9FB9
:10C62000C0012F9F900D3E9F900D112433E09695F1
:10C6300087953A95E1F7481B590B44365105A8F404
:10C64000E5ECF2E007C08091C00085FFFCCF319699
:10C650009093C60090819923B1F78FE398E04AE068
:10C6600050E00E94E33944E650E0CA01A0E0B0E0A7
:10C670008093E10F9093E20FA093E30FB093E40F48
:10C680005093890040938800E091A40FF091A50F8A
:10C6900080899189A289B389B695A7959795879541
:10C6A000B095A095909581959F4FAF4FBF4F8093C8
:10C6B000C20F9093C30FA093C40FB093C50F809384
:10C6C000C60F9093C70FA093C80FB093C90F809364
:10C6D000CA0F9093CB0FA093CC0FB093CD0F809344
:10C6E000CE0F9093CF0FA093D00FB093D10F109295
:10C6F000D20F1092D30F1092D40F1092D50F06C004
:10C7000080ED97E09093890080938800C091A40FFA
:10C71000D091A50F209709F450C588A18093D60F1A
:10C720009091890380FF3AC0119A8FEF809385031F
:10C73000992309F46EC020B1217031E0232759F10B
:10C740008091D70F882339F188819981AA81BB8193
:10C75000181619061A061B06F4F48091B20F909170
:10C76000B30FA091B40FB091B50F8093A60F909323
:10C77000A70FA093A80FB093A90F3093D80F888963
:10C780009989AA89BB898093D20F9093D30FA093E4
:10C79000D40FB093D50F2093D70F3BC0119831E041
:10C7A000309385039923A9F180B18695869580956C
:10C7B000282F217080FF2BC08091D90F882339F159
:10C7C00088819981AA81BB81181619061A061B0651
:10C7D000F4F48091B20F9091B30FA091B40FB09187
:10C7E000B50F8093A60F9093A70FA093A80FB093B7
:10C7F000A90F3093D80F88899989AA89BB8980931A
:10C80000D20F9093D30FA093D40FB093D50F209352
:10C81000D90F8091D60F9091890381FF3EC0449833
:10C820008FEF80938603992309F474C080B18295B9
:10C830008F708095282F217080FF2CC08091DA0F97
:10C84000882341F18C819D81AE81BF811816190624
:10C850001A061B06FCF48091B60F9091B70FA091B9
:10C86000B80FB091B90F8093AA0F9093AB0FA0931C
:10C87000AC0FB093AD0F81E08093DB0F888999896D
:10C88000AA89BB898093D20F9093D30FA093D40F22
:10C89000B093D50F2093DA0F3DC0449A31E0309326
:10C8A00086039923B9F180B1829586958695837028
:10C8B0008095282F217080FF2BC08091DC0F88236A
:10C8C00039F18C819D81AE81BF81181619061A0637
:10C8D0001B06F4F48091B60F9091B70FA091B80F9A
:10C8E000B091B90F8093AA0F9093AB0FA093AC0FA8
:10C8F000B093AD0F3093DB0F88899989AA89BB89E2
:10C900008093D20F9093D30FA093D40FB093D50FF1
:10C910002093DC0F8091D60F9091890382FF39C05C
:10C92000A29A8FEF80938703992309F46EC020E0C9
:10C9300037992CC021E08091DD0F882339F188855B
:10C940009985AA85BB85181619061A061B06F4F4E4
:10C950008091BA0F9091BB0FA091BC0FB091BD0F09
:10C960008093AE0F9093AF0FA093B00FB093B10F21
:10C970002093DE0F88899989AA89BB898093D20F79
:10C980009093D30FA093D40FB093D50F2093DD0FC6
:10C990003CC0A29831E0309387039923B1F186B16E
:10C9A0008295869587708095282F217080FF2BC0F7
:10C9B0008091DF0F882339F188859985AA85BB8509
:10C9C000181619061A061B06F4F48091BA0F9091F6
:10C9D000BB0FA091BC0FB091BD0F8093AE0F909391
:10C9E000AF0FA093B00FB093B10F3093DE0F8889D3
:10C9F0009989AA89BB898093D20F9093D30FA09372
:10CA0000D40FB093D50F2093DF0F8091D60F99A14B
:10CA100083FF12C0913031F49FB7F89480910B01DD
:10CA20008B7F05C09FB7F89480910B018F7E809318
:10CA30000B019FBF8FEF11C0913031F49FB7F89475
:10CA400080910B01846005C09FB7F89480910B0121
:10CA5000806180930B019FBF81E08093880360E039
:10CA600070E08CC18091C00087FF19C04091C60062
:10CA7000E0913B08F0913C0831969F012F77307090
:10CA8000319780913D0890913E082817390739F079
:10CA9000E554F84F408330933C0820933B082881AD
:10CAA00039814A815B818091C20F9091C30FA0911F
:10CAB000C40FB091C50F280F391F4A1F5B1F209369
:10CAC000C20F3093C30F4093C40F5093C50F12167B
:10CAD0001306140615066CF5139A88899989AA8994
:10CAE000BB89281B390B4A0B5B0B2093C20F309379
:10CAF000C30F4093C40F5093C50F2091B20F3091D4
:10CB0000B30F4091B40F5091B50F809185039927D1
:10CB100087FD9095A92FB92F820F931FA41FB51FD2
:10CB20008093B20F9093B30FA093B40FB093B50F4F
:10CB300013982C813D814E815F818091C60F909129
:10CB4000C70FA091C80FB091C90F280F391F4A1FF6
:10CB50005B1F2093C60F3093C70F4093C80F5093AD
:10CB6000C90F12161306140615066CF5469A888925
:10CB70009989AA89BB89281B390B4A0B5B0B209327
:10CB8000C60F3093C70F4093C80F5093C90F209121
:10CB9000B60F3091B70F4091B80F5091B90F8091F7
:10CBA0008603992787FD9095A92FB92F820F931F90
:10CBB000A41FB51F8093B60F9093B70FA093B80F23
:10CBC000B093B90F4698288539854A855B85809151
:10CBD000CA0F9091CB0FA091CC0FB091CD0F280F21
:10CBE000391F4A1F5B1F2093CA0F3093CB0F40930E
:10CBF000CC0F5093CD0F12161306140615066CF5C4
:10CC0000409A88899989AA89BB89281B390B4A0BC4
:10CC10005B0B2093CA0F3093CB0F4093CC0F5093F4
:10CC2000CD0F2091BA0F3091BB0F4091BC0F5091A6
:10CC3000BD0F80918703992787FD9095A92FB92F64
:10CC4000820F931FA41FB51F8093BA0F9093BB0F41
:10CC5000A093BC0FB093BD0F40982C853D854E85A9
:10CC60005F858091CE0F9091CF0FA091D00FB091A2
:10CC7000D10F280F391F4A1F5B1F2093CE0F30930F
:10CC8000CF0F4093D00F5093D10F121613061406F6
:10CC900015060CF04DC089A1813031F49FB7F8948E
:10CCA00080910B01816005C09FB7F89480910B01C2
:10CCB000806480930B019FBF88899989AA89BB8969
:10CCC000281B390B4A0B5B0B2093CE0F3093CF0FF1
:10CCD0004093D00F5093D10F2091BE0F3091BF0FD2
:10CCE0004091C00F5091C10F80918803992787FD13
:10CCF0009095A92FB92F820F931FA41FB51F809362
:10CD0000BE0F9093BF0FA093C00FB093C10F89A126
:10CD1000813031F49FB7F89480910B018E7F05C06C
:10CD20009FB7F89480910B018F7B80930B019FBF7D
:10CD30008091D20F9091D30FA091D40FB091D50FC5
:10CD40000196A11DB11D8093D20F9093D30FA09394
:10CD5000D40FB093D50F2091D20F3091D30F4091C3
:10CD6000D40F5091D50F6F5F7F4F88899989AA8919
:10CD7000BB89281739074A075B0738F48091E00F11
:10CD800090E0681779070CF46DCE2091D20F3091A6
:10CD9000D30F4091D40F5091D50F8C899D89AE89C6
:10CDA000BF8982179307A407B50708F4E3C0E09092
:10CDB000E10FF090E20F0091E30F1091E40FAC8CC3
:10CDC000BD8CCE8CDF8CA8019701C601B501AA27C6
:10CDD000279FB12D389FF001489FF00D479FE00D30
:10CDE000F11D289FB00DE11DFA1F379FB00DE11D09
:10CDF000FA1F469FB00DE11DFA1F369FB10DEA1FC5
:10CE0000FA1FB695EA1FFA1F11248CAD9DAD8E0F47
:10CE10009F1F9093E60F8093E50F28AD39AD4AAD83
:10CE20005BADA0E0B0E0281739074A075B0720F4A4
:10CE30003093E60F2093E50F6091E50F7091E60FB8
:10CE40008CE96134780718F060E47CE904C09EE462
:10CE50006132790730F0769567957695679584E02D
:10CE600007C0E7E261317E0730F07695679582E092
:10CE70008093E00F08C081E08093E00F603271057D
:10CE800010F460E270E060527040F8E060307F07BC
:10CE9000E8F0472F50E0440F551F440F551F455FE2
:10CEA000574F9A012E5F3F4FF901859194919C0154
:10CEB000AA27639FC001629F810D9A1F06948A1F53
:10CEC0009A1F1124FA01459154911EC0CB019695E9
:10CED00087958C7F855F934FFC0145915491FC01B0
:10CEE000329625913491862F90E087709070FC01E6
:10CEF0002E9FC0012F9F900D3E9F900D1124B3E0F7
:10CF000096958795BA95E1F7481B590B443651051C
:10CF1000A8F4E5ECF2E007C08091C00085FFFCCFEB
:10CF200031969093C60090819923B1F78FE398E0F2
:10CF30004AE050E00E94E33944E650E05093890013
:10CF4000409388009A0140E050E08091E10F909179
:10CF5000E20FA091E30FB091E40F820F931FA41F83
:10CF6000B51F8093E10F9093E20FA093E30FB0936E
:10CF7000E40FFEC02091D20F3091D30F4091D40F17
:10CF80005091D50F888D998DAA8DBB8D82179307EF
:10CF9000A407B50708F0E4C06091E70F7091E80FAF
:10CFA0008091E90F9091EA0F2C8D3D8D4E8D5F8D14
:10CFB000AA27639FB12D749FF001849FF00D839F7A
:10CFC000E00DF11D649FB00DE11DFA1F739FB00DC0
:10CFD000E11DFA1F829FB00DE11DFA1F729FB10D76
:10CFE000EA1FFA1FB695EA1FFA1F11248091E50F78
:10CFF0009091E60F8E179F0738F4C05CDF4F688171
:10D000007981C054D04003C0BC016E1B7F0BC05C53
:10D01000DF4F288139814A815B81CB01A0E0B0E0FC
:10D0200082179307A407B50708F4B901FCE9613436
:10D030007F0718F060E47CE904C02EE461327207D7
:10D0400030F0769567957695679584E007C037E26E
:10D050006131730730F07695679582E08093E00F39
:10D0600008C081E08093E00F6032710510F460E247
:10D0700070E06052704048E060307407E8F0472F7D
:10D0800050E0440F551F440F551F455F574F9A01FD
:10D090002E5F3F4FF901859194919C01AA27639FD0
:10D0A000C001629F810D9A1F06948A1F9A1F112446
:10D0B000FA01459154911EC0CB01969587958C7FBE
:10D0C000855F934FFC0145915491FC013296259167
:10D0D0003491862F90E087709070FC012E9FC001E4
:10D0E0002F9F900D3E9F900D112423E096958795DC
:10D0F0002A95E1F7481B590B44365105A8F4E5EC95
:10D10000F2E007C08091C00085FFFCCF319690937C
:10D11000C60090819923B1F78FE398E04AE050E090
:10D120000E94E33944E650E0509389004093880020
:10D130009A0140E050E08091E70F9091E80FA091B4
:10D14000E90FB091EA0F820F931FA41FB51F8093C0
:10D15000E70F9093E80FA093E90FB093EA0F08C090
:10D160008091EB0F9091EC0F909389008093880051
:10D170002091D20F3091D30F4091D40F5091D50F01
:10D18000E091A40FF091A50F80899189A289B389BC
:10D19000281739074A075B0780F01092A50F1092F5
:10D1A000A40F90918D0F80918E0F981731F0809180
:10D1B0008E0F8F5F8F7080938E0FFF91EF91DF91B5
:10D1C000CF91BF91AF919F918F917F916F915F911F
:10D1D0004F913F912F911F910F91FF90EF90DF9012
:10D1E000CF90BF90AF900F900BBE0F900FBE0F90DF
:10D1F0001F9018958091D80F882349F48091DB0FF8
:10D20000882329F48091DE0F882309F49CC0EBE089
:10D21000F0E1949108C08091C00085FFFCCF90930D
:10D22000C600319694919923B1F7EDE4F0E1949121
:10D2300008C08091C00085FFFCCF9093C600319656
:10D2400094919923B1F78091D80F8823F1F06091E0
:10D25000A60F7091A70F8091A80F9091A90F0E941F
:10D2600081C22091610A3091620A4091630A509113
:10D27000640A0E94E6C1AB01BC0189E490E10E940E
:10D28000E31C89E390E10E9469BC8091DB0F882355
:10D29000F1F06091AA0F7091AB0F8091AC0F90915B
:10D2A000AD0F0E9481C22091650A3091660A4091BB
:10D2B000670A5091680A0E94E6C1AB01BC0185E390
:10D2C00090E10E94E31C85E290E10E9469BC80919C
:10D2D000DE0F8823F1F06091AE0F7091AF0F809157
:10D2E000B00F9091B10F0E9481C22091690A3091D4
:10D2F0006A0A40916B0A50916C0A0E94E6C1AB0128
:10D30000BC0181E290E10E94E31C81E190E10E9476
:10D3100069BCE8EDF2E007C08091C00085FFFCCF5A
:10D3200031969093C60090819923B1F78091C00007
:10D3300085FFFCCF8AE08093C6001092D80F109230
:10D34000DB0F1092DE0F089560E070E08FE793E44A
:10D3500020918E0330918F0340919003509191035F
:10D360000E94E6C1DC019B01AC0120933610309392
:10D3700037104093381050933910CB0180933A10F6
:10D3800090933B10A0933C10B0933D100895FC0186
:10D3900097FF03C08091131003C0EF5EFF4E8081A2
:10D3A00090E008951092EE0F1092ED0F1092111070
:10D3B00074981092F00F1092EF0F1092121075984F
:10D3C0001092F20F1092F10F10921310A598089579
:10D3D0001F93182F0E94D2690E94CA17882309F050
:10D3E00036C0ECE5F0E1949108C08091C00085FF63
:10D3F000FCCF9093C600319694919923B1F78FE3B7
:10D4000098E0612F70E04AE050E00E94B9398091C5
:10D41000C00085FFFCCF8AE08093C600EBEBF0E113
:10D42000949108C08091C00085FFFCCF9093C60006
:10D43000319694919923B1F78091C00085FFFCCF7C
:10D440008AE08093C6008EEA90E10E9478BC0E9438
:10D4500075181F9108951F93182F0E94D2690E947A
:10D46000CA17882309F036C0ECE5F0E1949108C0B2
:10D470008091C00085FFFCCF9093C60031969491B7
:10D480009923B1F78FE398E0612F70E04AE050E014
:10D490000E94B9398091C00085FFFCCF8AE080935B
:10D4A000C600E5EFF0E1949108C08091C00085FFCF
:10D4B000FCCF9093C600319694919923B1F7809157
:10D4C000C00085FFFCCF8AE08093C60088EE90E123
:10D4D0000E9478BC0E9475181F9108951F920F92A8
:10D4E0000FB60F920BB60F9211242F933F934F93C9
:10D4F0005F936F937F938F939F93AF93BF93EF93BC
:10D50000FF9390919E03992391F480911110809341
:10D510001B108111749A8091121080931A1081113E
:10D52000759A80911310809319108111A59A80919A
:10D530001B10981708F0749880911A10981708F02B
:10D54000759880911910981708F0A5989F5F9F779C
:10D5500090939E0380911C10833009F450C0843056
:10D5600028F48130F9F08230D8F50DC0853009F407
:10D5700071C0853008F45FC0863009F487C08730F9
:10D5800009F08FC087C088E080937B0080E480939F
:10D590007C0080917A00806480937A000E94DB8E08
:10D5A00081E01BC08091780090917900A0E0B0E00C
:10D5B0002091291030912A1040912B1050912C105D
:10D5C000280F391F4A1F5B1F2093291030932A1000
:10D5D00040932B1050932C1082E080931C1061C05C
:10D5E00088E080937B0082E480937C0080917A00C5
:10D5F000806480937A000E94DB8E83E0EECF80917E
:10D60000780090917900A0E0B0E020911D10309159
:10D610001E1040911F1050912010280F391F4A1FD3
:10D620005B1F20931D1030931E1040931F105093CA
:10D63000201084E0D2CF88E080937B0081E4809347
:10D640007C0080917A00806480937A000E94DB8E57
:10D6500085E0C3CF8091780090917900A0E0B0E0A0
:10D6600020912510309126104091271050912810BC
:10D67000280F391F4A1F5B1F209325103093261057
:10D68000409327105093281086E0A7CF0E94DB8E8E
:10D6900087E0A3CF10921C1080912D108F5F809394
:10D6A0002D1080912D10803108F479C080911410D4
:10D6B0008823C1F48091291090912A109093F40F3F
:10D6C0008093F30F80912510909126109093F60F80
:10D6D0008093F50F80911D1090911E109093001073
:10D6E0008093FF0F81E08093141010922D10109200
:10D6F000291010922A1010922B1010922C101092B8
:10D7000025101092261010922710109228101092B7
:10D7100021101092221010922310109224101092B7
:10D720001D1010921E1010921F10109220102091A8
:10D73000F30F3091F40F80919A0390919B03281777
:10D7400039071CF080E00E942B6A2091F30F309182
:10D75000F40F8091151090911610821793071CF00A
:10D7600080E00E94E8692091F50F3091F60F8091DA
:10D770009C0390919D03281739071CF081E00E94BB
:10D780002B6A2091F50F3091F60F80911710909130
:10D790001810821793071CF081E00E94E869FF913E
:10D7A000EF91BF91AF919F918F917F916F915F9119
:10D7B0004F913F912F910F900BBE0F900FBE0F9086
:10D7C0001F901895EF92FF920F931F93E090F70F21
:10D7D000F090F80F0091F90F1091FA0F6091ED0F92
:10D7E0007091EE0F882777FD8095982F0E9481C257
:10D7F00020E030E040EA51E40E9405C19B01AC0109
:10D80000C801B7010E94DFC1882394F4C801B701A1
:10D810000E944EC270930610609305100E94571329
:10D820006093091070930A1080930B1090930C1062
:10D83000E090FB0FF090FC0F0091FD0F1091FE0F98
:10D840006091EF0F7091F00F882777FD8095982FEA
:10D850000E9481C220E030E040EA51E40E9405C10C
:10D860009B01AC01C801B7010E94DFC1882394F479
:10D87000C801B7010E944EC2709308106093071050
:10D880000E94571360930D1070930E1080930F1029
:10D89000909310101F910F91FF90EF9008952F9289
:10D8A0006F927F928F929F92AF92BF92CF92DF92B0
:10D8B000EF92FF920F931F93DF93CF93CDB7DEB715
:10D8C00029970FB6F894DEBF0FBECDBF8C01E62EB0
:10D8D00061E06E1568F5ECE5F0E1949108C0809187
:10D8E000C00085FFFCCF9093C60031969491992398
:10D8F000B1F78FE398E06E2D70E04AE050E00E94AF
:10D90000B939E2E2F1E1949108C08091C00085FF4D
:10D91000FCCF9093C600319694919923B1F78091F2
:10D92000C00085FFFCCF8AE08093C6000E94B71834
:10D93000AE2DB0E0FD01EE0FFF1FE95FFB4F8081D0
:10D94000918199878887892B09F49FC0A55FBB4F78
:10D950009C919B832224239479C0222D30E0A9013D
:10D96000440F551F440F551FE885F985E40FF51F37
:10D9700085919491081719070CF067C0C9010197A8
:10D98000880F991F880F991FFC013296A885B985C9
:10D99000EA0FFB1FC590D4908A0F9B1FFC01659175
:10D9A00074917A836983FA013296EA0FFB1FE5903E
:10D9B000F490FD01E40FF51FA590B490B6018827FF
:10D9C00077FD8095982F0E9481C26C837D838E8322
:10D9D0009F8389819A81081B190BB801882777FDDD
:10D9E0008095982F0E9481C23B014C01EC18FD08E4
:10D9F0000027F7FC0095102FC801B7010E9481C2D3
:10DA00009B01AC01C401B3010E94BFC47B018C0126
:10DA1000A981BA81AA1ABB0ACC24B7FCC094DC2C19
:10DA2000C601B5010E9481C29B01AC01C801B701CA
:10DA30000E94E6C19B01AC016C817D818E819F813A
:10DA40000E9406C1E62F692F09C02394BB812B16C3
:10DA500008F483CFE0E070E080E060E0FB812F1607
:10DA600079F5E22DF0E0EE0FFF1FEE0FFF1F32976A
:10DA700068857985E60FF71F65917491882777FD92
:10DA80008095982F0E9481C219C0B801882777FD20
:10DA90008095982F0E9481C220E030E04AEF5EE33B
:10DAA0000E94BFC420E030E040E85DE30E94BFC4B4
:10DAB00020E030E040E050E00E9406C1E62F692FF0
:10DAC0002E2F372F482F562FB901CA0129960FB68E
:10DAD000F894DEBF0FBECDBFCF91DF911F910F91A4
:10DAE000FF90EF90DF90CF90BF90AF909F908F907E
:10DAF0007F906F902F900895CF92DF92EF92FF92D8
:10DB00000F931F9360E070E08FE793E420918E0302
:10DB100030918F0340919003509191030E94E6C190
:10DB2000E0919F03F091A0030F2EF0E0EF2EF0E0C4
:10DB3000FF2EF0E00F2FF0E01F2FF02DE0922E10BF
:10DB4000F0922F1000933010109331109B01482F4A
:10DB5000592F20933610309337104093381050933C
:10DB60003910F093A203E093A103E0923210F092F7
:10DB700033100093341010933510CB01DA018093E9
:10DB80003A1090933B10A0933C10B0933D106C9AC8
:10DB90006D9A9D9A8091010180618093010187E0D7
:10DBA00061E070E00E94CD1787ED80937A001092BB
:10DBB0007E0010927D0080917D00816080937D00C9
:10DBC00080917D00826080937D0080917D008460E3
:10DBD00080937D0080E888BD80916E008460809392
:10DBE0006E006AEF70E080E090E00E94651385E0CF
:10DBF00090E090933F1080933E1009C080911510E3
:10DC00009091161040969093161080931510809165
:10DC100015109091161060E00E944F6C20E030E0EB
:10DC200040EA50E40E94DFC187FDE8CF83E191E044
:10DC30009093A00380939F0309C080919A039091D1
:10DC40009B03409790939B0380939A0380919A0340
:10DC500090919B0360E00E944F6C20E030E849E81F
:10DC600053E40E94EDC3181644F385E090E09093CE
:10DC700041108093401009C08091171090911810A6
:10DC800040969093181080931710809117109091E0
:10DC9000181061E00E944F6C20E030E040EA50E450
:10DCA0000E94EDC3181644F383E191E09093A20320
:10DCB0008093A10309C080919C0390919D0340979C
:10DCC00090939D0380939C0380919C0390919D036E
:10DCD00061E00E944F6C20E030E849E853E40E9484
:10DCE000EDC3181644F31F910F91FF90EF90DF9052
:10DCF000CF9008958091F30F9091F40F60E00E940F
:10DD00004F6C6093F70F7093F80F8093F90F909317
:10DD1000FA0F8091F50F9091F60F61E00E944F6C21
:10DD20006093FB0F7093FC0F8093FD0F9093FE0F99
:10DD300080E090E0A0E0B0E08093011090930210AA
:10DD4000A0930310B09304100E943E898FB7F894FB
:10DD5000109214108FBF08952F923F924F925F92AE
:10DD60006F927F928F929F92AF92BF92CF92DF92EB
:10DD7000EF92FF920F931F93DF93CF93CDB7DEB750
:10DD800065970FB6F894DEBF0FBECDBF809114101B
:10DD9000882309F436C20E947A6E87EF9FE09A8B3F
:10DDA000898BADEEBFE0B88BAF87E9E0F0E1FC878F
:10DDB000EB8781E190E19A878987AAE4B0E1B8878F
:10DDC000AF83ECE4F0E1FE83ED8384E690E19C8395
:10DDD0008B83ACE6B0E1BA83A9831D8A1C8A1E86B8
:10DDE0001D86EFE3F1E1B491BB8BE989FA8960808C
:10DDF000718082809380AF85B8896D917C918827EE
:10DE000077FD8095982F0E9481C2A40193010E9402
:10DE100005C17B018C01EC89FD89EE5BFF4E6083BF
:10DE200071838283938320E030E040E251E40E94DA
:10DE3000EDC318162CF421E0EF81F8852083E6C0AD
:10DE4000C801B70120E030E040E251EC0E94DFC1A0
:10DE500088232CF4E1E0AF81B885EC93C2C0AF8198
:10DE6000B8858C91882369F080E090E0A0E0B0E074
:10DE7000ED81FE8180839183A283B383AF81B885D6
:10DE80001C92C801B70120918A0330918B03409105
:10DE90008C0350918D030E94BFC41B012C01EC899F
:10DEA000FD89EC5AFF4E6083718382839383C8019E
:10DEB000B701ED81FE8120813181428153810E9431
:10DEC00006C15B016C01EC89FD89E25DFF4EE080DB
:10DED000F18002811381A80197010E94DFC187FDB3
:10DEE00012C0EC89FD89EA5CFF4EE080F18002817E
:10DEF0001381C601B501A80197010E94EDC3181650
:10DF000014F086017501AD81BE81ED92FD920D93F5
:10DF10001C931397C801B70120918E0330918F0392
:10DF200040919003509191030E94BFC45B016C012A
:10DF3000EC89FD89E45AFF4E608371838283938369
:10DF4000C401B301EB81FC81208131814281538185
:10DF50000E9405C120919203309193034091940354
:10DF6000509195030E94BFC420ED3CEC4CE45DE36E
:10DF70000E94BFC47B018C01A981BA816D917D9102
:10DF80008D919C9123E333E343E75FE30E94BFC499
:10DF90009B01AC01C801B7010E9406C17B018C0145
:10DFA000E981FA816083718382839383AB81BC8131
:10DFB0006D927D928D929C921397C201B101A60140
:10DFC00095010E9406C1A80197010E9405C17B012D
:10DFD0008C0120E030E040E050E00E94DFC1882367
:10DFE0005CF40F2EF0E0EF2EF0E0FF2EF0E00F2FAC
:10DFF000F0E01F2FF02D14C0C801B70120E030E081
:10E0000040E853E40E94EDC3181654F40F2EF0E0DC
:10E01000EF2EF0E0FF2EF0E80F2FF3E41F2FF02D8E
:10E02000ED85FE85E25CFF4E60817181882777FD7A
:10E030008095982F0E9481C29B01AC01C401B3015D
:10E040000E94EDC31816F4F4ED85FE85E156FC4FF1
:10E0500060817181882777FD8095982F0E9481C209
:10E060009B01AC01C401B3010E94DFC1882354F4B9
:10E07000C801B7010E944EC275956795E985FA857A
:10E08000608303C0A985BA851C92EB85FC858081DD
:10E090009181A281B3810097A105B10509F45DC00A
:10E0A0000E945713AB85BC852D913D914D915C919C
:10E0B000621B730B840B950B61547C49804090402C
:10E0C00008F44BC0ED85FE85EB5FFF4E60817181EA
:10E0D000665F7F4F882777FD8095982F0E9481C2C9
:10E0E0009B01AC01E989FA89608171818281938108
:10E0F0000E94DFC188235CF5AF85B8891D921C9210
:10E1000085E491E10E9469BC9B89EFE3F1E108C0DD
:10E110008091C00085FFFCCF9093C600319694910A
:10E120009923B1F7E9EDF2E007C08091C00085FFC7
:10E13000FCCF31969093C60090819923B1F78091DE
:10E14000C00085FFFCCFBAE0B093C60006C0EB85E7
:10E15000FC85108211821282138289899A89049621
:10E160009A8B898BAC89BD891496BD8BAC8BEF855E
:10E17000F8893296F88BEF878D859E8502969E876B
:10E180008D87AB85BC851496BC87AB87E985FA85FE
:10E190003196FA87E9878F819885019698878F83D2
:10E1A000AD81BE811496BE83AD83EB81FC81349634
:10E1B000FC83EB8389819A8104969A838983AC8955
:10E1C000BD89189709F011CE0E9457132091741041
:10E1D000309175104091761050917710621B730B3F
:10E1E000840B950B685873418040904050F00E941A
:10E1F00057136093741070937510809376109093FA
:10E20000771065960FB6F894DEBF0FBECDBFCF91E5
:10E21000DF911F910F91FF90EF90DF90CF90BF9013
:10E22000AF909F908F907F906F905F904F903F90B6
:10E230002F9008952F923F924F925F926F927F920C
:10E240008F929F92AF92BF92CF92DF92EF92FF9206
:10E250000F931F93DF93CF93CDB7DEB7E6970FB63B
:10E26000F894DEBF0FBECDBF6C8F7D8F8E8F9F8FDA
:10E270005EAB4DAB39A328A30E945713698B7A8BF1
:10E280008B8B9C8B2DA93EA9233031051CF4E8EE25
:10E29000F2E019C0EBEFF2E007C08091C00085FF0B
:10E2A000FCCF31969093C60090819923B1F780916D
:10E2B000C00085FFFCCF14C48091C00085FFFCCF57
:10E2C00031969093C60090819923B1F78091C00058
:10E2D00085FFFCCF8AE08093C6000E94D2694DA9D9
:10E2E0005EA957FF74C080E88093131089899A89CA
:10E2F000AB89BC898D879E87AF87B88B89879A87C2
:10E30000AB87BC8719AA1AAA1BAA1CAA1F8A1E8A35
:10E3100091E09D8B1D821E821F82188670E8A72EB9
:10E32000B12CC12CD12C60E8262E312C412C512C43
:10E3300020E030E040E050E029833A834B835C8367
:10E340000F2EF0E06F2EF0E47F2EFCE18F2EF6E42E
:10E350009F2EF02D4DA95EA94F5E5F4E5BA34AA391
:10E36000E9E3F2E154915CA3E4E3F2E184918DA34B
:10E37000EDE2F2E194919EA3E6E2F2E1A491AFA373
:10E38000E0E2F2E1B491B8A7EAE1F2E1249129A731
:10E39000EDE0F2E134913AA7E7E0F2E144914BA7D6
:10E3A000E1E0F2E154915CA7EBEFF1E184918DA7FC
:10E3B000ADA9BEA9AA0FBB1FAA0FBB1FA950B04F82
:10E3C000BFA7AEA7E2ECF1E1B491B8AB07C0EDA9ED
:10E3D000FEA9EF5EFF4E80E8808388CF8091141005
:10E3E000882309F4A3C20E947A6EEDA9FEA9F7FF63
:10E3F0000DC0F0910110F9AB209102102AAB3091C1
:10E4000003103BAB409104104CAB11C0AEA5BFA5AF
:10E41000BC91B9ABEEA5FFA5F181FAABAEA5BFA546
:10E420001296BC91BBABEEA5FFA5F381FCAB698155
:10E430007A818B819C8129A93AA94BA95CA90E9468
:10E44000EDC3181644F089A99AA9ABA9BCA9898380
:10E450009A83AB83BC83C401B30129A93AA94BA910
:10E460005CA90E94DFC187FD06C089A99AA9ABA952
:10E47000BCA93C014D012D89222309F451C069A991
:10E480007AA98BA99CA92C8D3D8D4E8D5F8D0E9404
:10E49000EDC318160CF04AC20E94571329853A851D
:10E4A0004B855C85621B730B840B950B695873411C
:10E4B0008040904008F43AC2D601C5018219930900
:10E4C000A409B5094DA95EA957FF07C0B595A79541
:10E4D000979587958093131007C0B595A795979545
:10E4E0008795EAA1FBA180830E9457136D877E87E1
:10E4F0008F87988B9B01AC0189859A85AB85BC85FC
:10E50000281B390B4A0B5B0B2D833E834F835887A7
:10E510002C8D3D8D4E8D5F8D29833A834B835C839B
:10E5200069A97AA98BA99CA92C8D3D8D4E8D5F8DF3
:10E530000E94DFC188230CF0F8C10E9457132D857B
:10E540003E854F855889621B730B840B950B695868
:10E5500073418040904008F4E8C10E9457136987D6
:10E560007A878B879C874E895F89452B09F4B8C1D0
:10E57000DC01CB012D853E854F855889821B930B8D
:10E58000A40BB50B2D813E814F815885280F391F73
:10E590004A1F5B1F288F398F4A8F5B8F2D813E81E9
:10E5A0004F815885281B390B4A0B5B0BCA01B901F7
:10E5B000A20191010E9491C5288D398D4A8D5B8DF4
:10E5C0000E94F9C52A0D3B1D4C1D5D1D24313105EE
:10E5D000410551055CF424E1222E312C412C512CB3
:10E5E00094E1A92EB12CC12CD12C1FC059016A0174
:10E5F0003DEEA316B104C104D1042CF08CEEA82E7C
:10E60000B12CC12CD12C41E8A416B104C104D10411
:10E610001CF41501260109C00FEF202E312C412CCE
:10E62000512C2A183B084C085D089CA1E9E3F2E153
:10E6300008C08091C00085FFFCCF9093C600319642
:10E6400094919923B1F78FE398E0B601A5012AE0F0
:10E6500030E00E9484399DA1E4E3F2E108C080919A
:10E66000C00085FFFCCF9093C6003196949199230A
:10E67000B1F78FE398E0B201A1012AE030E00E94F7
:10E6800084399EA1EDE2F2E108C08091C00085FFCF
:10E69000FCCF9093C600319694919923B1F78FE304
:10E6A00098E0B401A30122E030E00E94943A9FA1D7
:10E6B000E6E2F2E108C08091C00085FFFCCF9093B4
:10E6C000C600319694919923B1F78FE398E0498180
:10E6D0005A816B817C8122E030E00E94943A8091E3
:10E6E000C00085FFFCCF8AE08093C6008E899F8999
:10E6F00003970CF4F5C0C201B1010E9481C220E071
:10E7000030E040E850E40E94BFC47B018C01698185
:10E710007A818B819C81A40193010E9405C120ED27
:10E720003FE049E450E40E94BFC420E030E040E014
:10E730005FE30E94BFC49B01AC01C801B7010E9406
:10E74000E6C17B018C01688D798D8A8D9B8D0E943D
:10E7500081C220E030E04AE754E40E94E6C13B0178
:10E760004C0198A5E0E2F2E108C08091C00085FF6D
:10E77000FCCF9093C600319694919923B1F78FE323
:10E7800098E0B801A70122E030E00E94943A99A5F0
:10E79000EAE1F2E108C08091C00085FFFCCF9093D0
:10E7A000C600319694919923B1F78FE398E0B401B4
:10E7B000A30122E030E00E94943A8091C00085FFDE
:10E7C000FCCF8AE08093C600C801B7012AE939E985
:10E7D00049E15FE30E94BFC47B018C019AA5EDE093
:10E7E000F2E108C08091C00085FFFCCF9093C60085
:10E7F000319694919923B1F78091C00085FFFCCFA9
:10E800008AE08093C6009BA5E7E0F2E108C0809112
:10E81000C00085FFFCCF9093C60031969491992358
:10E82000B1F78FE398E0B801A70122E030E00E9441
:10E83000943A8091C00085FFFCCF8AE08093C600A7
:10E840009CA5E1E0F2E108C08091C00085FFFCCF0B
:10E850009093C600319694919923B1F7C801B701FE
:10E86000A80197010E9406C1A40193010E94E6C17C
:10E87000AB01BC018FE398E022E030E00E94943AC3
:10E880008091C00085FFFCCF8AE08093C6009DA5E3
:10E89000EBEFF1E108C08091C00085FFFCCF9093C1
:10E8A000C600319694919923B1F7C801B701A4012C
:10E8B00093010E94BFC420E030E040E05EE30E948C
:10E8C000BFC4AB01BC018FE398E022E030E00E94BE
:10E8D000943A8091C00085FFFCCF8AE08093C60007
:10E8E000D201C1018A0D9B1DAC1DBD1DEDA9FEA964
:10E8F000F7FF07C0B595A795979587958093131057
:10E9000007C0B595A79597958795EAA1FBA1808348
:10E910002E893F892F5F3F4F3F8B2E8B6C8C7D8CD8
:10E920008E8C9F8C31E03D8B01C01D8A6C8D7D8D5E
:10E930008E8D9F8D20E030E040EA51E40E9406C1B8
:10E940009B01AC0169A97AA98BA99CA90E94EDC37E
:10E9500018169CF4E2EDF1E1949108C08091C0009A
:10E9600085FFFCCF9093C600319694919923B1F71F
:10E970008091C00085FFFCCFB3C00E945713298946
:10E980003A894B895C89621B730B840B950B615D23
:10E9900077408040904008F454C04DA95EA957FFCD
:10E9A00011C060911310ECECF1E1949108C08091DA
:10E9B000C00085FFFCCF9093C600319694919923B7
:10E9C000B1F711C0AAA1BBA16C91E6ECF1E1949161
:10E9D00008C08091C00085FFFCCF9093C60031969F
:10E9E00094919923B1F7162F8FE398E049A95AA97A
:10E9F0006BA97CA922E030E00E94943A98A9E2EC4D
:10EA0000F1E108C08091C00085FFFCCF9093C60063
:10EA1000319694919923B1F78FE398E0612F70E0DC
:10EA20004AE050E00E94B9398091C00085FFFCCFD8
:10EA30008AE08093C6000E945713698B7A8B8B8B78
:10EA40009C8B0E9457137B018C010E9457132D85CC
:10EA50003E854F855889E21AF30A040B150B298568
:10EA60003A854B855C85E21AF30A040B150BE60E1A
:10EA7000F71E081F191F31E8E3163FE4F30632E1E1
:10EA8000030730E0130798F0E5EAF1E1949108C03C
:10EA90008091C00085FFFCCF9093C6003196949181
:10EAA0009923B1F78091C00085FFFCCF19C04E8932
:10EAB0005F8988A199A18417950774F5E4E5F1E1D0
:10EAC000949108C08091C00085FFFCCF9093C60050
:10EAD000319694919923B1F78091C00085FFFCCFC6
:10EAE0008AE08093C600E6960FB6F894DEBF0FBEAC
:10EAF000CDBFCF91DF911F910F91FF90EF90DF90ED
:10EB0000CF90BF90AF909F908F907F906F905F90CD
:10EB10004F903F902F9008950E9443BD5FCCFC0121
:10EB2000118212820895FC018281882311F081E014
:10EB300081830895FC018181811111820895CF9311
:10EB4000DF93DC01AA5ABF4F8C91A655B04082508A
:10EB5000823050F1ED01CD5ADF4FFD01EE58FF4FED
:10EB60008BE1019009928150E1F7FD01EF5AFF4FCF
:10EB7000A059BF4F8D919C911197A057B0409183A0
:10EB80008083ED01CE58DF4FFD01EF56FF4F8BE143
:10EB9000019009928150E1F7A157BF4F8D919C914F
:10EBA00011975F978D939C93DF91CF910895FC010E
:10EBB00083E094E0918380838781882321F0CF01D3
:10EBC00004960E94B13E08950F931F938C010E94FA
:10EBD000B7610E949461C8018D529F4F0E94B13E5F
:10EBE000F801118281E492E10E9446371F910F9152
:10EBF0000895CF92DF92EF92FF920F931F93DF93CE
:10EC0000CF93CDB7DEB76F970FB6F894DEBF0FBEC8
:10EC1000CDBF8C016B010A5A1F4FD8018C9106554C
:10EC20001040882321F49EE2E92EF12C03C08FE4EA
:10EC3000E82EF12CE00EF11E83E094E09A838983A4
:10EC40001C821B8218861D82B7016C5F7F4FCE012C
:10EC50000596A60121E00E94BE45882391F5EDE4CA
:10EC6000F2E1949108C08091C00085FFFCCF9093A1
:10EC7000C600319694919923B1F7E3E5F2E19491BE
:10EC800008C08091C00085FFFCCF9093C6003196EC
:10EC900094919923B1F709C08091C00085FFFCCF02
:10ECA0000894C11CD11C9093C600F6019081992351
:10ECB00099F78091C00085FFFCCF8AE08093C60061
:10ECC0003CC0D801AF56BF4FF801EE58FF4F8BE163
:10ECD00001900D928150E1F7F801E157FF4F005983
:10ECE0001F4FD8018D919C910057104091838083D4
:10ECF000D801AE58BF4FF70134968BE101900D92C9
:10ED00008150E1F700591F4FF70182819381D801AB
:10ED10008D939C9300571040D801AD5ABF4FFE0110
:10ED200035968BE101900D928150E1F70F5A1F4FFC
:10ED30008B819C81F80191838083CE0101960E9492
:10ED4000D7756F960FB6F894DEBF0FBECDBFCF91CB
:10ED5000DF911F910F91FF90EF90DF90CF9008957A
:10ED6000EF92FF920F931F937C018C010D521F4F66
:10ED7000C8010E94613EC8010E94B13EF7011082A5
:10ED80001F910F91FF90EF9008950F931F93FC0137
:10ED900012AA15AA11AA10AA23E034E037A726A7C1
:10EDA000ED5AFF4F108233961082359711821082F0
:10EDB00032932293B3961082339610823597118244
:10EDC000108232932293B396108233961082359735
:10EDD0001182108232932293B09689E18083339618
:10EDE0001082789610823B96108233961082359767
:10EDF00011821082329322937F96108211821282A6
:10EE0000138238961082118212821382E65FF040DC
:10EE10001182128210828F010E501F4FD8011D9255
:10EE20001D921D921C921397E650FF4F81E0808344
:10EE3000EA5FF04015A614A60E94571368577C4E4F
:10EE40008F4F9F4FF80160837183828393831F915B
:10EE50000F910895CF92DF92EF92FF920F931F933D
:10EE6000CF93DF937C016B01DB010D900020E9F76C
:10EE70008D0101501040061B170BE3EDF0E0EE0E84
:10EE8000FF1ED7011C92EDE2FFEFEE0EFF1ECB013D
:10EE90006EE470E00E943F10EC01009731F4F8013D
:10EEA0003197EC0DFD1D86010EC060E270E00E94FE
:10EEB0003F108C010F5F1F4FCE016AE270E00E948D
:10EEC0003F10FC0131978DE081838AE082831382B9
:10EED000C70181539F4FB8010E94C04683ED90E067
:10EEE000E80EF91ED7018C91882319F1EDE7F2E1C4
:10EEF000949108C08091C00085FFFCCF9093C6001C
:10EF0000319694919923B1F7E4E8F2E1949108C025
:10EF10008091C00085FFFCCF9093C60031969491FC
:10EF20009923B1F78091C00085FFFCCF8AE08093E0
:10EF3000C600DF91CF911F910F91FF90EF90DF906E
:10EF4000CF900895CF93DF93EC018A81882309F451
:10EF50003BC0ECEAF2E1949108C08091C00085FFCB
:10EF6000FCCF9093C600319694919923B1F7CA5083
:10EF7000DF4F488159816A817B81C65FD0408FE332
:10EF800098E02AE030E00E946539EAEAF2E19491E3
:10EF900008C08091C00085FFFCCF9093C6003196D9
:10EFA00094919923B1F7C251DF4F488159816A8109
:10EFB0007B818FE398E02AE030E00E946539809100
:10EFC000C00085FFFCCF12C0EAE9F2E1949108C0CD
:10EFD0008091C00085FFFCCF9093C600319694913C
:10EFE0009923B1F78091C00085FFFCCF8AE0809320
:10EFF000C600DF91CF9108952F923F924F925F927A
:10F000006F927F928F929F92AF92BF92CF92DF9238
:10F01000EF92FF920F931F93DF93CF93CDB7DEB79D
:10F02000AC970FB6F894DEBF0FBECDBF5C014B01AD
:10F03000FC018281882309F438C1C5018D529F4F9C
:10F040000E94B13EF50111821A8A1D8A198A188A16
:10F0500083E094E09F878E873DE4C32ED12CCA0CB9
:10F06000DB1C2EE230E0A20EB31EF601B182A082BC
:10F0700022ED3FEFA20EB31EF40180818F3209F022
:10F0800090C0C4016FE270E00E943F107C010894C0
:10F09000E11CF11C3E010894611C711C260122E157
:10F0A000222E312C2C0E3D1E77C0C7016FE270E07E
:10F0B0000E943F106C01009709F481C0E816F90620
:10F0C00008F07DC08C010E191F09C301B701A8010A
:10F0D0000E945F10060D171DF8011082F30107C092
:10F0E0008091C00085FFFCCF31969093C60090813F
:10F0F0009923B1F78091C00085FFFCCFFAE0F0932F
:10F10000C600F201608171816115710519F460E03A
:10F1100070E002C06C5F7F4FC101A30121E00E943B
:10F12000BE45882371F5E8EEF2E1949108C0809124
:10F13000C00085FFFCCF9093C6003196949199232F
:10F14000B1F7FE01319607C08091C00085FFFCCF6A
:10F1500031969093C60090819923B1F7E6EEF2E1E3
:10F16000949108C08091C00085FFFCCF9093C600A9
:10F17000319694919923B1F78091C00085FFFCCF1F
:10F180008DC02EE030E02C0F3D1FF2013183208333
:10F1900076010894E11CF11CE114F10409F085CF1B
:10F1A0000BC08FE490E0A80EB91EF601B182A082D8
:10F1B00021EB3FEFA20EB31ED82C092D02C0DE2C8E
:10F1C0000F2D8DE490E0A80EB91EF501808191818C
:10F1D00023EB3FEFA20EB31E009719F480E090E0FE
:10F1E00001C004966D2D702F0E949046882339F13E
:10F1F000E8EDF2E1949108C08091C00085FFFCCF5A
:10F200009093C600319694919923B1F78D2D902F4C
:10F210009C01F90107C08091C00085FFFCCF3196A9
:10F220009093C60090819923B1F786EF90E0A80EE5
:10F23000B91EF501108211821282138232C0E0ECF5
:10F24000F2E1949108C08091C00085FFFCCF9093BB
:10F25000C600319694919923B1F78D2D902F9C0182
:10F26000F90107C08091C00085FFFCCF31969093D3
:10F27000C60090819923B1F7EEEBF2E1949108C0BA
:10F280008091C00085FFFCCF9093C6003196949189
:10F290009923B1F78091C00085FFFCCF8AE080936D
:10F2A000C600CE010E960E94D775AC960FB6F894A4
:10F2B000DEBF0FBECDBFCF91DF911F910F91FF90A9
:10F2C000EF90DF90CF90BF90AF909F908F907F9006
:10F2D0006F905F904F903F902F9008952F923F92A4
:10F2E0004F925F926F927F928F929F92AF92BF9256
:10F2F000CF92DF92EF92FF920F931F93DF93CF9302
:10F30000CDB7DEB7AD970FB6F894DEBF0FBECDBF59
:10F310005C014B014DA7FC018281882309F4E8C1FF
:10F3200053ED452E512C4A0C5B1CC2010E94B13E8C
:10F33000F50111821A8A1D8A198A188A83E094E0DD
:10F340009F878E874DE4C42ED12CCA0CDB1C8EE225
:10F3500090E0A80EB91EF601B182A08282ED9FEF67
:10F36000A80EB91EF40180818F3209F08CC0C4014F
:10F370006FE270E00E943F107C010894E11CF11CD8
:10F380003E010894611C711C160178C0C7016FE230
:10F3900070E00E943F106C01009709F482C0E816EB
:10F3A000F90608F07EC08C010E191F09C301B701D0
:10F3B000A8010E945F10060D171DF8011082F301CD
:10F3C00007C08091C00085FFFCCF31969093C600A6
:10F3D00090819923B1F78091C00085FFFCCFFAE0BE
:10F3E000F093C600F101608171816115710519F416
:10F3F00060E070E002C06C5F7F4FCE014296A301D7
:10F4000021E00E94BE45882371F5E0E6F3E1949186
:10F4100008C08091C00085FFFCCF9093C600319654
:10F4200094919923B1F7FE01319607C08091C000F5
:10F4300085FFFCCF31969093C60090819923B1F758
:10F44000EEE5F3E1949108C08091C00085FFFCCF08
:10F450009093C600319694919923B1F78091C000A2
:10F4600085FFFCCF15C18EE090E08C0F9D1FF10150
:10F470009183808376010894E11CF11CE114F1046E
:10F4800009F084CF0BC0EFE4F0E0AE0EBF1EF60132
:10F49000B182A08281EB9FEFA80EB91E082DF92C36
:10F4A00001C00E2DF501E35BFF4F9DA5992309F4E3
:10F4B000ADC0608171816115710519F460E070E083
:10F4C00002C06C5F7F4FC201402F5F2D21E00E9480
:10F4D000BE45882309F46AC0E4EEF0E0AE0EBF1E1C
:10F4E000F50140815181628173818AE090E0A80E2C
:10F4F000B91EF501408351836283738382E19FEFDC
:10F50000A80EB91EE0E5F3E1949108C08091C00017
:10F5100085FFFCCF9093C600319694919923B1F763
:10F52000802F9F2D9C01F90107C08091C00085FFAD
:10F53000FCCF31969093C60090819923B1F7E8E40F
:10F54000F3E1949108C08091C00085FFFCCF9093B7
:10F55000C600319694919923B1F78FE398E02AE0A1
:10F5600030E00E9465398091C00085FFFCCF8AE0C1
:10F570008093C600E6EFF0E0AE0EBF1EF5011082EC
:10F58000118212821382EAE3F3E1949108C0809120
:10F59000C00085FFFCCF9093C600319694919923CB
:10F5A000B1F78091C00085FFFCCF97C0E6E2F3E1A0
:10F5B000949108C08091C00085FFFCCF9093C60055
:10F5C000319694919923B1F7802F9F2D9C01F901D9
:10F5D00007C08091C00085FFFCCF31969093C60094
:10F5E00090819923B1F7E4E2F3E1949108C080910E
:10F5F000C00085FFFCCF9093C6003196949199236B
:10F60000B1F78091C00085FFFCCF42C0608171815D
:10F610006115710519F460E070E002C06C5F7F4F06
:10F62000C201402F5F2D26E50E94BE45882309F0C8
:10F6300033C0E0E1F3E1949108C08091C00085FF00
:10F64000FCCF9093C600319694919923B1F7802F07
:10F650009F2D9C01F90107C08091C00085FFFCCF60
:10F6600031969093C60090819923B1F7EEE0F3E1D3
:10F67000949108C08091C00085FFFCCF9093C60094
:10F68000319694919923B1F78091C00085FFFCCF0A
:10F690008AE08093C60028C081E0F5018083ECEF0A
:10F6A000F2E1949108C08091C00085FFFCCF909357
:10F6B000C600319694919923B1F7F40107C0809167
:10F6C000C00085FFFCCF31969093C60090819923AE
:10F6D000B1F78091C00085FFFCCF8AE08093C6001F
:10F6E000802F9F2D0E948CBCCE010E960E94D77554
:10F6F000AD960FB6F894DEBF0FBECDBFCF91DF91B0
:10F700001F910F91FF90EF90DF90CF90BF90AF903F
:10F710009F908F907F906F905F904F903F902F9031
:10F720000895EF92FF920F931F93CF93DF938C0175
:10F73000FC01128285A9882321F0C801C2960E948B
:10F74000B13E6CEAE62EF12CE00EF11EC70160E03E
:10F7500045E30E945B3C882309F5EDE4F2E19491D6
:10F7600008C08091C00085FFFCCF9093C600319601
:10F7700094919923B1F7E2EAF3E1949108C0809162
:10F78000C00085FFFCCF9093C600319694919923D9
:10F79000B1F78091C00085FFFCCF7DC0E801CF5458
:10F7A000DF4FCE01B70141E00E945547882341F564
:10F7B000CE01B70140E00E945547882309F5EDE7E7
:10F7C000F2E1949108C08091C00085FFFCCF909336
:10F7D000C600319694919923B1F7EFE8F3E1949143
:10F7E00008C08091C00085FFFCCF9093C600319681
:10F7F00094919923B1F78091C00085FFFCCF4BC055
:10F80000C801C296BE010E94B241882309F5EDE706
:10F81000F2E1949108C08091C00085FFFCCF9093E5
:10F82000C600319694919923B1F7EFE7F3E19491F3
:10F8300008C08091C00085FFFCCF9093C600319630
:10F8400094919923B1F78091C00085FFFCCF23C02C
:10F8500081E0F8018283EDE4F2E1949108C08091A7
:10F86000C00085FFFCCF9093C600319694919923F8
:10F87000B1F7E4E7F3E1949108C08091C00085FFFF
:10F88000FCCF9093C600319694919923B1F7809163
:10F89000C00085FFFCCF8AE08093C600D801AD5A36
:10F8A000BF4FF801F2968BE101900D928150E1F784
:10F8B000F80180A991A90F5A1F4FF8019183808305
:10F8C00001551040C8018E96035B1F4FF8019183CC
:10F8D0008083DF91CF911F910F91FF90EF9008955A
:10F8E0002F923F924F925F926F927F929F92AF9230
:10F8F000BF92CF92DF92EF92FF920F931F93DF930D
:10F90000CF93CDB7DEB7CC55D0400FB6F894DEBF5D
:10F910000FBECDBF6C01662311F52AEF30E0C20E99
:10F92000D31ED6018C91E6E0FFEFCE0EDF1E8823BA
:10F9300009F4E2C022EF30E0C20ED31ED601ED90F2
:10F94000FD900D911C91EEE0FFEFCE0EDF1E0E94A8
:10F950005713E616F7060807190708F4CDC02AEF73
:10F9600030E0C20ED31ED6011C92E6E0FFEFCE0EB1
:10F97000DF1ED60112968C91882341F4C6010E94A5
:10F98000917BF6018281882309F4B6C000D000D0B3
:10F99000EDB7FEB731967E010894E11CF11CADB7BE
:10F9A000BEB71296FC92EE92119784E792E1938390
:10F9B0008283D6019C968D919C919D97958384839B
:10F9C0000E946E108701EDB7FEB736960FB6F89419
:10F9D000FEBF0FBEEDBF570108C0D8018C9190E06B
:10F9E0000E9422C6F80181938F01F5010190002049
:10F9F000E9F73197EA19FB09802F8E198E176CF3FE
:10FA0000A2E3AA2EB12CAC0CBD1CC50140E050E015
:10FA100060E070E00E94973D9924FDE3EF2EF12C09
:10FA2000EC0EFD1E2E010894411C511CEFE16E2EC0
:10FA3000712C6C0E7D1E7DE6272E72E1372E42C0A2
:10FA4000D8018C9190E00E9422C6F80181938F0129
:10FA5000F70101900020E9F73197EE19FF09802F97
:10FA60008E198E176CF327968FAD27978E3751F12D
:10FA7000C701B20145E050E00E945110009711F516
:10FA800000D000D0EDB7FEB73196ADB7BEB7129635
:10FA90007C926E92119733822282558244820E9418
:10FAA0006E10EDB7FEB736960FB6F894FEBF0FBED8
:10FAB000EDBFC3010E94BF3789E692E10E9446373D
:10FAC00099249394C501B70140E050E00E94CE40D4
:10FAD000181614F48701BCCF992041F48FEF9FEFE3
:10FAE000D6019D969C938E939C9706C0F60184A5A3
:10FAF00095A5019695A784A7C45ADF4F0FB6F89431
:10FB0000DEBF0FBECDBFCF91DF911F910F91FF9050
:10FB1000EF90DF90CF90BF90AF909F907F906F90CD
:10FB20005F904F903F902F9008952F923F924F9269
:10FB30005F926F927F928F929F92AF92BF92CF927D
:10FB4000DF92EF92FF920F931F93DF93CF93CDB786
:10FB5000DEB7CF58D0400FB6F894DEBF0FBECDBF92
:10FB60008C013B016A0184E090E0C80ED91EF801C7
:10FB70007096C757DF4FF983E883C958D040C80152
:10FB80000396CA57DF4F99838883C658D040C85719
:10FB9000DF4F1882C858D04036E6E32EF12CEC0E29
:10FBA000FD1EF7013B96C557DF4FF983E883CB581D
:10FBB000D0402BEF822E912C800E911E9CEFA92E0F
:10FBC000B12CA00EB11E8EE0282E312C2C0E3D1E25
:10FBD000B7E44B2E512C4C0E5D1EC2010496C35748
:10FBE000DF4F99838883CD58D040EDE4F2E19491C2
:10FBF000C157DF4F9883CF58D04049C1F701838563
:10FC0000282F30E0A901487150704031510509F0AA
:10FC10004CC1F4019081913009F447C1923009F44C
:10FC200044C1F701DE0111969081903239F08E2F98
:10FC30008E19883011F48EE28D939D933196C557BD
:10FC4000DF4F88819981CB58D040E817F90761F7D9
:10FC50001C921E86F3018081882329F4C10165E28C
:10FC600073E00E943410C101B3010E943410C1013D
:10FC7000BE016F5F7F4F0E943410C10165E273E0E7
:10FC80000E9434101CA61FA61BA61AA683E094E0AF
:10FC900099A788A7CE018C96B601AE014F5F5F4F42
:10FCA00021E00E94BE45882309F03EC0F401808116
:10FCB0008823D1F5C157DF4F9881CF58D040EDE46C
:10FCC000F2E108C08091C00085FFFCCF9093C60090
:10FCD000319694919923B1F7E7E2F3E007C0809160
:10FCE000C00085FFFCCF31969093C6009081992388
:10FCF000B1F78091C00085FFFCCFFAE0F093C60019
:10FD0000FE01319607C08091C00085FFFCCF31967F
:10FD10009093C60090819923B1F78091C00085FF30
:10FD2000FCCF8AE08093C600C357DF4FA881B9811A
:10FD3000CD58D040FE01BC968BE101900D928150D0
:10FD4000E1F78AA59BA5F2019383828383E094E087
:10FD500091838083C801B101A2010E94957DC201F7
:10FD60000E94D775CE0188960E94D77590C0953EA7
:10FD700009F48DC09E3209F48AC09F3509F487C00A
:10FD8000F8019089992331F09E3209F480C09F35A3
:10FD900009F47DC023FD7BC080E04031510509F4AA
:10FDA00081E0F80183A7882349F4F701808587342F
:10FDB00009F06DC081858E3709F469C0CA57DF4FDD
:10FDC000A881B981C658D040F7018081803241F0C6
:10FDD0008E2F8E19883011F48EE28D9380818D9351
:10FDE0003196C557DF4F88819981CB58D040E817AD
:10FDF000F90759F71C92F4018081882329F5F30152
:10FE000007C08091C00085FFFCCF31969093C6005B
:10FE100090819923B1F7CA57DF4FE881F981C6581D
:10FE2000D04007C08091C00085FFFCCF31969093F1
:10FE3000C60090819923B1F78091C00085FFFCCF67
:10FE4000FAE0F093C60023C0813039F4F5018081D7
:10FE500091810196918380831AC08230C1F4C85782
:10FE6000DF4FF881C858D0402F2F30E0F501808156
:10FE7000918128173907F1F0C857DF4FF881C8582A
:10FE8000D040FF5FC857DF4FF883C858D040C60145
:10FE9000B701C757DF4F48815981C958D0400E94E8
:10FEA000CE4018160CF4AACE05C0F7019081992314
:10FEB00009F05DCFC157DF4F0FB6F894DEBF0FBE1C
:10FEC000CDBFCF91DF911F910F91FF90EF90DF9009
:10FED000CF90BF90AF909F908F907F906F905F90EA
:10FEE0004F903F902F900895EF92FF920F931F93A2
:10FEF000DF93CF93CDB7DEB76F970FB6F894DEBF21
:10FF00000FBECDBF7C018C01035B1F4F815B9F4FF8
:10FF1000F801918380832BEF30E0E20EF31E21E0A5
:10FF2000F70121937F011182108224E03FEFE20E5E
:10FF3000F31E049640E050E060E070E00E94973DC0
:10FF4000F80120813181DE011596F90134968BE1AB
:10FF500001900D928150E1F7F901828193819C8398
:10FF60008B8383E094E09A838983C7016AE373E01B
:10FF70008E010F5F1F4FA8010E94957DC8010E944E
:10FF8000D775F701E450FF4F808191816F960FB6CE
:10FF9000F894DEBF0FBECDBFCF91DF911F910F91BF
:10FFA000FF90EF900895EF92FF920F931F93DF93CE
:10FFB000CF93CDB7DEB76F970FB6F894DEBF0FBE05
:10FFC000CDBF7C018C01035B1F4F815B9F4FF8010C
:10FFD000918380832BEF30E0E20EF31E22E0F701E5
:10FFE000208325E03FEFE20EF31EF701E450FF4FC0
:10FFF00060831182049640E050E060E070E00E946F
:020000021000EC
:10000000973DF80120813181DE011596F901349682
:100010008BE101900D928150E1F7F901828193818A
:100020009C838B8383E094E09A838983C7016AE38E
:1000300073E08E010F5F1F4FA8010E94957DC801DC
:100040000E94D7756F960FB6F894DEBF0FBECDBF76
:10005000CF91DF911F910F91FF90EF900895EF9254
:10006000FF920F931F93DF93CF93CDB7DEB76F97B8
:100070000FB6F894DEBF0FBECDBF7C018BEF90E0D2
:10008000E80EF91EF701108285E09FEFE80EF91ED9
:1000900087010E5C1F4FC80140E050E060E070E057
:1000A0000E94973DDE011596F8018BE101900D92BB
:1000B0008150E1F7F70180A991A99C838B8383E0AC
:1000C00094E09A838983C7016AE373E08E010F5F2E
:1000D0001F4FA8010E94957DC8010E94D7756F9699
:1000E0000FB6F894DEBF0FBECDBFCF91DF911F9149
:1000F0000F91FF90EF900895DF93CF93CDB7DEB7C8
:1001000028970FB6F894DEBF0FBECDBF80913B039A
:1001100090913C03A0913D03B0913E0389839A8363
:10012000AB83BC83FE01319684E690E02081F9998F
:10013000FECF1FBA92BD81BD20BD0FB6F894FA9ACA
:10014000F99A0FBE01968836910511F03196EECFDF
:10015000E1E6FAE02081F999FECF1FBA92BD81BD98
:1001600020BD0FB6F894FA9AF99A0FBE0196883717
:10017000910511F03196EECFE1E5FAE02081F99991
:10018000FECF1FBA92BD81BD20BD0FB6F894FA9A7A
:10019000F99A0FBE01968838910511F03196EECF8D
:1001A000E1E7FAE02081F999FECF1FBA92BD81BD47
:1001B00020BD0FB6F894FA9AF99A0FBE01968839C5
:1001C000910511F03196EECFE5E8FAE02081F9993A
:1001D000FECF1FBA92BD81BD20BD0FB6F894FA9A2A
:1001E000F99A0FBE01968C39910511F03196EECF38
:1001F000E9E8FAE02081F999FECF1FBA92BD81BDEE
:1002000020BD0FB6F894FA9AF99A0FBE0196803A7B
:10021000910511F03196EECFE1E8FAE02081F999ED
:10022000FECF1FBA92BD81BD20BD0FB6F894FA9AD9
:10023000F99A0FBE0196843A910511F03196EECFEE
:10024000E9E9FAE02081F999FECF1FBA92BD81BD9C
:1002500020BD0FB6F894FA9AF99A0FBE0196883A23
:10026000910511F03196EECFEDE4FAE02081F99995
:10027000FECF1FBA92BD81BD20BD0FB6F894FA9A89
:10028000F99A0FBE01968C3A910511F03196EECF96
:10029000EDE8FAE02081F999FECF1FBA92BD81BD49
:1002A00020BD0FB6F894FA9AF99A0FBE0196803BDA
:1002B000910511F03196EECFE1E9FAE02081F9994C
:1002C000FECF1FBA92BD81BD20BD0FB6F894FA9A39
:1002D000F99A0FBE0196843B910511F03196EECF4D
:1002E000E5E9FAE02081F999FECF1FBA92BD81BD00
:1002F00020BD0FB6F894FA9AF99A0FBE0196883B82
:10030000910511F03196EECFEDEBF5E02081F999F2
:10031000FECF1FBA92BD81BD20BD0FB6F894FA9AE8
:10032000F99A0FBE0196843C910511F03196EECFFB
:10033000E8E7F0E12081F999FECF1FBA92BD81BDB7
:1003400020BD0FB6F894FA9AF99A0FBE0196863C32
:10035000910511F03196EECFEAE7F0E12081F999AD
:10036000FECF1FBA92BD81BD20BD0FB6F894FA9A98
:10037000F99A0FBE0196883C910511F03196EECFA7
:10038000ECE7F0E12081F999FECF1FBA92BD81BD63
:1003900020BD0FB6F894FA9AF99A0FBE01968A3CDE
:1003A000910511F03196EECFEEE7F0E12081F99959
:1003B000FECF1FBA92BD81BD20BD0FB6F894FA9A48
:1003C000F99A0FBE01968C3C910511F03196EECF53
:1003D000E0E8F0E12081F999FECF1FBA92BD81BD1E
:1003E00020BD0FB6F894FA9AF99A0FBE01968E3C8A
:1003F000910511F03196EECFE2E8F0E12081F99914
:10040000FECF1FBA92BD81BD20BD0FB6F894FA9AF7
:10041000F99A0FBE0196803D910511F03196EECF0D
:10042000EAE8F3E02081F999FECF1FBA92BD81BDC1
:1004300020BD0FB6F894FA9AF99A0FBE0196843D42
:10044000910511F03196EECFEEE8F3E02081F999B5
:10045000FECF1FBA92BD81BD20BD0FB6F894FA9AA7
:10046000F99A0FBE0196883D910511F03196EECFB5
:10047000E2E9F3E02081F999FECF1FBA92BD81BD78
:1004800020BD0FB6F894FA9AF99A0FBE8B3D9105EC
:1004900019F001963196EECF80913F039091400381
:1004A000A0914103B09142038D839E83AF83B887AF
:1004B000FE01359684E690E02081F999FECF1FBABF
:1004C00092BD81BD20BD0FB6F894FA9AF99A0FBE7D
:1004D0008736910519F001963196EECFEFEAF3E1F8
:1004E000949108C08091C00085FFFCCF9093C60016
:1004F000319694919923B1F7EEE7F5E1949108C014
:100500008091C00085FFFCCF9093C60031969491F6
:100510009923B1F78091C00085FFFCCF8AE08093DA
:10052000C60028960FB6F894DEBF0FBECDBFCF91A0
:10053000DF910895DF93CF93CDB7DEB7E0970FB685
:10054000F894DEBF0FBECDBFDE011196EDE2F4E000
:1005500080E101900D928150E1F7DE015196EDE1CD
:10056000F4E080E101900D928150E1F7DE01919677
:10057000EDE0F4E080E101900D928150E1F7898196
:100580009A81AB81BC818093610A9093620AA093A7
:10059000630AB093640A89899A89AB89BC8980937C
:1005A000510A9093520AA093530AB093540A89A116
:1005B0009AA1ABA1BCA18093710A9093720AA093F7
:1005C000730AB093740A8D819E81AF81B885809340
:1005D000650A9093660AA093670AB093680A8D89AA
:1005E0009E89AF89B88D8093550A9093560AA0933F
:1005F000570AB093580A8DA19EA1AFA1B8A58093C8
:10060000750A9093760AA093770AB093780A898541
:100610009A85AB85BC858093690A90936A0AA093FA
:100620006B0AB0936C0A898D9A8DAB8DBC8D8093CB
:10063000590A90935A0AA0935B0AB0935C0A89A561
:100640009AA5ABA5BCA58093790A90937A0AA0934A
:100650007B0AB0937C0A8D859E85AF85B88980938F
:100660006D0A90936E0AA0936F0AB093700A8D8DF5
:100670009E8DAF8DB8A180935D0A90935E0AA09382
:100680005F0AB093600A8DA59EA5AFA5B8A9809317
:100690007D0A90937E0AA0937F0AB093800A80E03F
:1006A00090E4ACE9B5E48093850A9093860AA09320
:1006B000870AB093880A80E090E8ABE3B5E48093C2
:1006C000890A90938A0AA0938B0AB0938C0A20E03F
:1006D00030E040E050E02093810A3093820A40935A
:1006E000830A5093840A80E29EE4A0E0B0E0809305
:1006F0004D0A90934E0AA0934F0AB093500A20934C
:10070000990A30939A0A40939B0A50939C0A80E07E
:1007100090E0A0EAB1E480938D0A90938E0AA093B2
:100720008F0AB093900A8DEC9CECACECBEE3809306
:10073000910A9093920AA093930AB093940A80E04E
:1007400090E0A0EAB0E48093950A9093960AA09373
:10075000970AB093980A2093C5053093C605409335
:10076000C7055093C8052093C1053093C205409337
:10077000C3055093C4052093BD053093BE05409337
:10078000BF055093C00582ED90E09093791080935F
:10079000781086E490E090937B1080937A1010920A
:1007A0007D1010927C108AEF90E090937F108093E0
:1007B0007E1084E690E090938110809380101092D8
:1007C0008310109282108AE999E9A1EBB1E4809339
:1007D0008A0390938B03A0938C03B0938D0385E8D9
:1007E00094EFA0E1BEE380938E0390938F03A093D8
:1007F0009003B093910380E190E7A9E5B4E480937E
:10080000920390939303A0939403B093950380E095
:1008100090E0A0E8BFE38093960390939703A093A2
:100820009803B0939903E0960FB6F894DEBF0FBE1D
:10083000CDBFCF91DF910895CF93DF93CFEAD3E17E
:10084000FE01949108C08091C00085FFFCCF909379
:10085000C600319694919923B1F7EEE6F5E19491B3
:1008600008C08091C00085FFFCCF9093C6003196F0
:1008700094919923B1F78091C00085FFFCCF8AE065
:100880008093C600FE019491EFEAF3E108C08091E5
:10089000C00085FFFCCF9093C600319694919923B8
:1008A000B1F74091610A5091620A6091630A7091B8
:1008B000640A86E695E10E94E31C4091650A509126
:1008C000660A6091670A7091680A83E695E10E9462
:1008D000E31C4091690A50916A0A60916B0A709119
:1008E0006C0A80E695E10E94E31C40916D0A5091EC
:1008F0006E0A60916F0A7091700A8DE595E10E9411
:10090000E31CE3E4F3E007C08091C00085FFFCCF67
:1009100031969093C60090819923B1F78091C000E1
:1009200085FFFCCF8AE08093C600FE019491EFEA38
:10093000F3E108C08091C00085FFFCCF9093C60012
:10094000319694919923B1F7E3E4F5E1949108C0CD
:100950008091C00085FFFCCF9093C60031969491A2
:100960009923B1F78091C00085FFFCCF8AE0809386
:10097000C600FE019491EFEAF3E108C08091C00047
:1009800085FFFCCF9093C600319694919923B1F7DF
:100990004091510A5091520A6091530A7091540A41
:1009A0008AE395E10E94E31C4091550A5091560A52
:1009B0006091570A7091580A87E395E10E94E31C01
:1009C0004091590A50915A0A60915B0A70915C0AF1
:1009D00084E395E10E94E31C40915D0A50915E0A18
:1009E00060915F0A7091600A81E395E10E94E31CC7
:1009F000E3E4F3E007C08091C00085FFFCCF3196AF
:100A00009093C60090819923B1F78091C00085FF33
:100A1000FCCF8AE08093C600FE019491EFEAF3E1F7
:100A200008C08091C00085FFFCCF9093C60031962E
:100A300094919923B1F7E3E1F5E1949108C0809195
:100A4000C00085FFFCCF9093C60031969491992306
:100A5000B1F78091C00085FFFCCF8AE08093C6008B
:100A6000FE019491EFEAF3E108C08091C00085FF98
:100A7000FCCF9093C600319694919923B1F74091A1
:100A8000710A5091720A6091730A7091740A8AE037
:100A900095E10E94F71C4091750A5091760A609189
:100AA000770A7091780A87E095E10E94F71C4091DF
:100AB000790A50917A0A60917B0A70917C0A84E0ED
:100AC00095E10E94F71C40917D0A50917E0A609149
:100AD0007F0A7091800A81E095E10E94F71CE3E4AF
:100AE000F3E007C08091C00085FFFCCF3196909362
:100AF000C60090819923B1F78091C00085FFFCCF9B
:100B00008AE08093C600FE019491EFEAF3E108C009
:100B10008091C00085FFFCCF9093C60031969491E0
:100B20009923B1F7ECECF4E1949108C08091C000F6
:100B300085FFFCCF9093C600319694919923B1F72D
:100B40008091C00085FFFCCF8AE08093C600FE0143
:100B50009491EFEAF3E108C08091C00085FFFCCFDB
:100B60009093C600319694919923B1F74091850AEC
:100B70005091860A6091870A7091880A83EC94E10B
:100B80000E94E31C4091890A50918A0A60918B0A65
:100B900070918C0A80EC94E10E94E31CE3E4F3E0A2
:100BA00007C08091C00085FFFCCF31969093C600AE
:100BB00090819923B1F78091C00085FFFCCF8AE036
:100BC0008093C600FE019491EFEAF3E108C08091A2
:100BD000C00085FFFCCF9093C60031969491992375
:100BE000B1F7E7E2F4E1949108C08091C00085FF7D
:100BF000FCCF9093C600319694919923B1F78091E0
:100C0000C00085FFFCCF8AE08093C600FE0194916E
:100C1000EFEAF3E108C08091C00085FFFCCF90931C
:100C2000C600319694919923B1F74091810A509171
:100C3000820A6091830A7091840A8EE194E10E9495
:100C4000E31C4091990A50919A0A60919B0A709115
:100C50009C0A8BE194E10E94E31C40914D0A509163
:100C60004E0A60914F0A7091500A88E194E10E9407
:100C7000F71C40918D0A50918E0A60918F0A7091F5
:100C8000900A85E194E10E94E31C4091910A509101
:100C9000920A6091930A7091940A82E194E10E9411
:100CA000E31C4091950A5091960A6091970A7091C1
:100CB000980A8FE094E10E94E31CE3E4F3E007C0AC
:100CC0008091C00085FFFCCF31969093C600908143
:100CD0009923B1F78091C00085FFFCCF8AE0809313
:100CE000C600FE019491EFEAF3E108C08091C000D4
:100CF00085FFFCCF9093C600319694919923B1F76C
:100D0000EDEFF3E1949108C08091C00085FFFCCF26
:100D10009093C600319694919923B1F78091C000C9
:100D200085FFFCCF8AE08093C600FE019491EFEA34
:100D3000F3E108C08091C00085FFFCCF9093C6000E
:100D4000319694919923B1F74091BD055091BE051C
:100D50006091BF057091C00584EF93E10E94E31C90
:100D60004091C1055091C2056091C3057091C405C1
:100D700081EF93E10E94E31C4091C5055091C605A7
:100D80006091C7057091C8058EEE93E10E94E31C47
:100D9000E3E4F3E007C08091C00085FFFCCF31960B
:100DA0009093C60090819923B1F78091C00085FF90
:100DB000FCCF8AE08093C600FE019491EFEAF3E154
:100DC00008C08091C00085FFFCCF9093C60031968B
:100DD00094919923B1F7E0EEF3E1949108C08091EA
:100DE000C00085FFFCCF9093C60031969491992363
:100DF000B1F78091C00085FFFCCF8AE08093C600E8
:100E0000FE019491EFEAF3E108C08091C00085FFF4
:100E1000FCCF9093C600319694919923B1F74091FD
:100E20008A0350918B0360918C0370918D0386ED42
:100E300093E10E94E31C60918E0370918F03809177
:100E40009003909191032DEB37E346E05EE30E941F
:100E5000E6C1AB01BC0183ED93E10E94CF1C609120
:100E600092037091930380919403909195032DEBDD
:100E700037E346E05EE30E94BFC4AB01BC0180EDF6
:100E800093E10E94CF1CE3E4F3E007C08091C0002F
:100E900085FFFCCF31969093C60090819923B1F7DE
:100EA0008091C00085FFFCCF8AE08093C600DF916F
:100EB000CF9108950F931F93DF93CF93CDB7DEB7F4
:100EC00028970FB6F894DEBF0FBECDBF80913F03C9
:100ED00090914003A0914103B09142038D839E8382
:100EE000AF83B887FE01319604E610E0F999FECF92
:100EF00012BD01BDF89A80B580830F5F1F4F083681
:100F0000110511F03196F2CFCE010596BE016F5F4B
:100F10007F4F43E050E00E945110009709F071C1EB
:100F2000E1E6FAE0F999FECF12BD01BDF89A80B56D
:100F300080830F5F1F4F0837110511F03196F2CFF4
:100F4000E1E5FAE0F999FECF12BD01BDF89A80B54E
:100F500080830F5F1F4F0838110511F03196F2CFD3
:100F6000E1E7FAE0F999FECF12BD01BDF89A80B52C
:100F700080830F5F1F4F0839110511F03196F2CFB2
:100F8000E5E8FAE0F999FECF12BD01BDF89A80B507
:100F900080830F5F1F4F0C39110511F03196F2CF8E
:100FA000E9E8FAE0F999FECF12BD01BDF89A80B5E3
:100FB00080830F5F1F4F003A110511F03196F2CF79
:100FC000E1E8FAE0F999FECF12BD01BDF89A80B5CB
:100FD00080830F5F1F4F043A110511F03196F2CF55
:100FE000E9E9FAE0F999FECF12BD01BDF89A80B5A2
:100FF00080830F5F1F4F083A110511F03196F2CF31
:10100000EDE4FAE0F999FECF12BD01BDF89A80B582
:1010100080830F5F1F4F0C3A110511F03196F2CF0C
:10102000EDE8FAE0F999FECF12BD01BDF89A80B55E
:1010300080830F5F1F4F003B110511F03196F2CFF7
:10104000E1E9FAE0F999FECF12BD01BDF89A80B549
:1010500080830F5F1F4F043B110511F03196F2CFD3
:10106000E5E9FAE0F999FECF12BD01BDF89A80B525
:1010700080830F5F1F4F083B110511F03196F2CFAF
:10108000EDEBF5E0F999FECF12BD01BDF89A80B500
:1010900080830F5F1F4F043C110511F03196F2CF92
:1010A000E8E7F0E1F999FECF12BD01BDF89A80B5ED
:1010B00080830F5F1F4F063C110511F03196F2CF70
:1010C000EAE7F0E1F999FECF12BD01BDF89A80B5CB
:1010D00080830F5F1F4F083C110511F03196F2CF4E
:1010E000ECE7F0E1F999FECF12BD01BDF89A80B5A9
:1010F00080830F5F1F4F0A3C110511F03196F2CF2C
:10110000EEE7F0E1F999FECF12BD01BDF89A80B586
:1011100080830F5F1F4F0C3C110511F03196F2CF09
:10112000E0E8F0E1F999FECF12BD01BDF89A80B573
:1011300080830F5F1F4F0E3C110511F03196F2CFE7
:10114000E2E8F0E1F999FECF12BD01BDF89A80B551
:1011500080830F5F1F4F003D110511F03196F2CFD4
:10116000EAE8F3E0F999FECF12BD01BDF89A80B527
:1011700080830F5F1F4F043D110511F03196F2CFB0
:10118000EEE8F3E0F999FECF12BD01BDF89A80B503
:1011900080830F5F1F4F083D110511F03196F2CF8C
:1011A000E2E9F3E0F999FECF12BD01BDF89A80B5EE
:1011B00080830B3D110521F00F5F1F4F3196F2CF59
:1011C000EFEAF3E1949108C08091C00085FFFCCF65
:1011D0009093C600319694919923B1F7E5EBF3E132
:1011E000949108C08091C00085FFFCCF9093C60009
:1011F000319694919923B1F78091C00085FFFCCF7F
:1012000021C00E949A82EFEAF3E1949108C0809194
:10121000C00085FFFCCF9093C6003196949199232E
:10122000B1F7E4E4F3E007C08091C00085FFFCCF94
:1012300031969093C60090819923B1F78091C000B8
:1012400085FFFCCF8AE08093C6000E941C8428960C
:101250000FB6F894DEBF0FBECDBFCF91DF911F91C7
:101260000F91089528E288E190E00FB6F894A895D0
:10127000809360000FBE209360000895A8950895A4
:101280000F931F938C01FC01868160E00E94BD15C5
:1012900081E090E00E94BE13F801868161E00E9427
:1012A000BD1581E090E00E94BE13F801868160E0E8
:1012B0000E94BD1584E690E00E94BE131F910F911D
:1012C0000895CF92DF92EF92FF920F931F93CF93E7
:1012D000DF93D82EC92E282F392FC9018C01C0E0E9
:1012E000D0E0E62EFF24F801878161E00E940A1514
:1012F000B7010C2E02C0759567950A94E2F76170EC
:10130000F80187810E94BD1521960F5F1F4FC830DD
:10131000D10549F78D2D9C2D0E944089DF91CF91F9
:101320001F910F91FF90EF90DF90CF900895CF9293
:10133000DF92EF92FF920F931F93CF93DF93D82EFC
:10134000C92E282F392FC9018C01C0E0D0E0E62E2C
:10135000FF24F801878161E00E940A15B7010C2E75
:1013600002C0759567950A94E2F76170F80187816C
:101370000E94BD1521960F5F1F4FC430D10549F75C
:101380008D2D9C2D0E944089DF91CF911F910F914F
:10139000FF90EF90DF90CF9008951F93CF93DF934E
:1013A000EC01162F8C81642F0E94BD158D818F3F1B
:1013B00019F060E00E94BD158F8584FF05C0CE0145
:1013C000612F0E9461890EC0612F70E084E07595E5
:1013D00067958A95E1F7CE010E949789CE01612F2A
:1013E0000E949789DF91CF911F91089541E00E945B
:1013F000CD8981E090E0089540E00E94CD89089574
:10140000EF92FF920F931F93CF93DF938C017A019A
:101410006770660F660F660F60640E94FC89C0E00B
:10142000D0E0D801ED91FC91D701AC0FBD1F019028
:10143000F081E02DC8016C9119952196C830D10535
:1014400081F7DF91CF911F910F91FF90EF90089559
:10145000FC016089862F8460808B6C60CF010E94C4
:10146000FC890895DF93CF93CDB7DEB728970FB6E9
:10147000F894DEBF0FBECDBF9C01FE013196A5E4FE
:10148000B4E088E00D9001928150E1F7F901838981
:10149000481710F0482F4150E42FF0E0EE0FFF1FE7
:1014A000EC0FFD1F8181680F6068C9010E94FC89F3
:1014B00028960FB6F894DEBF0FBECDBFCF91DF9157
:1014C000089561E00E94FC8980ED97E00E94BE13C0
:1014D0000895CF93DF93EC01423018F08F85886038
:1014E0008F874B8B1C8A222329F0413019F48F857A
:1014F00084608F8780E593EC0E94BE138C8160E04E
:101500000E94BD158E8160E00E94BD158D818F3FC8
:1015100019F060E00E94BD156F8564FD1DC0CE010D
:1015200063E00E94978984E991E10E94BE13CE0195
:1015300063E00E94978984E991E10E94BE13CE0185
:1015400063E00E94978986E990E00E94BE13CE0175
:1015500062E00E94978916C06062CE010E94FC89F9
:1015600084E991E10E94BE136F856062CE010E9402
:10157000FC8986E990E00E94BE136F856062CE010F
:101580000E94FC896F856062CE010E94FC8984E024
:10159000888BCE010E94288ACE010E94618A82E057
:1015A000898BCE0166E00E94FC89DF91CF9108957E
:1015B0006F927F928F92AF92CF92EF920F931F9381
:1015C000DF93CF93CDB7DEB73C01162F842FF30105
:1015D000448325830683E782C086A18682869E8512
:1015E00093879F859487988995879989968761E0E5
:1015F0000E940A15F30185818F3F19F061E00E9476
:101600000A15F301868161E00E940A15112319F081
:10161000F301178603C080E1F3018787C30160E10E
:1016200041E020E00E94698ACF91DF911F910F91E4
:10163000EF90CF90AF908F907F906F9008958F92A2
:10164000AF92CF92EF920F931F93CF93DF93DC0172
:10165000362F542F722F102FAE2C8C2C13961C92D9
:101660001E92129781E494E011969C938E9300D081
:101670000F92EDB7FEB73196CDB7DEB71982118262
:1016800012821382CD0161E0432F2FEF052FE72E49
:10169000C12E0E94D88A0F900F900F900F90DF916B
:1016A000CF911F910F91EF90CF90AF908F900895B1
:1016B000109284100895FC012081822F90E06AE04E
:1016C00070E00E94C4C5CB016AE070E00E94C4C50E
:1016D000805D8093C010822F90E06AE070E00E94ED
:1016E000C4C5805D8093C1101092C21080EC90E15F
:1016F0000895FC01608171818281938120E030E056
:1017000040E251E40E94BFC40E944EC29B0177FF99
:1017100002C08DE201C08BE28093C01037FF03C08E
:10172000309521953F4FC90168EE73E00E94C4C512
:10173000CB016AE070E00E94C4C5805D8093C11057
:10174000C90164E670E00E94C4C5CB016AE070E0A4
:101750000E94C4C5805D8093C210C9016AE070E038
:101760000E94C4C5CB016AE070E00E94C4C5805DE0
:101770008093C3108EE28093C410C9016AE070E0C8
:101780000E94C4C5805D8093C5101092C61080EC85
:1017900090E10895EF92FF920F931F93FC016081F7
:1017A00071818281938120E030E048EC52E40E9414
:1017B000BFC40E944EC27B018C0197FD12C020E184
:1017C00037E240E050E00E94F9C5CA01B9012AE0C1
:1017D00030E040E050E00E94F9C5605D6093C010C9
:1017E00003C08DE28093C01017FF08C010950095CC
:1017F000F094E094E11CF11C011D111DC801B7011A
:1018000028EE33E040E050E00E94F9C5CA01B9017A
:101810002AE030E040E050E00E94F9C5605D60934E
:10182000C110C801B70124E630E040E050E00E945A
:10183000F9C5CA01B9012AE030E040E050E00E9459
:10184000F9C5605D6093C2108EE28093C310C80139
:10185000B7012AE030E040E050E00E94F9C5CA013B
:10186000B9012AE030E040E050E00E94F9C5605D37
:101870006093C410C801B7012AE030E040E050E0B6
:101880000E94F9C5605D6093C5101092C61080EC8F
:1018900090E11F910F91FF90EF900895FC018081DE
:1018A0009181843691055CF064E670E00E94C4C5C5
:1018B000CB016AE070E00E94C4C5805D01C080E297
:1018C0008093C010808191818A3091055CF06AE03C
:1018D00070E00E94C4C5CB016AE070E00E94C4C5FC
:1018E000805D01C080E28093C110808191816AE0B7
:1018F00070E00E94C4C5805D8093C2101092C31036
:1019000080EC90E10895DF93CF930F920F92CDB7C3
:10191000DEB7FC0160817181828193810E944EC299
:101920007A836983CE0101960E944E8C0F900F90AE
:10193000CF91DF910895FC018081918184369105DA
:1019400034F164E670E00E94C4C5CB016AE070E047
:101950000E94C4C5805D8093C010808191816AE03F
:1019600070E00E94C4C5CB016AE070E00E94C4C56B
:10197000805D8093C110808191816AE070E00E9457
:10198000C4C5805D8093C2101092C31024C08A30F9
:101990009105C4F06AE070E00E94C4C5CB016AE022
:1019A00070E00E94C4C5805D8093C01080819181E9
:1019B0006AE070E00E94C4C5805D8093C1101092FF
:1019C000C21009C06AE070E00E94C4C5805D8093C7
:1019D000C0101092C11080EC90E10895EF92FF9238
:1019E0000F931F93FC01E080F18002811381C801F5
:1019F000B70120E030E040E050E00E94EDC318164F
:101A00001CF4C801B70103C0C801B70190580E9477
:101A10004EC27B018C0180E1E81687E2F80680E087
:101A2000080780E01807A4F0C801B70120E137E2F9
:101A300040E050E00E94F9C5CA01B9012AE030E057
:101A400040E050E00E94F9C5605D6093C0100CC09A
:101A500080E28093C01098EEE91693E0F90690E0DA
:101A6000090790E01907A4F0C801B70128EE33E098
:101A700040E050E00E94F9C5CA01B9012AE030E017
:101A800040E050E00E94F9C5605D6093C11008C05D
:101A90008093C11094E6E916F10401051105A4F044
:101AA000C801B70124E630E040E050E00E94F9C5EB
:101AB000CA01B9012AE030E040E050E00E94F9C5D7
:101AC000605D6093C21008C08093C2109AE0E9166E
:101AD000F10401051105A4F0C801B7012AE030E0C6
:101AE00040E050E00E94F9C5CA01B9012AE030E0A7
:101AF00040E050E00E94F9C5605D6093C31002C0F1
:101B00008093C310C801B7012AE030E040E050E004
:101B10000E94F9C5605D6093C4101092C51080ECFE
:101B200090E11F910F91FF90EF900895EF92FF9237
:101B30000F931F93FC01608171818281938120E06A
:101B400030E040E251E40E94BFC40E944EC297FFC1
:101B500002C02DE201C02BE22093C0107B018C015A
:101B600097FF08C010950095F094E094E11CF11CDB
:101B7000011D111DC801B70120E137E240E050E02E
:101B80000E94F9C5CA01B9012AE030E040E050E006
:101B90000E94F9C5605D6093C110C801B70128EECD
:101BA00033E040E050E00E94F9C5CA01B9012AE0E3
:101BB00030E040E050E00E94F9C5605D6093C210E3
:101BC000C801B70124E630E040E050E00E94F9C5CA
:101BD000CA01B9012AE030E040E050E00E94F9C5B6
:101BE000605D6093C310C801B7012AE030E040E0B7
:101BF00050E00E94F9C5CA01B9012AE030E040E096
:101C000050E00E94F9C5605D6093C4108EE280933D
